:020000040000FA
:1000000000F80202A57100001936000095430000B7
:1000100000000000000000000000000000000000E0
:1000200000000000C05C0100085D010019360000FE
:10003000000000000000000019360000DD7900001B
:10004000293300001936000019360000C571000080
:10005000CD4B00008D6C0000A93500009D360000DE
:100060005918000095170000193600001D360000D1
:10007000A14B000069900000457100007171000003
:10008000193600001936000019360000017E000004
:10009000217E0000193600001936000019360000D4
:1000A000B9820000C38200002B33000059700000A9
:1000B00019360000F56C0000000000000000000090
:1000C0000348854600F016FF00480047D9D30000DA
:1000D00000F8020230B50B46014600202022012420
:1000E00009E00D46D5409D4205D31D469540491B6C
:1000F0002546954040191546521E002DF1DC30BDB5
:1001000070B500242546002801DA01244042002968
:1001100001DA01254942FFF7DDFFAC4200D0404241
:10012000002C00D0494270BDF8B5002425460029B6
:1001300004DA0E46012400214042B141002B04DACA
:100140001E46002352420125B34100F0D1FC8C46EB
:1001500017461E46AC4203D0002540428D41AC46B6
:10016000002C02D0002657429E4161463A46334653
:1001700001B0F0BD03460B439B0703D009E008C95B
:10018000121F08C0042AFAD203E00B780370401C47
:10019000491C521EF9D27047D2B201E00270401CD5
:1001A000491EFBD270470022F6E710B513460A46F7
:1001B00004461946FFF7F0FF204610BDCAB2401EA4
:1001C0004178401C8A4202D00029F9D100207047B2
:1001D000421C0178401C0029FBD1801A704730B5C1
:1001E00004460020034600E05B1C934203D2E05C1F
:1001F000CD5C401BF8D030BD30B50546002003462D
:1002000000E05B1C934205D2EC5CC85C201A01D173
:10021000002CF6D130BD00000FB400B58DB00990B0
:100220000B9010A900200091C0430A9000200C9070
:1002300006480690064807906A4609A80F9900F0FC
:10024000C1FC0DB008BC04B018470000E50B00006D
:10025000050C0000FFB5002083B0009050680190AD
:1002600091691446002697680498884705460C99BA
:100270000698084305D009E0A169761C04988847D0
:100280000546216A284688470028F5D1681C03D016
:100290000198C00704D017E00020C04307B0F0BDAC
:1002A0002068011D2160006800900DE00198C007E2
:1002B00004D1009805700098401C0090A169761C3C
:1002C0007F1E049888470546002F1CDD681C1AD045
:1002D000069800280FD0E817C00E401941118A0077
:1002E00006994009511840012A1A096801209040D6
:1002F0000142DBD107E00C980028D7D1216A2846BB
:1003000088470028D2D0E169049888470C980028D3
:1003100007D1002E05DD0198C00702D10098002109
:100320000170A068B84204DD0C98002804D0002FAA
:1003300002D00120C043B1E73046AFE770B50646B2
:1003400011F0D2FF046805460A220021304600F071
:10035000C5FC2C6070BDF8B502464A40D40F42007F
:100360004B0052085B089A4202D2024608461146E8
:100370004A0023D0C30D4A00DDB2120EAD1A202D63
:1003800035DA49020126490AF6058A19002C00D0FF
:10039000524220214F1B1146B9402A411018C20D6C
:1003A0009A4221D0002C17D0012D08DCDA05801AE2
:1003B000D20F8019D207DBB200F0D0FCF8BDDA050D
:1003C000801A012340001B06C01880185A4280186A
:1003D000CA0F1043490007E04908C2071143DA0574
:1003E000801A80194008801800F0B0FCF8BD610048
:1003F0000122511A001BF7E70122D2075140AAE758
:100400000122D2075040A6E7024670B54A40D30FFA
:10041000DB0740002DD04A002AD0010E140E000246
:1004200012020919400A520A8418E501044654438D
:10043000000A120A2E045043A4194219200CC54385
:10044000AA18120C0125AD03521C521912047F394F
:10045000240400D0521C104301D44000491EC2B2F3
:100460000C06C0092018401C4008802A02D003E076
:10047000002070BD40084000002900DA0020184329
:1004800070BD70B502464A40D50F40004A00ED07E6
:1004900040085208002814D0002A12D0C40DD30DF1
:1004A00041020120C0055202490A520AE41A091801
:1004B00012187D34914201D3641C00E04900002CE5
:1004C00001DA002070BD0023914201D3891A034351
:1004D000400849000028F7D100290AD0914202D1F2
:1004E0000121C90705E0914201D2012101E001216A
:1004F000C943E005C018401900F028FC70BD000099
:10050000F0B507460846584087B0C00F0490480031
:100510000E46590040084908BC1A884105D23846A1
:1005200031461E4617460B46024658004008104307
:100530004CD0300D039040055900400D490D0590F9
:10054000401A0290402872DA18030121000B0905B5
:100550000843019004980092002805D00199524266
:100560000020884100920190029840210A1A0199C6
:10057000009800F0EDFA05460C466B4607CB00F0FC
:1005800008FBC0197141039A0E0D0023D71756407E
:100590001A467A40164344D0049A002A2DD0029A73
:1005A000012A039A15DC1205C01A9141012636056D
:1005B000001C7141D20F059ED20700930192029652
:1005C0002A46234600F010FC07B0F0BD38463146FD
:1005D000FAE71605224A0F46B218C01AB7410121A0
:1005E0000905001C4F4100187F4111461818794138
:1005F000E20F10436D19644113E0E2076D081543E3
:100600006408C2071443039A01261205C01A9141D7
:100610003605001C7141CE07400830434908C01818
:1006200051412A46234600F0D2FBCDE7FFE704986C
:1006300001224000C117121A00238B410498314651
:10064000C417381AA141EEE730B40124E40763402F
:1006500030BC55E730B40124E407614030BC4FE7BB
:100660000000E0FFF0B51FB488B00B990998002492
:1006700048400999C00F490049080991C0070B99E2
:100680000090490049080B9109990898A64608432B
:100690001CD00B990A98084318D0099801244000EF
:1006A000420D4800410D099824050003000B20432A
:1006B00009900B980003000B20430B9050181C4925
:1006C0004018002201901446104605E00020014623
:1006D0000DB0F0BD032801DA034600E003239C4679
:1006E000C11A0AAE0AE05F0008ADED5B4F00F75B90
:1006F0007D430027AA187C41491C5B1E6145F2DD41
:10070000410004AB5A522104120C0A43240C401C31
:100710000828DFDB01980290009970460191009053
:10072000059B049A0799069800F05EFBD0E700004D
:100730000DFCFFFFF0B50C465C4085B0E40FE4070C
:1007400003944C0000266408590094464908024668
:100750000296224321D062460A431ED06200570D02
:100760004A000E032303550D012402462C4924059B
:10077000781B1B0B360B4018234326436146009021
:100780001C46501AB44103D30098401C009002E06C
:10079000921800985B41002803DA0020014605B05A
:1007A000F0BD0020012109050746864611E0644698
:1007B0001D46141BB54106D36546521BB341744612
:1007C00007430C43A646CD07400849082843921822
:1007D0005B4105460D43EAD11046184313D06046ED
:1007E000194650407140084306D06046101AB34184
:1007F00006D20122002306E000220123DB0702E0EB
:100800000122D2435310009874460105381C6141FF
:10081000029C039D0019694100F0D9FABFE700006E
:10082000FD0300000122D207002800DB101A002976
:1008300000DB511A814201D8012070470020704727
:100840000122D207002800DB101A002900DB511A10
:10085000814201D201207047002070470122D20757
:10086000002800DB101A002900DB511A814201D355
:1008700001207047002070470122D207002800DBCA
:10088000101A002900DB511A814201D9012070475A
:10089000002070470122D207002800DB101A00292F
:1008A00000DB511A814201D10120704700207047BE
:1008B00010B5002904DB0C460121C9074042A141C3
:1008C000002B04DB1C460123DB075242A341801AA4
:1008D000994101D3012010BD002010BD10B50029A1
:1008E00004DB0C460121C9074042A141002B04DB77
:1008F0001C460123DB075242A341101A8B4101D34E
:10090000012010BD002010BDC217C10F504010B50E
:100910004018CA079623002100F020FA10BD10B538
:1009200000229623114600F019FA10BD0EB5C21729
:10093000C10F5040CA0740180021054B0293019295
:1009400000910A460B4600F04FFA03B000BD0000CC
:10095000330400000EB505490291002100910A46BA
:100960000B46019100F040FA03B000BD33040000D3
:100970003EB5CA17CB0F002450405140C01861410A
:10098000DA07054B0293019200942246234600F0B9
:100990002BFA03B030BD000033040000C20F410049
:1009A00040020123400ADB05D207090EC0187F2947
:1009B00001DA00207047962903DC9623591AC840B3
:1009C00001E096398840002AF4D040427047410047
:1009D00040020122400AD205090E80187F2901DA5F
:1009E00000207047962903DC9622511AC8407047B0
:1009F000963988407047000070B5CD0F4A00090352
:100A00000123090B1B0519430B4BED070024520D65
:100A10009A4201DA002070BD074B34339A4203DC5E
:100A20009A1A00F0A5F802E00449511888402C43B6
:100A3000F1D0404270BD0000FF030000CDFBFFFF7E
:100A400070B5CD0F4A0009030123090B1B0519439B
:100A50000D4BED070024520D9A4202DA00200146A8
:100A600070BD094B34339A4203DC9A1A00F080F8C7
:100A700003E0064BD21800F06BF82C43F0D00022B4
:100A800040428A41114670BDFF030000CDFBFFFFCD
:100A9000C20FD207400040080BD0C10D0723DB0175
:100AA000C91840020905400A1143C2084007114312
:100AB0007047002001467047CB0FDB07490010B597
:100AC000490802460A4307D00A0D07240903E40136
:100AD000090B121B002A01DC002010BDC900440FC5
:100AE0000C43C100E018D205801800F02FF910BDAA
:100AF000F0B51FB40646002082B00546402401919F
:100B000000901BE0019922460F46304600F030F875
:100B1000049A059B801A994110D310461946224623
:100B200000F016F8361A8F41019722460120002165
:100B3000009F00F00DF838184D4100902046641ECB
:100B40000028DFDC019B00982946324607B0F0BD43
:100B500010B5202A04DB0146203A9140002010BD48
:100B6000914020239C1A0346E3401943904010BD56
:100B700010B5202A04DB0846203AD040002110BDE1
:100B80000B46D340D0402024A21A91400843194676
:100B900010BD10B5202A06DBCB170846203A1041BD
:100BA000C1170B4306E00B461341D0402024A21A84
:100BB00091400843194610BD02681378511801602E
:100BC0001846704710B5D16004495161044911625B
:100BD00000211161114600F0ADF910BDB90B000004
:100BE000210F00004268002A08D001680B78491CD8
:100BF000002B03D0521E06C0184670470121C16069
:100C0000881E70474268002A0BD0C3680168002B19
:100C100007D183688B4204D0491E521C06C00020B5
:100C200070470020C04370470FB400B589B00A4632
:100C30000DA9009100230C99002ACB60234B069349
:100C4000234B079301D0042300E00023214A0292A2
:100C5000214A0892019302466B46002000F095FB62
:100C600009B008BC04B01847F0B585B007460020AD
:100C7000C04301901E46002015460C46009102918B
:100C800004903B466A46314604A8FFF7CDFF04991D
:100C900002466018002D05D0002901D0034600E06F
:100CA00023462B6000290ED0002A02DD00998142E4
:100CB00009D0001B019000943B466A4631460294DD
:100CC00004A8FFF7B1FF05B0F0BD0000E50B000080
:100CD000050C0000FFFFFF7F210F0000F7B5009C0F
:100CE0000F4600262578641C002D05D000F014F96D
:100CF0000068405DC007F5D12B2D02D02D2D18D0F6
:100D0000641E39462046029A00F06AFC002F04D087
:100D10003968A14201D10099396071050224002986
:100D20000BDA4042002803DD11F0DEFA0460A00770
:100D3000FEBD012080020643E3E70028F8DA11F047
:100D4000D3FA04600048FEBDFFFFFF7F002904DAEC
:100D5000401C490001D140084000704770B4002495
:100D6000050C05D11024000402D1002921D0112442
:100D7000050E01D100020834050F01D10001241D28
:100D8000850F01D18000A41C002801DB4000641CF9
:100D9000002908D020252E1B0D46F540A14000D08B
:100DA00001212943084301061B1B000ADB1D02D554
:100DB000002070BC7047DB05181880180029F8DA8D
:100DC000401C4900F5D170BC40084000704710B588
:100DD000002B08DA0024401C614192185B411A4341
:100DE00001D14008400010BDF0B51FB482B00546E7
:100DF0000C0003D0084611F05FFA02E011F05CFA33
:100E000020300246009021462846FFF7A1FE049BB1
:100E1000059A04460F4618431143084314D0184658
:100E200010431BD0009840210A1A18460599FFF775
:100E30009FFE05460E46009A05990498FFF788FE26
:100E4000084305D0012004E02046394607B0F0BD34
:100E50000020C11705430E432C43374300990E98D9
:100E60006305401A7905E40A00220C43FD0A0A30A2
:100E700002D500200146E9E70105101969410C9CE3
:100E80000D9D00196941FFF7A2FFDFE74A00090342
:100E90000123090B1B0519430A4B10B5520D9A4249
:100EA00002DA0020014610BD064B34339A4203DCBF
:100EB0009A1AFFF75DFE10BD034BD218FFF748FEEC
:100EC00010BD0000FF030000CDFBFFFF10B500299F
:100ED00004DB0124E40740428C412146002B04DB63
:100EE0001C460123DB075242A341994200D19042A4
:100EF00010BD0000064C0125064E05E0E36807CC56
:100F00002B430C3C98471034B442F7D3FFF7DCF87E
:100F1000005701002057010000487047842C010051
:100F200010B50446FFF7F8FF0068005DC007C00F6A
:100F300010BD0000F3B58DB000200A9001200B9089
:100F4000002608460C300C46099062690121099878
:100F50009047051E2ED0252D2DD0216A88470028C8
:100F600018D06269012109989047216A88470028B2
:100F7000F7D1411E62690998904700E0761CA1698B
:100F80000D988847216A88470028F7D1E1690D98B4
:100F90008847DAE7A1690D9888470746A84201D13A
:100FA000761CD2E7E1690D9888477F1C02D10A9828
:100FB000002877D049E1002762693D463946099803
:100FC00090472A280CD16269012109989047012590
:100FD00006E00A214F433F18303FEBD41020054371
:100FE0006269012109989047014630390A2903D2E4
:100FF0009B498F42DEDCECE7E90600D4994F6C2870
:101000000AD04C2810D0682824D06A282ED0742802
:101010000CD07A280AD00DE0626901210998904726
:101020006C2823D004211CE02020054362690121A3
:1010300009989047A760656065284FD026DC58283E
:1010400039D01ADC452849D012DC252834D0412873
:10105000B0D143E06269012109989047682802D025
:1010600008210D43E6E70120C002DEE70220DCE7AD
:10107000462833D047282CD130E05B2870D0612837
:101080002CD063286CD0642823D161E06F284FD026
:1010900009DC662822D0672820D0692826D06E284F
:1010A00017D12EE0CDE070284DD073286FD0752871
:1010B0004ED078280DD154E0A1690D988847054697
:1010C000252800D16CE7E1690D9888476D1C00D197
:1010D0006DE7BAE00A224CE00A2252E001202346E2
:1010E0006A46C0430D9900F050F9A3E0284640211C
:1010F00008436060A807234601D5002239E000229A
:101100003FE0E80700D020E72068011D216000686B
:10111000290501D5067018E7290701D5068014E7CF
:10112000A90703D5F117066041600EE706600CE7DA
:101130002846402108436060A807234601D50822BD
:1011400017E008221DE0484928460840606016E084
:101150002846402108436060A8072346BCD5B9E76C
:1011600015E02846402108436060A80707D52346BC
:1011700010220120C0430D99C046C0465AE02346C4
:1011800010220120C0430D99C046C04652E0002104
:101190000C910B460091632802D05B2807D043E0F6
:1011A000E80601D40120A060012000903CE06269C3
:1011B0000121099890475E2805D101200C90014635
:1011C0006269099890472169002906D10B4601AA56
:1011D0008F00491CD3510829FADB002835D021693A
:1011E00000290ED1C117C90E09184A11930001AA8E
:1011F0009A1849094901411A01201368884003439C
:10120000136062690121099890475D28E5D10C9827
:10121000002808D0002001AB81005A58401CD2435E
:101220005A500828F8DB01AB01202246C0430D9933
:10123000FFF710F800280ADA401C06D10B980028A6
:1012400003D00020C0430FB0F0BD0A98FBE7E907C8
:1012500002D10A99491C0A91361800200B9074E6B5
:10126000CCCCCC0CFFFFFF7FF1F7FFFFFFB5087878
:1012700089B01546FF2805D0491C2D2804D000222E
:10128000002407E000240BE00122F9E70A235C4375
:101290000419491C0878FF28F8D1002A00D06442BC
:1012A000002004902A7801462D2A01D02B2A0FD144
:1012B0006D1C2D2A02D00022049209E00122FBE7D6
:1012C00000260A2233466D1C00F0DDF93818714102
:1012D0002F78FF2FF4D10C9AA218069202460A43E7
:1012E00004D0FF23069A9133DA4205DA00210998E7
:1012F0000A4606C00DB0F0BD0024B74AB54D2646DB
:10130000079200F00DFA029006980391002801DA86
:10131000474200E0074639050020AF4A001C514112
:101320000191009012E0F80707D022462B46304684
:101330000799FFF797F90646079122462B46104674
:101340001946FFF78FF904460D467F10002FEAD1AA
:101350000698019B0028009A0399029806DAFFF785
:10136000E9F93246079BFFF7E5F905E0FFF77AF95F
:101370003246079BFFF776F9049A002A02D0012231
:10138000D2075140099A03C2B4E7FFB591B00020DB
:1013900009900025ED432E209E685C681F46019051
:1013A000B9696D1C129888470090396A88470028EF
:1013B000F6D10098401C0AD00D20C0018443002EB5
:1013C00012DD00982B2809D02D280DD103E0002034
:1013D000C04315B0F0BD012080020443B9696D1C03
:1013E00012988847761E009003A9600501D52D202C
:1013F00000E02B206A461073491C0CA80F91029044
:101400000AE0B9696D1C12988847009001204002DB
:1014100004431398761E0560002E02DD00983028E4
:10142000EFD001990098884245D18020044308E01C
:101430000998401E09900120400204431399681C3A
:101440000860B9696D1C761E129888470090302894
:10145000EED030E00199884205D1200603D48020E7
:101460000443761E1DE0009811F00CF8002825D0EA
:10147000012149020C43009807AA0F990332303822
:10148000761E914208D208700F98401C0F902006DB
:1014900007D50998401E03E0200602D40998401C95
:1014A0000990A00502D51399681C0860B9696D1CE4
:1014B000129888470090002ECCDC59E0002E57DDB2
:1014C0000098652801D0452852D1A00550D50320A9
:1014D00000028443B9696D1C761E129888470090FB
:1014E000002E0CDD2B2804D02D2808D1FF20013040
:1014F0000443B9696D1C12988847761E0090E00578
:1015000001D52D2100E02B21029801700298401C8A
:101510000290019025E00120400204430EA90298A8
:101520000131761E88420ED20098029930380006AA
:10153000000E087003D10299019881420AD90298DD
:10154000401C029006E0E00501D5244801E0234854
:1015500040420990B9696D1C129888470090139811
:101560000560002E04DD009810F08CFF0028D2D119
:10157000F969129888470F99FF200870029903AA09
:10158000087000200A900B900CA90AA8099BFFF78D
:101590006DFEA00502D40120C0431AE724200442B6
:1015A00009D0E00713D138680B9A0A99031D3B60F4
:1015B000006806C00BE00B990A98FFF77DFA014618
:1015C000E00704D13868021D3A60006801602846CF
:1015D000FFE60000000014400000F03FF1D8FFFFDC
:1015E000F7B582B0029C00272078641C154601974D
:1015F000302802D0002D15D015E020780127641C7A
:10160000782804D0582802D0002D09D00BE0002DF6
:1016100001D0102D07D1002710252078641C02E08E
:10162000082500E00A250026009610E00099012711
:1016300069430818020C294680B2714300908E1845
:101640003804864201D3012001902078641C294689
:1016500000F056F80028E9DA0398002805D0002F9A
:1016600001D0641E00E0029C04600198002806D0AE
:1016700010F03AFE02210160C81E05B0F0BD0099CD
:1016800030040843F9E7F0B51FB486B0002000909D
:10169000019002900698069980B204900798090C70
:1016A00002040014114307900027089D0998069131
:1016B0003E463C4603900398A9B20204000C0390F6
:1016C00004982D0C1543484300212246FFF740FAA9
:1016D000C719714110340E46402CECDB3846029A93
:1016E000FFF736FA009A019B801800905941029842
:1016F0000191103002904028CCDB00980BB0F0BD77
:101700003A2800D23038202302469A43412A01D396
:1017100010463738884201D30020C043704700008C
:101720000EB5054A02920022009213460192FFF77D
:101730005BFB03B000BD00003304000070B58C18E3
:101740000578401C6B075B0F01D10378401C2A1100
:1017500006D10278401C03E006780E70401C491C3C
:101760005B1EF9D12B0705D40023521E0DD40B703C
:10177000491CFAE70378401CCB1A921C03E01D7841
:101780000D70491C5B1C521EF9D5A142D8D3002014
:1017900070BD000010B52148016A8A0715D44A07B8
:1017A00015D4C90732D01E498A89002A15D0531E84
:1017B0008B8182688C6904C48C610A691B040DD01A
:1017C000002A22D10121016010BD022100E0042184
:1017D000C16113488021416110BD0A69012A09D104
:1017E000026801239A430260C361FF206830993088
:1017F0000C4A106001204861CA69002A05D0886936
:1018000009898B00C01A904710BD10BDFF226832B5
:10181000054806A109A30EF0C9F9C04608D0014049
:10182000A895010280E200E0E43B01004144435FEF
:1018300049525148616E646C65720000556E65785E
:101840007065637465642041444320696E746572F9
:10185000727570740D0A000070B582B00023019398
:10186000444801688A6A4C6813252540132D02D12B
:10187000CB689B07DB0F4361930772D453070AD4ED
:10188000D30711D1130724D5048F838E1C1B102C72
:101890000EDD102310E0042088620220032142A202
:1018A0000FF0E0F902B070BD0120886202B070BD97
:1018B000048F1B1B1C0610D0DBB20024058FC66AE8
:1018C00075192D5D0D74641CA342F7D1048FE318C4
:1018D0000387D20607D400212FE04B6A0824A343D4
:1018E0004B62D206F7D5CB68C28E448F141B5B04C3
:1018F000DB0EA34201D3438FD31ADAB2002A16D0EB
:10190000097D438F046BE1540199012A10D0012312
:101910001C46890145582D7D41184E8F9B19096B36
:10192000CD54641CE3B201999A42F2D800E0002140
:101930008B01C3185C8FA2185A878A0181184B8FBC
:10194000CC8EA3420BD301230B618058002242624C
:10195000CA6B002A03D03A31098801A8904702B027
:1019600070BD02208862044804A1084A08A30EF052
:101970001DF9C04688900102FD3B01004145535FBF
:1019800049525148616E646C65720000CE020000DD
:1019900041455320696E707574206F766572666C70
:1019A0006F770D0A00000000414553206F75747079
:1019B000757420756E646572666C6F770D0A000031
:1019C000F0B581B001243F2900D993E00346806837
:1019D000456B2D688E0001A7BE59B7461B1B000042
:1019E000371B0000131B0000131B0000F51A00003A
:1019F000F51A0000F51A0000F51A0000F51A0000AB
:101A0000F51A0000F51A0000F51A0000F51A00009A
:101A1000F51A0000491B0000651B0000F51A0000C4
:101A2000F51A0000F51A0000F51A0000F51A00007A
:101A3000F51A0000F51A0000F51A0000F51A00006A
:101A4000F51A0000F51A0000F51A0000F51A00005A
:101A5000F51A0000F51A0000F51A0000F51A00004A
:101A6000F51A0000F51A0000F51A0000F51A00003A
:101A7000F51A0000F51A0000F51A0000F51A00002A
:101A8000F51A0000F51A0000F51A0000F51A00001A
:101A9000F51A0000F51A0000F51A0000F51A00000A
:101AA000F51A0000F51A0000F51A0000F51A0000FA
:101AB000F51A0000DD1A0000DD1A0000DD1A000032
:101AC000DD1A0000DD1A0000DD1A0000DD1A00003A
:101AD000DD1A0000DD1A0000DD1A0000434800692D
:101AE0000024022809D001280DD0002802D103CA01
:101AF00005F052F8204601B0F0BD03CA05F03EF8EB
:101B0000204601B0F0BD03CA05F05CF8204601B0E4
:101B1000F0BD022931D0022430E0344D00242C6184
:101B20006C619849354A01F0F3FE6869401C6861B0
:101B3000204601B0F0BD01F025FF284602F092F9E1
:101B40000024204601B0F0BD284909690C234B430D
:101B50002749CA58C918496801F0DAFE002420460E
:101B600001B0F0BD0024204604F0E4FF0128C1D1FB
:101B70001E483030204900241CE001241B490F6915
:101B80000C26314679431A4A51188968214208D0F7
:101B900000247D1C15490D614C61052D10D315499C
:101BA00006E012494869401C4861032812D32949BC
:101BB00000241846224602F005F9204601B0F0BD87
:101BC0006E430B498A598919496801F0A1FE2046E4
:101BD00001B0F0BD0E20009000240A2228462146C4
:101BE00002F0E0F8204601B0F0BDC046A099010225
:101BF000882C01009433010074330100F747010081
:101C0000B0B504290FD804468068C04679440979E4
:101C100049008F44020A0E1C1700104910A201F05F
:101C200077FE0020B0BD0120B0BD01F0ABFE00206A
:101C3000B0BD00250321284604F08CFF064920464C
:101C40002A4602E003490022204602F0BBF80020A9
:101C5000B0BDC04684330100043401008813000085
:101C6000415445300D0A0000B0B582B001240A2964
:101C700010D883687944097949008F440E290505F5
:101C80000B0B0B0B0B0B1A00194909680024224699
:101C900002F098F8204602B0B0BD506814490860C0
:101CA000144915A2184601F033FE0024204602B064
:101CB000B0BD0024019403CA09A201AB02F0A0F94F
:101CC0000228E7D1019804F099FF204602B0B0BD88
:101CD000184601F057FE0024204602B0B0BDC046B1
:101CE0002B4353513A2025642C252A0D0A0000006D
:101CF000D89A01028813000041542B4353510D0A16
:101D000000000000B0B582B00546002404F070FF6A
:101D100001280DD108498C60E86B426853684B601C
:101D2000009401926A4602F04DF8204602B0B0BD20
:101D3000E443204602B0B0BDCC930102B0B50546E5
:101D4000881E02280AD3A868012913D0002915D1BA
:101D50000C490DA201F0DCFD0020B0BD02200146BF
:101D600004F0F8FE064900242846224602F02AF82C
:101D70002046B0BD01F006FE0020B0BD0120B0BD80
:101D8000543301008813000041542B4346554E3D07
:101D9000300D0A0080B5E0B00320C101684610F0A4
:101DA00073FA06480078002804D003206A460146EA
:101DB0000EF058FF002060B080BDC046A59801021B
:101DC000F0B597B008201490642013902548109027
:101DD00002200E904B20C0011690234D284614304F
:101DE000129001270F97B802119003200EA906F058
:101DF00061FB0026F443002802D0204617B0F0BD56
:101E00000C35284602F03CF80028F6D180200C90D2
:101E100016490B910A9016480990164808901648E2
:101E200007901648069039200590154804901548EB
:101E300003900D95144D03A9284601F0D3FD002809
:101E4000DBD1009501970F4C104911A2124B20468F
:101E500001F06CFF1149204601F09CFF34462046FA
:101E600017B0F0BD50C001023C97010250C40102FE
:101E7000D0C40102652F0000C52F0000212F0000F3
:101E800014350100D099010260C90102F432010049
:101E9000414952373830450014340100951D000087
:101EA00010B50348002404700FF068FE204610BDF2
:101EB000EC9E010280B501F071F9002080BD0000A8
:101EC000F0B58DB00E4600270C970B970A9709972F
:101ED0000897079706970597029080680490406BD3
:101EE0000068019004F020FE04465BA105220392E5
:101EF000FEF782F95A4D00281ED05AA1052220462D
:101F0000FEF77AF9002817D058A105222046FEF7DF
:101F100073F900280FD059A105222046FEF76CF96D
:101F2000002809D057A105222046FEF765F90028B0
:101F300007D156A500E04FA505A820212A4602F0AA
:101F400031F901203F2E00D936E0C0467E44367973
:101F50007600B7443340474A57313131313131315E
:101F6000313165303131313131313131313131312E
:101F70003131313131313131313131313131313151
:101F8000313131313131313131311F1F1F1F1F1FAD
:101F90001F1F1F1FBE48416A04290CD1039A4262C9
:101FA00087620C2050433D490A580818416805AB28
:101FB000049801F0ADFC38460DB0F0BDB44C0020E3
:101FC0006062A062CD49364A049801F0A1FCA06A83
:101FD000401CA062EFE7049801F0D4FC019801F0E6
:101FE00041FFE8E7AA48406A05E0A949486A01229A
:101FF0000243032A1CD1A649421C4A628F62062A68
:10200000CFD30BE0A2494A6A012013460343052BB4
:10201000D2D1501C48628F62062803D31E490DE0BE
:102020009B48406A0C2141431C4842584018BDE778
:10203000886A401C8862032805D31649002202984A
:1020400001F0C0FEB7E70E20009000210A2201989F
:10205000029B01F0A7FEAEE73436303030000000BE
:102060001F48010034363030320000003436303042
:1020700031000000554E494E455400003436303092
:1020800036000000343630303300000043544E45F3
:1020900054000000F432010044330100C42C01005C
:1020A0009247010070B5022956D30F2907D1784C09
:1020B000217A012905D1002222728F494AE00120AC
:1020C00070BD866801F002FF002004F03BFD01288E
:1020D00003D10020032104F03DFD0025284604F033
:1020E00029FD012804D130346A490022204631E01C
:1020F000304600F0EFFD00282ED03046FFF702FEFC
:10210000002829D004F030FD012807D15F498D60F7
:10211000F06B4268E26252684A601AE0022004F002
:1021200009FD012808D159498D61F06B4268E262CE
:1021300052684A6110310CE0022004F003FD0128CE
:102140000AD152498D62F06B4268E26252684A627B
:1021500020312A4601F036FE002070BD10B582B055
:1021600003460120272931D87944097949008F4451
:102170002C132D2D162D2D2D2D2D2D2D2D2D2D2CC2
:102180002D2D2D2D2D2D2D2D2D2D1C2D2D2D2D2D90
:102190002D2D2D2D2D2D2D2905F0F8F815E0DF49D9
:1021A0000022184601F00EFE0FE00020019003CA45
:1021B00008A201AB01F024FF012806D1019805F027
:1021C00011FA02E0024801210172002002B010BDA4
:1021D000A09901022B51495552433A2022636C6F5A
:1021E000736564222C25640D0A000000B0B5022935
:1021F0004AD30F2914D18568002004F0A3FC0128DC
:1022000003D10020032104F0A5FC0024204604F0A3
:1022100091FC012806D1D94830301E49002231E016
:102220000120B0BD2846FFF76DFD00282CD004F03A
:102230009BFC012808D115498C60E86B4268CF4BA4
:10224000DA6252684A601CE0022004F073FC012844
:1022500009D10E498C61E86B4268C84BDA6252685A
:102260004A6110310DE0022004F06CFC01280BD112
:1022700006498C62E86B4268C04BDA6252684A6277
:102280002031224601F09EFD0020B0BD5490010295
:10229000A09901027433010080B5022905D30429F5
:1022A00005D19E49002201F08DFD002080BD012056
:1022B00080BDC046B0B50546881E02280AD3A8686E
:1022C000012913D0002915D10C490DA201F020FBE2
:1022D0000020B0BD0220032104F03CFC064900248C
:1022E0002846224601F06EFD2046B0BD01F04AFBB3
:1022F0000020B0BD0120B0BD943301008813000060
:1023000041542B4346554E3D310D0A0010B50F295F
:102310000BD001291DD000291DD1FFF7C1FD0020E0
:10232000022104F017FC002010BD0446002004F038
:1023300001FC012803D10020022104F00BFC002045
:1023400004F000FC012804D104490022204601F0D9
:1023500039FD002010BD012010BDC04684330100AE
:10236000F0B581B00124322928D805468768786BFA
:102370000668C0467944097949008F442F3F1919EE
:10238000191F1F1F1F1F1F1F1F1F221F1F1F1F1F60
:102390001F1F1F1F1F1F1F1F1F1F1F1F1F1F1F1F4D
:1023A0001F1F1F1F1F1F1F1F1F1F1F1F1F1F260055
:1023B0001E4900242846224601F004FD204601B0B3
:1023C000F0BD1B48017800291FD018490024284679
:1023D000224601F0F7FC204601B0F0BD0024FC626B
:1023E0003969384688470028FAD011480470FC62E1
:1023F000FFF756FD0E20009001220EE0304601F05E
:1024000031FD0024204601B0F0BD01210170FFF72D
:1024100051FD0E20009000240522304621462B4617
:1024200001F0C0FC204601B0F0BDC04614330100ED
:10243000DC9A010210B586B0034601203B2900D981
:1024400056E0C0467944097949008F4450505151B3
:10245000335151515151515151515151515151518A
:10246000515151515151515151515151515151515C
:10247000515151515151515151515151515151514C
:1024800051391D1D1D1D1D1D0020059003CA02AAE6
:10249000009218A205AB01F0B3FD022827D1039AE0
:1024A000029817A1FDF7A8FE002820D1059805F095
:1024B00099F81CE0B5490022184601F083FC16E0AB
:1024C000002002900590049003CA05AA019204AA74
:1024D00000920DA202AB01F093FD032807D1049AEC
:1024E0000599029805F04AF9029805F0BFF8002016
:1024F00006B010BD25642C2025700D0A00000000D8
:10250000434C4F53454400002B52454345495645E3
:102510002C25642C25643A0D0A25650064330100DE
:10252000012901D80020704701207047B0B5054649
:10253000881E03280BD2104604F01EFB0F48C16A08
:1025400000242846224601F03DFC2046B0BDAC6880
:1025500001290BD000290ED104F0E8FA03460849FE
:1025600008A2204601F0D4F90020B0BD204601F0B9
:1025700009FA0020B0BD0120B0BDC046A0990102FB
:102580008813000025730D0A0000000070B582B0AA
:1025900001240F293DD803468568686B0668C0464C
:1025A0007944097949008F4407141E343434342F98
:1025B000373434343434434E664800240470846124
:1025C000C461012101716649664A284601F0A0F9FB
:1025D0001FE0284601F0D6F9304601F043FC002404
:1025E000204602B070BD5B4800240471826904215A
:1025F00011430278002A2ED0052958D1016A491CBE
:10260000016259D2624961E0524B187800240028D7
:1026100031D0204602B070BD4E4B1878012816D13B
:1026200003CA183351A201F0EBFC002002B070BDC8
:10263000484800248461012101710078484900283C
:1026400012D1484A11E0434E307900281BD00024B3
:10265000204602B070BD052932D10024012101704D
:102660008461C46101713E493F4A284601F050F936
:10267000204602B070BD03CA183340A201F0C0FC6E
:10268000204602B070BD002004F05CFA012803D19E
:102690000020032104F05EFA0024204604F04AFAE8
:1026A000012816D130362D49002430464BE0002158
:1026B0000162C169491CC1610E20009000241CE028
:1026C000C169491CC161652915D3304900241846E8
:1026D00039E02846FFF716FB00289AD004F044FAA8
:1026E000012812D11C4900248C60E86B4268F26218
:1026F00052684A6027E00E200090022230462146B0
:1027000001F050FB204602B070BD022004F012FA26
:10271000012809D1104900248C61E86B4268F262FB
:1027200052684A6110310EE0022004F00BFA0128D1
:1027300000D06EE7084900248C62E86B4268F262C0
:1027400052684A622031224601F03CFB204602B02A
:1027500070BDC046A099010254900102743301007B
:1027600088130000BB470100C64701002B434752B6
:1027700045473A20252A2C25640000002B4352456A
:10278000473A20252A2C256400000000643301000C
:1027900024330100B0B584B001243B2900D937E0CF
:1027A000134605468068C0467944097949008F443C
:1027B0004B5532322F2F2F2F2F2F2F2F2F2F2F2FE1
:1027C0002F2F2F2F2F2F2F2F2F2F2F2F2F2F2F2F19
:1027D0002F2F2F2F2F2F2F2F2F2F2F2F2F2F2F2F09
:1027E0002F2F2F2F2F2F1D1D1D1D1D1D0024039466
:1027F00003CB01AA00921C4A03AB01F001FC0228A2
:1028000006D1029A019819A1FDF7F6FC00280FD015
:10281000204604B0B0BD1848006804F0E3FE174934
:1028200000242846224601F0CDFA204604B0B0BD6F
:102830001148006804F0D6FE10490022284601F035
:10284000C1FA204604B0B0BD0B490B601E210CA29A
:1028500001F05EF80024204604B0B0BD01F092F80B
:102860000024204604B0B0BD1F490100434C4F5323
:1028700045204F4B00000000E09A01023433010074
:1028800041542B434950434C4F53453D25640D0A59
:1028900000000000F0B589B0044601203B2900D9B2
:1028A000AAE01646A7687A6B1568C046794409798C
:1028B00049008F44536AA071A1A1A1A1A1A1A1A126
:1028C000A1A18AA1A1A1A1A1A1A1A1A1A1A1A1A10F
:1028D000A1A1A1A1A1A1A1A1A1A1A1A1A1A1A1A1E8
:1028E000A1A1A1A1A1A1A1A1A1A11D1D1D1D1D1DF0
:1028F0000027089703CE06AA0092414A08AB01F0D0
:102900007FFB022877D13F4805680898854272D13D
:10291000079A069E3CA130460592FDF76DFC002803
:1029200047D03DA13046059AFDF766FC002840D00F
:102930003CA13046059AFDF75FFC0028314E5AD184
:10294000284604F069FE7068401C706003283CD380
:1029500003207060306804F0D7FD36E02948066037
:10296000304604F025FE05902648006804F0F4FD8A
:1029700004902448006804F0FBFD04990191029042
:102980000598012827D02EA026E0384600F0FAFF4F
:10299000284601F067FA2EE01A4D286804F03CFE44
:1029A0006868401C686003280FD300226A602249CF
:1029B0000DE0144E7760284604F044FE306804F0C1
:1029C00083FF002801D01B4900E00C49002220466B
:1029D00001F0F8F90FE019A000901A491AA2384640
:1029E000334600F095FF0E2000900021B4222846C7
:1029F000234601F0D7F9002009B0F0BD34330100BF
:102A00001F490100B4970102414C524541445920ED
:102A1000434F4E4E45435400434F4E4E4543542082
:102A20004F4B0000434F4E4E454354204641494CC6
:102A300000000000D4330100F43201005443500080
:102A4000554450008813000041542B4349505354BF
:102A50004152543D25642C222573222C22257322B9
:102A60002C25750D0A000000B0B582B014468A1EF0
:102A7000022A12D38568012917D000291CD12046CB
:102A800004F05CFD00901E210EA22846234600F0B3
:102A90003FFF0024204602B0B0BD09490024224671
:102AA00001F090F9204602B0B0BD284600F06AFF60
:102AB0000024204602B0B0BD0124204602B0B0BDC3
:102AC000E433010041545E4845415254434F4E4661
:102AD00049473D312C25642C25750D0A0000000066
:102AE000F0B583B014468A1E022A1CD385680129DA
:102AF00021D0002926D1164F3C60204604F010FD5D
:102B0000FDF766FB0646386804F00AFD710800917F
:102B100001901E210FA22846234600F0F9FE002452
:102B2000204603B0F0BD09490024224601F04AF9CD
:102B3000204603B0F0BD284600F024FF00242046C4
:102B400003B0F0BD0124204603B0F0BD34330100D2
:102B5000E49A010241545E48454152544245415471
:102B60004845583D25642C25752C25730D0A000019
:102B7000F0B585B0044601203B2900D988E0A5685E
:102B80007944097949008F444257825E8383838365
:102B90008383838383838383638383838383838325
:102BA00083838383838383838383838383838383F5
:102BB00083838383838383838383838383831D1DB1
:102BC0001D1D1D1D0020049003CA02AA0092314A57
:102BD00004AB01F015FA022859D12F4885680498F2
:102BE000854254D1039E029F2CA138463246FDF700
:102BF00003FB00283DD02BA138463246FDF7FCFAF6
:102C0000002844D1284604F0EDFC29493BE0224C41
:102C1000A260104604F0B8FC002838D001F059FB3F
:102C2000E060002833D0A36840680090234924A2C4
:102C3000284600F06DFE2AE017480021C1602846B2
:102C400000F0A0FE23E01448806804F0CBFC19E0FB
:102C500000F008FF012804D10F48C16803C901F042
:102C600009F80D48C0680CC81349284600F090FECA
:102C70000DE0284604F088FC0028074907D0C96801
:102C800001F0FDFA0B490022204601F09BF80020DC
:102C900005B0F0BD1F490100B497010253454E44F1
:102CA000204F4B0053454E44204641494C00000004
:102CB0006433010034330100204E0000881300000B
:102CC00041542B43495053454E443D25642C2575B2
:102CD0000D0A0000F0B583B0074601F0F7F80026B2
:102CE000304604F05BFC032835460BD1042128460E
:102CF00004F0DAFDF86B51492A4601F063F83046DA
:102D000003B0F0BD02970024204604F047FC0428DD
:102D1000254609D10298C06B49492A4601F052F86C
:102D20002646304603B0F0BD0027384604F036FC96
:102D300005283D4609D10298C06B40492A4601F05A
:102D400041F83E46304603B0F0BD019701252846C4
:102D500004F024FC0328029FC8D00125284604F073
:102D60001DFC0428D6D00125284604F017FC0528B0
:102D7000019FE0D00225284604F010FC0328029FA2
:102D8000B4D00225284604F009FC0428C2D002254C
:102D9000284604F003FC0528019FCCD0254C206870
:102DA000401C0321FDF7ACF90D46084604F0F6FB84
:102DB0000628029F08D1284604F0E6FB002803D02D
:102DC00001F087FA00282AD1681C0321FDF798F941
:102DD0000D46084604F0E2FB062808D1284604F018
:102DE000D3FB002803D001F074FA002817D1681C27
:102DF0000321FDF785F90D46084604F0CFFB0021BD
:102E0000CE43062800D07AE7284604F0BDFB002810
:102E100000D174E701F05DFA002800D16FE725606A
:102E2000F86B05492A4600F0CDFF0026304603B076
:102E3000F0BDC046E89A0102F4330100B43301004A
:102E4000C433010080B58AB0082007906420069042
:102E500009480390022001904B20C0010990C0480E
:102E6000143005900120029080020490032001A9F3
:102E700005F020FB0AB080BD50C00102B0B582B0A1
:102E800001220F293ED803468068446B2468C0465F
:102E90007944097949008F44071F25273435353592
:102EA0003535353535350A152C49002204E02B49D6
:102EB000CA68092A20D8521CCA601649164A00F06E
:102EC00027FD1EE0002003F035FE012819D123481C
:102ED00030300E49002212E000F054FD204600F090
:102EE000C1FF0EE00D4908E00E20009000210122F4
:102EF000204600F057FF04E005490022184600F084
:102F000061FF0022104602B0B0BDC046743301001C
:102F10005433010088130000D2470100043301003C
:102F200080B5032005F0AEFA80BD00000B48406B71
:102F30000249411A484248417047C04634330100B3
:102F40000648416B0020002905D0054A914203D074
:102F500049680029FAD1704701207047A099010201
:102F600044330100B0B514460D460846114601F041
:102F70002EF801281ED1285D00281BD1002C0FD06F
:102F80006019401E00780A280AD17B480078002882
:102F900010D003200A4A01462B460DF063FE09E0DB
:102FA00075480078002805D00320054A01462B46C5
:102FB0000DF058FE03202946224605F04FFBB0BD18
:102FC0005B470100F0B585B0054604A800240470F5
:102FD000E743002D12D0EA68002A0FD0686A002863
:102FE0000CD0A86A002809D0401EE96A814200D3AB
:102FF0008EE004A928469047002803D03C4620468E
:1030000005B0F0BD564EE86A411CE962696A049A4F
:103010000A54E86A696A002202920A54E86A092896
:1030200006D1696A09224D48FDF7D9F800283ED03B
:103030003078411E022908D800F048FFB168401AD4
:103040004849884264D8464E30780A2820D0012862
:1030500023D16E6A3A213046FDF7B0F8002847D0F8
:10306000019002980390E96A03AB30463EA200F05B
:10307000C7FF02284CD10398002849D00A21384ABA
:10308000117001990818696A401AC01C50602FE03D
:103090007068E96A81422BD13AE004A800780A28D6
:1030A0000FD00D2814D101202863E86A1AE001200E
:1030B000307000F00BFFB0603078411E0229BBD9A0
:1030C000C3E7296B012904D102202863E86A03E0E1
:1030D000296BE86A022905D1022817D10298E86213
:1030E000286305E0012803D1686A00783E280FD0E4
:1030F000A86AE96A401E81420AD2EA6804A9284601
:1031000090470028164E00D17DE777E702982863A4
:10311000E96A686A00F05BFF012819D1E86A0028B3
:103120000CD06B6AC018401E00780A2806D11248DD
:10313000007800280CD0032010A206E00E4800788A
:10314000002805D06B6A032010A201460DF08AFD0D
:1031500003480470204605B0F0BDC0469E40010003
:103160003C970102DC0500002B524543454956457A
:103170002C252A2C25643A00A59801025B41542095
:10318000526563765D202573000000005B4154208A
:10319000526563765D2025730D0A000010B5064C5C
:1031A0002078002109F0FAF8044807F07DF820782B
:1031B000012109F0F3F810BDC696010260E3160084
:1031C000B0B50F2001F064FC194D687028703328E9
:1031D0002AD120243721204601F0A6FC21200321FA
:1031E00001F0A2FC2220402101F09EFC23200821B6
:1031F00001F09AFC3020AA2101F096FCE848022157
:103200000187322001F090FC3320012101F08CFC79
:103210005F21204601F088FC0F2001F039FC287066
:103220000A2007F041F8B0BDDD480021C187B0BDDC
:103230000C960102F0B581B0344C212100916172ED
:10324000334909886170D24FFA8962713D6B3D62E2
:10325000304B1B782370090AA170110AA171B9784B
:10326000814207D10BF0C8FB6421FCF733FF3982A0
:10327000B9783D6B28484843284940180A21FCF793
:1032800029FF45197D630BF04DFB40190CF052F8F6
:1032900006460D462248007D0BF0D8FE21490988DC
:1032A0002222A15482B2D20B801802B2D01752103F
:1032B000B2186841130E009D6355130C2025635509
:1032C0003B6EA3761D0AE5761D0C25771B0E6377F2
:1032D00023462233090A5970A277BA65F865BA669F
:1032E000F866100AE0770BF087FB78627B6B282189
:1032F000012220460EF04EFF0BF07EFBF86109F034
:1033000067FC0028FBD1002001B0F0BD0ED4010203
:10331000D4980102A498010280CE0B0040C20C0098
:103320003C900102B098010270477047F0B587B039
:103330004F480068FDF7FAFA04460D464D48406ACA
:10334000FDF7A6FB02460B4620462946FDF7F2F99B
:1033500002460B46002448492046FDF775F90490C3
:10336000039106208E49085EFDF7E0FA0190009176
:103370000120069040020290404F05E04E4908515E
:103380007F1C241D642C70D0387805283C48F5D16A
:1033900005973C4801593C4E31613C480359B360A4
:1033A0003B480059B0613B4A1259326200275D1A0E
:1033B00035637369F1689941069B00DB3B46002B3E
:1033C00001D0029BC918304E7163F369716A101AFB
:1033D0009941069A00DB3A46002A01D0029A8918E0
:1033E000FDF7C6FA02460B4604980399FDF73AF931
:1033F000FDF726FB244A9062D162401BC10F4018A2
:10340000401010601546FDF791FA234A234BFDF753
:1034100029F9A863E963224A224BFDF723F93A46CA
:10342000214BFDF71FF93A46204BFDF769F8054699
:103430000E4615480564416428463A461C4BFDF784
:1034400037FA0028059F9BD1002228463146194BA8
:10345000FDF744FA002893D128463146019A009B93
:10346000FDF74EF8FDF7C8FA88E707B0F0BDC04693
:1034700008970102F02D01000000F03F18980102AA
:10348000FFFF0100A09F01022096010204A001029B
:103490003CE00102A0E00102699006699006903FBD
:1034A00052257997532ED33F0000594000003E40EB
:1034B00000408FC0006AF84028D20102F0B583B006
:1034C0000BF09AFA324CA064E26C831A31498B42B9
:1034D00003D8D24382188A4257D9216C0B1A2E4A3C
:1034E000934252D3C343C91891424ED3E06403F0D0
:1034F00093FBE079411CE1710121084041402172B8
:10350000002840D100F022FD207800281FD0234D54
:103510002B464033002104E06D1C401E9B1C0028FC
:1035200016D02F787E1C2E70092FF5D8CFB27C00D4
:103530001A4A121902921A88019200914021029CA3
:10354000019A62520099154AD655491CE4E70021B8
:103550000F4801701248448F2046FDF7E0F90146FC
:10356000104F3D682846FDF787F906467F20C105C4
:103570002846FCF7F0FE0546601CFDF7C5F9002E55
:1035800000D1284638600EF0F9FA03B0F0BDC0460D
:1035900030990102FF25B80301DC7C01009A010289
:1035A0003AA90102BC980102B0B582B0194C20685A
:1035B000056801A90020087007E090470198401CA9
:1035C00001A90870C0B2082822D20122110481404A
:1035D000294209D02268516080002018826A002A9E
:1035E000ECD001A80121E8E7130283402B4201D06F
:1035F000022104E082402A42E0D0032113462268DF
:103600005360800020188268002AD7D001A8D4E730
:1036100002B0B0BDD8920102FEE7000010B5094823
:103620000168CA6920231343CB610269032A08D1C8
:10363000012293050C689C430C605102C26E0A4340
:10364000C26610BD4C93010281B010B581B00393E6
:10365000002807D0C16A002904D003AB0093C46AD4
:103660000021A04701B010BC01BC01B00047000020
:1036700080B5024608480068002807D091B2120CB5
:1036800003889A4203D040690028F9D180BD002206
:1036900000F0F4FA80BDC0465CC90102F0B581B00B
:1036A0005C4C2068856BE80707D0E168002904D0EE
:1036B00000208847206801218163A80707D5216978
:1036C000002904D00120884720680221816368070F
:1036D00007D56169002904D00220884720680421A9
:1036E0008163280707D5A169002904D003208847F2
:1036F000206808218163E80607D5E169002904D024
:1037000004208847206810218163A80607D5216A14
:10371000002904D00520884720682021816368069D
:1037200007D5616A002904D0062088472068402117
:103730008163280607D5A16A002904D0072088479D
:103740002068802181630126E80507D5E16A002908
:1037500004D037020820884720688763A80507D56A
:10376000216B002904D077020920884720688763ED
:10377000680507D5616B002904D0B7020A20884785
:1037800020688763280507D5A16B002904D0F702BC
:103790000B20884720688763E80407D5E16B002980
:1037A00004D037030C20884720688763A80407D516
:1037B000216C002904D077030D2088472068876397
:1037C000680407D5616C002904D0B7030E20884730
:1037D00020688763280407D5A16C002904D0F7036B
:1037E0000F20884720688763E80307D5E16C00292C
:1037F00004D037041020884720688763A80307D5C2
:10380000216D002904D07504112088472068856344
:1038100001B0F0BDDC93010202480068411E8841FE
:103820007047C046C0980102F0B58DB0002862D044
:103830000446406800285ED0A06840285BD8E56A4E
:10384000002D58D00746204640300026039003E064
:10385000019E4AE0039848E0402101220691FCF7CE
:103860009BFCAE4202963ED2002031460190099068
:103870000398069B3E46002EEAD0606A0491405CA5
:1038800007900998401C05900021042708916518AD
:10389000EA5C012A17D10A966268D3191B1F1B68BC
:1038A000099E9E5D0798864208D1059D5B5D002BB1
:1038B0000A9E22D00898401C089003E04035002260
:1038C0002A70A668069B0837491CB142DFD30898C6
:1038D0000028BFD00499491CE06A814205980990EC
:1038E0000398C8D301E003983E463746E56A029E36
:1038F000761CAE42B0D30DB0F0BD616A0B91E16AA7
:103900000C91D1590BAA204600F09CF80DB0F0BDE7
:1039100081B0B0B583B00D460446079307AB029360
:103920008069E1690EF0B0FC2062654800780028EB
:1039300003D1216AA06900F09FF96369A169226A35
:10394000204698470146A06B002905D069460C60C7
:103950000021224B0A460CE000F084FA7D20810011
:103960002846FCF7B7FB0246A06B69460C600021B5
:103970001B4B00F0D3FA002003B0B0BC02BC01B076
:103980000847C04680B5806B00F06CFA002080BD0F
:1039900070B582B00D460446466911461A46B047D6
:1039A0000146A06B002907D069460C6000210B4B33
:1039B0000A4600F0B3FA0EE000F054FA7D208100D0
:1039C0002846FCF787FB0246A06B69460C60002185
:1039D000034B00F0A3FA002002B070BDC93A00000A
:1039E000DF3A000070B50D460446802100F0C0FAB1
:1039F0002868E06368686060A868A060E868E060C4
:103A00002869206168696061A869A061E869002689
:103A10002662E061286A6062686A2663E662A062E4
:103A2000A86A60632046383000F02AFA002802D0E5
:103A3000F643304670BD214801682160046030467D
:103A400070BDC04670B514460D460646881E032854
:103A500002D8B06B00F006FAF06B2946224600F05F
:103A60000DF970BD16480178012048407047C046E6
:103A700070B512480468002C1FD0114E11A52169A1
:103A800020468847002815D1307800280DD1E16AFA
:103A9000606A00F09CFA0146606A012903D0E16A7D
:103AA00000F0E8F8284600F0E3F82046FFF7BCFEF7
:103AB0000020E0622468002CE1D170BD58C90102E9
:103AC00050C901020D0A000010B50446806B00F0D9
:103AD000C9F9E06B0521002200F0D0F810BD10B547
:103AE0000446806B00F0BEF9E06B0421002200F078
:103AF000C5F810BDF0B581B000910646C7680468EE
:103B0000A01C3946FCF7E6FA00257068814201D115
:103B1000ED430BE0601C3946FCF7DCFA316032699A
:103B20005143B06808180099FCF724FB284601B0FF
:103B3000F0BDB0B5012400250560446008300EC01A
:103B4000B0BD70B50E460446C1680068401CFCF765
:103B5000C1FA00256068814202D1ED43284670BD5C
:103B600022695043A16841183046FCF703FBE16825
:103B70006068401CFCF7AEFA6160284670BDB0B5C5
:103B8000002400280DD0054600688842FDD3401A65
:103B9000286068684018E968FCF79CFA696020466C
:103BA000B0BDE4432046B0BDB0B5002400280ED01F
:103BB0000546006840182860EA689042FDD8A86869
:103BC00040181146FCF786FAA9602046B0BDE443D0
:103BD0002046B0BDF0B583B0164602460027F84334
:103BE000002E22D01C46002B1FD00D46D168136832
:103BF00099421AD9CB1AAB4217D392680192521943
:103C00008A423A4607D9019A8A1A0292029A5219AE
:103C10009342029A09D3029201981018FCF75AFABB
:103C20003160029840192060384603B0F0BD40680A
:103C300070478068704702460020002A04D0106058
:103C400050609060D1607047C0437047002803D037
:103C5000016848424841704701207047002805D05C
:103C60000168C068411A48424841704701207047C6
:103C7000002070470020704700207047F0B583B0E7
:103C800014460D4606464088012818D130690028A0
:103C90000CD0A900405801782D2910D0F368716824
:103CA00009686A461160506010A205E0F368706808
:103CB0000068694621C115A23046FFF7C5FC776848
:103CC000FB683046294622469847012808D00AE07A
:103CD000C36830462946224698477F68012802D1AA
:103CE00078680028F4D103B0F0BDC04646534D3A81
:103CF000252D38732053544154453A252D323873BD
:103D0000204556454E543A25730D0A0046534D3A08
:103D1000252D38732053544154453A252D3238739C
:103D2000204556454E543A25750D0A00F0B581B030
:103D3000002828D01E460C460546079B0698009092
:103D400000206862A862E862104909886B802980B7
:103D50000F4B1F686C60009BAB602B460C33C4C3D9
:103D6000A861E8612862481C084908800848056085
:103D7000002C08D06C60002128460A46FFF77EFF21
:103D8000A468002CF6D101B0F0BDC046E0CC010221
:103D90005CC9010202460020002A01D0D1627047AE
:103DA000C043704710B582B004AC24881B881B0444
:103DB0001B196C462360024B00F0B0F802B010BD36
:103DC00071360000F0B597B016460291054642687C
:103DD000002A30D001966A60012100242846164648
:103DE0002246FFF74BFF3046029FBE4232D003A867
:103DF0005021FCF7D8F932467268002F0CD003AF7F
:103E0000029811C74068083F824209D039460831FC
:103E10003C4600280F46F4D1002A019EDBD10AE07F
:103E2000019E38686860002128463246FFF726FF69
:103E30007F68002FF5D102988468002C08D06C6050
:103E4000002128463246FFF719FFA468002CF6D15E
:103E500017B0F0BD00212846019E3246FFF70EFF45
:103E6000E9E70000014600201F2901D9C04370473F
:103E700018224A43344901238B50891888607047BF
:103E800010B50021CC4300280BD00A4A1368002B40
:103E900009D01832491C2029F8D306D106A0FFF713
:103EA000E7FE204610BD0123136001600024204678
:103EB00010BDC046E0C9010274696D6572204944B5
:103EC0002069732066756C6C0D0A00002648006836
:103ED0007047C04670B520241B4D234E2868022829
:103EE00017D13068A968EA68401A904211D9696907
:103EF000002907D02879002807D0022028603068E0
:103F0000A86004E00120286003E0012028602869FF
:103F100088471835641EE1D170BDC046F0B504462F
:103F200000201F2C01D9C043F0BD059D1826664313
:103F3000054C0227A751A41921710B49096826468F
:103F4000083626C66361F0BDE0C901020648016873
:103F5000491C01600548416802680023521C026048
:103F60004B4143607047C04694AD010298AD0102D9
:103F700080B5FCF718F980BDB0B50278002A24D0CE
:103F8000441C0021084601E0573A08E0234600019E
:103F9000D5B2302D0C4611D3392D02D8303A144603
:103FA0000CE0412D0C4609D3462D01D8373AF6E7EF
:103FB0001446613CE4B2062CE6D30024E2B2801839
:103FC0005C1C1A78002AE1D1B0BD0020B0BD10B54C
:103FD0000246012000290DD00023D45C202C02D3FE
:103FE0007F2C04D307E00D2C01D00A2C05D15B1CDB
:103FF0008B42F2D310BD002010BD002010BD000088
:1040000081B0F0B584B0099300230393002800D158
:10401000C2E0002A00D1BFE009AB03931678002E5E
:1040200000D1A8E05623DB43009300231D4600295E
:1040300000D1A2E0252E3FD1971C52781446643C53
:104040000023142C43D8C0467C4424796400A74440
:104050000A99A3A3A3A3A3A3A3A3A3A34CA3A3A32A
:10406000A3A3A3A35F000297039A131D03931268EF
:1040700001920122002317461E460478FF0703D051
:104080002D2C01D1164607E02746303F092F09D8CD
:104090000A275F433B19303B491E401C002700297B
:1040A000EBD13946029A019C002C03D0012E00D19D
:1040B0005B4223606B1C06E00378B3425BD1491E70
:1040C000521C401C2B461678002EAFD164E02A2AE1
:1040D00062D13A780378934204D0491E401C0029EB
:1040E000F8D100216B1C3A46EDE7039A131D0393A8
:1040F0003E7812680023C45CB44233D0491E5B1C76
:104100000029F8D13C46C7180021002A2ED12EE004
:104110000297039A131D039312680023009E0778E9
:10412000302F18D33A2F02D2344627340BE0612FB8
:1041300003D3672F344606D30DE03C46413C052CA3
:1041400009D8344620341B011B19DB19491E401CB9
:104150000029E4D10021029C002A00D013606B1CCE
:104160002246B0E73C46C718002A00D009C26B1CA3
:1041700022463846A7E700230EE0252E0BD15178C2
:10418000652908D103990A1D03920968002900D006
:1041900008606B1C00E02B46184604B0F0BC02BC63
:1041A00001B0084781B010B581B00C46039303AB52
:1041B00000930EF069F8A04200D3601E01B010BC5D
:1041C00002BC01B0084770B504460020002A1BD08D
:1041D000002C19D0002B17D014600120022B13D310
:1041E0002578002D10D0641C01208D4205D1651E5C
:1041F00000262E7085005451401C984204D2661C43
:104200002578002D3446F0D170BDB0B50446782134
:10421000FBF7D4FF002805D158212046FBF7CEFF3D
:10422000002828D04278002A23D0841C0021084688
:1042300023460001D5B2302D0C4613D3392D01D8B9
:10424000303A0EE0412D0C460CD3462D01D8373ABA
:1042500007E01446613CE4B2062C01D3002401E0DF
:10426000573A1446E2B280185C1C1A78002ADFD153
:10427000B0BD0020B0BD2046FCF760F8B0BD70B501
:1042800004460026F043002C0DD00D4600290AD02C
:10429000204610300121FFF772FCA9682034204627
:1042A000FFF76DFC304670BD70B504460026F04344
:1042B000002C0DD00D4600290AD0204610300121D7
:1042C000FFF772FCA96820342046FFF76DFC3046EA
:1042D00070BD70B50024002814D00546064610367F
:1042E0003046FFF7B3FC01280CD028462030FFF7FA
:1042F000ADFC012806D02C683046FFF798FC0C2155
:1043000041436418204670BDF0B583B00025029586
:10431000019500281FD00C46064607461037384640
:10432000FFF79CFC002816D13046203002AA01ABD2
:104330002146FFF74FFC00280DD135683846FFF7BE
:1043400078FC0C214143B068029A101868506D182F
:104350006C600198A860284603B0F0BD70B50546B2
:104360000C2058430024904211D2121A461829609A
:104370006860AE60EA60284610301946FFF75BFCC3
:10438000E96820352846FFF756FC204670BDE44317
:10439000204670BD04217046084204D0EFF3098323
:1043A000EFF3088203E0EFF30883EFF309829BB099
:1043B00004A8F0C044464D4656465F4608A8F0C0E3
:1043C0001846F0C86846F0C018690C9020201844C0
:1043D0000D9058690E9098690F90D8691090EFF37E
:1043E00010801190EFF3148012900949086813901F
:1043F0000849086814900849086815900749086832
:104400001690179318927046199068460BF0E8FDC5
:1044100004ED00E00CED00E010ED00E014ED00E034
:10442000F0B581B0032600243046214608F00CF890
:1044300004252846214608F007F80127304639466A
:104440003A4607F031FF30462146324608F024F85C
:10445000284639463A4607F027FF022128462246D9
:1044600008F01AF801B0F0BDF0B589B00890042545
:10447000284607F001FF0A27384605F015FF2846B1
:1044800007F00AFF0324204607F0FEFE07900526EA
:10449000304605F009FF284607F0EEFE384605F0E5
:1044A00003FF284607F0F8FE204607F0EDFE0690D1
:1044B000304605F0F9FE284607F0DEFE384605F0E6
:1044C000F3FE284607F0E8FE204607F0DDFE0590E3
:1044D000304605F0E9FE284607F0CEFE384605F0E6
:1044E000E3FE284607F0D8FE204607F0CDFE0490F4
:1044F000304605F0D9FE284607F0BEFE384605F0E6
:10450000D3FE284607F0C8FE204607F0BDFE039004
:10451000304605F0C9FE284607F0AEFE3846019742
:1045200005F0C2FE284607F0B7FE204607F0ACFEB5
:104530000290304605F0B8FE284607F09DFE38464A
:1045400005F0B2FE284607F0A7FE204607F09CFEC5
:104550000746304605F0A8FE284607F08DFE019874
:1045600005F0A2FE284607F097FE204607F08CFED5
:104570000446304605F098FE284607F07DFE069971
:10458000481E81410A460799481E8141480080180B
:104590008000059A511E8A4151004018049A511E0C
:1045A0008A4180188000039A511E8A4151004018A8
:1045B000029A511E8A4180188000791E8F4179002D
:1045C0004018611E8C4106190898002803D003206A
:1045D00007F052FE02E0032007F05EFE0A242046A8
:1045E00005F062FE0425284607F056FE204605F039
:1045F0005BFE284607F040FEF0B209B0F0BD70B592
:104600000446042007F038FE60B2002803D40320DB
:1046100007F032FE02E0032007F03EFE0A2528469E
:1046200005F042FE0426304607F036FE284605F027
:104630003BFE304607F020FE284605F035FE6006BA
:1046400003D4032007F018FE02E0032007F024FE45
:104650000A25284605F028FE0426304607F01CFEF1
:10466000284605F021FE304607F006FE284605F0F4
:104670001BFEA00603D4032007F0FEFD02E003208A
:1046800007F00AFE0A25284605F00EFE04263046ED
:1046900007F002FE284605F007FE304607F0ECFD65
:1046A000284605F001FEE00603D4032007F0E4FDF0
:1046B00002E0032007F0F0FD0A25284605F0F4FD8E
:1046C0000426304607F0E8FD284605F0EDFD3046AB
:1046D00007F0D2FD284605F0E7FD200703D40320AC
:1046E00007F0CAFD02E0032007F0D6FD0A252846A0
:1046F00005F0DAFD0426304607F0CEFD284605F029
:10470000D3FD304607F0B8FD284605F0CDFD600723
:1047100003D4032007F0B0FD02E0032007F0BCFD46
:104720000A25284605F0C0FD0426304607F0B4FDF2
:10473000284605F0B9FD304607F09EFD284605F0F5
:10474000B3FDA00703D4032007F096FD02E0032089
:1047500007F0A2FD0A25284605F0A6FD04263046EE
:1047600007F09AFD284605F09FFD304607F084FDCE
:10477000284605F099FDE00703D1032007F07CFDF2
:1047800002E0032007F088FD0A24204605F08CFD96
:104790000425284607F080FD204605F085FD2846C3
:1047A00007F06AFD204605F07FFD70BDF0B581B0D1
:1047B00003260025012430462946224607F074FDD1
:1047C000304607F069FD0626304605F06DFD0420F1
:1047D00007F062FD304605F067FD032007F054FD49
:1047E00000281BD0681CFA2D0546F6D30425284660
:1047F00007F042FD0326304607F03EFD0A27384603
:1048000005F052FD284607F047FD304607F044FD0D
:10481000384605F049FD204601B0F0BD03200121D6
:104820000A4607F041FD042007F026FD002420463B
:1048300001B0F0BD10B5854C608FFCF770F80146F3
:104840000748406AFBF7EEFF002808D1E08F0128F7
:1048500005D1022001210AF0DBFB08F037FF10BD73
:1048600098980102B0B50446C00703D1032007F0B1
:1048700003FD02E0032007F00FFD0825284607F09E
:104880000BFD284607F0F8FCA00703D4032007F02F
:10489000F3FC02E0032007F0FFFC0825284607F0A0
:1048A000FBFC284607F0E8FC600703D4032007F070
:1048B000E3FC02E0032007F0EFFC0825284607F0A0
:1048C000EBFC284607F0D8FC200703D4032007F0B0
:1048D000D3FC02E0032007F0DFFC0825284607F0A0
:1048E000DBFC284607F0C8FCE00603D4032007F0F1
:1048F000C3FC02E0032007F0CFFC0825284607F0A0
:10490000CBFC284607F0B8FCA00603D4032007F030
:10491000B3FC02E0032007F0BFFC0825284607F09F
:10492000BBFC284607F0A8FC600603D4032007F070
:10493000A3FC02E0032007F0AFFC0825284607F09F
:10494000ABFC284607F098FC60B2002803D4032093
:1049500007F092FC02E0032007F09EFC08242046AA
:1049600007F09AFC204607F087FC0724204607F052
:1049700093FC204607F080FCB0BDF0B581B0032762
:1049800000243846214607F04FFD3846214607F0FF
:104990005BFD012538462946224607F085FC0526A1
:1049A00038462946324607F077FD08273846214623
:1049B00007F04AFD38462946224607F075FC38467E
:1049C0002946324607F068FD07273846214607F09A
:1049D0003BFD38462946224607F066FC3846294604
:1049E000324607F059FD01B0F0BD000080B50B2044
:1049F00007F04AFC12490A78002804D0002A12D095
:104A000003F064FC80BD012AFAD1002008700F4930
:104A1000C8830C4908700C48012101700CF05EFA43
:104A200003F054FC80BD0748012202700A7006485A
:104A3000002101700CF072FA03F048FC80BDC04602
:104A40001C90010218900102199001023AA901027A
:104A500002488069811E48424841704778960102A9
:104A600080B5FDF7ADF9002801D00020C04380BD1E
:104A700080B5FEF765FA80BD10B504480F2100240B
:104A80002246FFF7FBF8204610BDC046D099010230
:104A9000F0B581B007460324204607F0FDFB04254E
:104AA000284607F0F9FB204607F0E6FB0A263046C9
:104AB00005F0FAFB284607F0DFFB3220FFF79FFDE9
:104AC000FFF774FEF8B2FFF79AFDFFF76FFE20467E
:104AD00007F0E2FB284607F0DFFB204607F0CCFB9F
:104AE000304605F0E1FB284607F0C6FB3320FFF710
:104AF00086FDFFF75BFE0020FFF7B6FC0746284661
:104B000007F0BAFB204607F0B7FB304605F0CCFBB8
:104B1000284607F0C1FB204607F0BEFB304605F0F3
:104B2000C3FB384601B0F0BDF0B581B00091074637
:104B30000324204607F0B0FB0426304607F0ACFB08
:104B4000204607F099FB0A25284605F0ADFB3046C4
:104B500007F092FB3220FFF752FDFFF727FEF8B275
:104B6000FFF74DFDFFF722FE0098FFF748FDFFF726
:104B70001DFE304607F080FB204607F07DFB2846EF
:104B800005F092FB304607F087FB204607F084FBD8
:104B9000284605F089FB284605F086FB01B0F0BDEC
:104BA00080B5074801210170064802680A43026087
:104BB00005480268002A02D000200146904780BDC7
:104BC000E6CC01021C100050E8CC0102F0B599B00F
:104BD000F548017BC67A427B0E92F44C221F136883
:104BE000F34A1268069242780C9202790592C76ADB
:104BF00004931F4001200F907A0200D5BCE03A02D6
:104C000000D5BFE0FA0102D50F98020622605025B8
:104C100008968A191826BB0102D50F98430623600F
:104C20004123079569430A96354655431426FC02ED
:104C300010D50F98040538463746DC4E3460DA4C00
:104C4000A469B464D84CE4697464DA4C241D3460FB
:104C50003E46074690000B90D8040D9068180990C6
:104C60000E9B73430F988203B902D04D22D50F9843
:104C700041052960CC480E96164602468169296591
:104C8000C169696509990D980143089800010818E0
:104C90000B994018C018C849098892794A4380186E
:104CA0000A301C4605F08CFE234632460E9EC04953
:104CB00088672A600F98C404380300D52C60F80375
:104CC00002D50F98000428600F984104B80300D55E
:104CD0002960380400D4E4E1039402910E93089211
:104CE0000D980B990C180A980C9941430C910F9848
:104CF000C0030B90286008F0E3FD002801D005F008
:104D000041FE0C98005B410B43D1099800190E99A4
:104D100040180599090140180E90E74D287B079B24
:104D20004343E97A0A010D9C2243D21841188B00B3
:104D3000D2180A9B4B43D1186A7B564389190E9EA1
:104D40002A791018DF4A1288424388181690306872
:104D5000C000800D10A9C882002511957079C00788
:104D60007ED110A80F998182069C00940020E8A2B1
:104D7000049B0BF077FF78E00F98820522603A02DF
:104D800000D43FE70F98C2052260FA0100D53BE747
:104D90003DE7072149030840032149038842089A57
:104DA00000D07EE1069708F069F90020169009907E
:104DB0001590C14CE07A217B08180A994143800084
:104DC0000D9A10434118627B0E9672438A186178DF
:104DD000A379079E7343D718FA683F263240637859
:104DE0009A420C976ED105960A9A4A4380580F2131
:104DF0000A0702400398401EC04B1B68DB090340B2
:104E0000981810900F98C0020B90B868800767D46C
:104E10002C46283C0AF09CFE05462068000609D571
:104E2000C3208401786A400704D40AF091FE401B35
:104E3000A042F7D905980002B96849080140B34873
:104E400003688268B868C40C20202040DB0700D0CB
:104E500095E0002310221D461C460E9E0B9FB1E0DC
:104E600010A88582B0681190069C701D924B19792C
:104E7000E20707D1491C1971D97A1A798A4202D3FB
:104E80001D7100E0D97001784278120251188278C1
:104E90001204891803229143017035715878401C1F
:104EA0005870D87A197B08185978884200D85D70F4
:104EB000D879401ED871596B002901D010A88847B5
:104EC0007E4DEDE010A80B998182F8683040637840
:104ED000009000207CA20F990BF0C4FE0E9E94E07F
:104EE000388A874A024010A8C2822022BA5C9307FF
:104EF000DB0F3C68C3720F9B1A4082726205D20CB2
:104F00000D9B1A431692FA68130E0372BB69FC6973
:104F10007C4D2D682D0C05745204920F4272119332
:104F20001394654CA07B002809980E9E0B9F5FD0C0
:104F300075480068007A0328099859D00C98007DBC
:104F400008400928099853D1C32084010AF000FEC3
:104F500005460C98406A41070BD45949096809066F
:104F6000890F06D10AF0F4FD401BA042F1D90C983C
:104F7000406A41030898884310A9888237E0D20725
:104F80000E9E0B9F03D108230022154619E00C9BAF
:104F90009A68029C224211D19A68520C02249443CE
:104FA0000022134615460DE0ECD1010228A0005066
:104FB0003CA10050FC1F0000E8D1010204250022A2
:104FC000134614460843104318432843204310A9AE
:104FD000888238420BD10C9B198A494A0A4010A991
:104FE000CA8219684905C90C0D9A11431691324CB1
:104FF0002921615C002908D03037B84205D010A9BA
:105000000846113012310AF037F8E77A2A48047B53
:10501000E519294800790E9027484078401C294618
:10502000FBF758F888000D9A1043189007996143D0
:105030003801104340182049497B4E4380191C21F8
:10504000694340180E9909191B4B1E4A12884A439E
:1050500080181790099A0C998A60987B002800D0D4
:105060004A629879401C9871187B99798142069F11
:1050700000D39A715978491C5970D97A081859780F
:1050800088420E4D00D85A70187A401E1872282097
:10509000185C002804D0996B002901D010A888471B
:1050A000089A174202D00F98000328601C48044950
:1050B000486019B0F0BDC046ECD1010228A00050F4
:1050C0003CA10050E8D101024857204554206964B2
:1050D0007820256420616E6420455420696478201E
:1050E000256420696E2052582064657363206D69C1
:1050F000736D617463680D0A000000003820004081
:10510000FF030000943000404894010260400040DA
:105110004D4143204556542025782025780D0A001E
:10512000FFFFFF03F0B5A5B01E460C9208910024C6
:10513000239422A90C8016A90C8024A909250D808E
:10514000598C0D91FAF7C6FF2A99012900D0DFE0AA
:105150003189012900D0DBE0318C012900D0D7E072
:105160000D99002900D1D3E0224607962C990B9186
:105170002B99069180B205900F9415A80580900098
:105180000E900C990C582E460025204629461746AD
:10519000FBF748FB0028119636D12C200A9778435C
:1051A0000899081817A90A4668C868C2E8C8E8C27A
:1051B000E8C8E8C2079F119880B280000E5822AD5F
:1051C000019523A8009020463946059A069B05F0D4
:1051D00079F80F98401C0F90288800282DD03B8A22
:1051E000239913AC039416A8029014A8019015AE4D
:1051F000009617A824AA05F03FFA25883088119058
:105200000120149E0A9A05E013A8058014952E46E5
:1052100028463A460E9F51000B9B119C5C52591830
:1052200008830D84D81986600F981885521C0D9834
:1052300082426DD024A805889FE7099616A800250C
:105240000580149524A80688239812902F4610955F
:1052500003E06D1CA8B2B04213D8A8B2800017A911
:105260000C5820461299FBF7EBFA0028F1D1002FD9
:10527000EFD115A8058016A8012707801494109473
:10528000E7E715A80288B01A012805D115A80680FD
:10529000099F1497119628E010200799095E0129AB
:1052A000119221DB551CA8B20C18109F0E9B09947B
:1052B00003E06D1CA8B2844218DDAAB2B242F8D84D
:1052C000800017AA10581090394634461E46FBF746
:1052D000A9FA33462646099C0028EAD115A805807C
:1052E000109F14971195E4E7109F0E9B1C463E46B5
:1052F00038461299FBF7C5F8FBF750FB0546052821
:1053000000D3052513A8058001200A9A274682E7C5
:1053100025B0F0BDF0B58BB00243159A149C139ED6
:105320002BD0054601A856C0129CD869196A09906D
:105330000A911E469F6B0123009309A807AA014604
:10534000059307F0CFF8716C3846FBF79AF80746DB
:10535000E06A616BFBF795F8002D069613D00446C2
:1053600011980199012924D10921081A0421069ACA
:10537000515E884229D16425B1E000203080207040
:1053800010700BB0F0BDB08800226425002829D031
:10539000059269493846FBF76FFA0028049C039E82
:1053A0006FD166493846FBF767FA00281DD05A25A9
:1053B00067E03C25082800D191E05F492046FBF7D3
:1053C0005BFA002819D0502589E00A291DDB1D2928
:1053D0003BDC59493846FBF74FFA0022002854D0ED
:1053E0005A253AE03346049C39E055493846FBF7E4
:1053F00043FA002821D0502543E050492046FBF7CE
:105400003BFA00282ED0462569E03C25012866D0CD
:1054100049492046FBF730FA0028D4D147492046B5
:10542000FBF72AFA0028EED145492046FBF724FA7B
:10543000002854D1434920466EE042493846FBF7E4
:105440001BFA00281CD128251BE03B493846FBF7F6
:1054500013FA0022002832D05025049C069B0299A2
:10546000039E41E036492046FBF706FA002836D174
:1054700034492046FBF700FA00282FD114252EE0EE
:1054800037250299059A069B2EE005922B4938464E
:10549000FBF7F2F9002896D129493846FBF7ECF9D9
:1054A0000028B0D127493846FBF7E6F90028049CCC
:1054B000069B0299039E059A3BD11E2514E0059296
:1054C0001E493846FBF7D8F900289CD11C493846BC
:1054D000FBF7D2F900281DD03C2500E02325049CD1
:1054E000069B0299039E059A258032700020087061
:1054F000307800280CD118681349FBF7AFF9002861
:1055000006D12088102803D30F3820800BB0F0BDBF
:105510000BB0F0BD0B493846FBF7AEF90028049CF0
:10552000069B0299039E059A01D11425DCE72325E9
:10553000DAE72D25D8E7C046CDCCCC3DCDCC4C3DCF
:10554000CDCCCC3C0AD7233C0000204070B588B0BD
:105550000C4606464088002820D0FBF7E0F905906D
:1055600005A804A901252A4607F026FA3088B18843
:10557000081AFBF7C9F90390049903A807AA2B4658
:1055800007F0DAF95249079D2846FBF775F900281C
:1055900008D0BF200006206008B070BD0020206049
:1055A00008B070BD4B492846FBF74AF9002804D0E3
:1055B0003F200006206008B070BD47492846FBF731
:1055C0005BF9002801D0002010E000212846FBF7FD
:1055D00053F9002801D0022008E040492846FBF793
:1055E0004BF9002801D0042000E0062001957F211E
:1055F000C905029180003A49091801A806AA0223A8
:1056000007F04EF90698206008B070BDF0B587B07D
:105610000C4605464768002638463146FBF73AF9FE
:10562000002802D0266007B0F0BD049704A803A9A3
:105630000126324607F0C0F9A8682968FAF7DCFEAF
:105640000290039902A806AA334607F075F920498B
:10565000069D2846FBF710F9002804D0BF20060657
:10566000266007B0F0BD1B492846FBF7E9F8002883
:1056700004D03F200606266007B0F0BD1649284634
:10568000FBF7FAF8002801D0002010E0002128469E
:10569000FBF7F2F8002801D0022008E00F49284665
:1056A000FBF7EAF8002801D0042000E0062000956E
:1056B0007F21C9050191800009490918684605AA9A
:1056C000022307F0EDF8059E266007B0F0BDC04646
:1056D000CDCC0C3F295C0FBFCDCC4C3ECDCC4CBECD
:1056E00050940102F0B587B00C4606467F2700882B
:1056F000002801D0FD0503E0B08800282ED0334DEE
:10570000FBF70DF903907088FBF709F9049003A8E3
:1057100002A90126324607F04FF9029904A806AA09
:10572000334607F009F92A49069E3046FBF7A4F8EC
:10573000002802D03F20010641E026493046FBF711
:105740007FF8002802D0BF20010638E02249304609
:10575000FBF792F8002805D0002024E0002020600C
:1057600007B0F0BD1D493046FBF786F8002801D090
:10577000022018E01A493046FBF77EF8002801D0D5
:10578000042010E017493046FBF776F8002801D0D6
:10579000062008E014493046FBF76EF8002801D0D7
:1057A000082000E00A200096F905019180000F49C9
:1057B0000918684605AA022307F072F805992846D9
:1057C000FAF722FE206007B0F0BDC046000080BF9F
:1057D000000038433333733F0000C842000070427A
:1057E000000020420000A0410000C040709401026F
:1057F000F0B59DB015460B917F210391C9051C9111
:1058000002911B9119A900248C8019941894179463
:10581000598C0691198C0F91DE8B998B0791997891
:1058200005911F882B21CA432799914201DB7F00F4
:1058300015E04022D243914211DC4922D2439142E9
:1058400002DB7908CF190AE05322D2439142EEDA03
:105850005D22D243914201DBBF0000E0FF000A97C6
:105860001396269E597E00290BD0002132460F4602
:10587000D170917051701170121D7F1C5C7EA74217
:10588000F6D30C9311952599149122990D911590A9
:1058900041088C4211D2FD4A2346A000845834545A
:1058A000270A451C7755250C871CF555240EC01C6E
:1058B00034545B1C9CB2A142EFD823981090012075
:1058C0000990009030463146149A159F3B4606F0E9
:1058D00017FE0D9800060890400E139D00D186E03B
:1058E00068000490002F3FD0002210461146144655
:1058F00006E01C461146159F401C82B2BA420ED2E9
:1059000083B2AB42F8D09200149B9A5E0FB2BA42B7
:10591000034600DC2346BA42EBDC0A46E9E7002FE7
:1059200025D0002210461146129206E0129311462D
:10593000159F401C82B2BA4214D283B2AB42F8D057
:10594000A5B2AB420CD09200149B9A5E0FB2BA4241
:10595000034600DC129BBA42139DE7DC0A46E5E7EA
:10596000139DE6E7129903E00024214600E00021A0
:10597000129110980183C4828582049FF057FAF730
:10598000C3FF7921C9050E91FAF73EFD1099C86150
:1059900009980743F057FAF7B7FF0E99FAF734FD65
:1059A000109F38622004C40B3057FAF7ADFF0E99F0
:1059B000FAF72AFD7862601C3056FAF7A5FF0E9CB4
:1059C0002146FAF721FDB86212980004C70BF05780
:1059D000FAF79AFF2146FAF717FD109CE062781C4F
:1059E0003056FAF791FF0E99FAF70EFD20631198E1
:1059F00005800C98407E410000278D4228463A469B
:105A0000149E1ED30A9880B28AB29300F45E844238
:105A10000BDA491C8AB2AA42F6D9002728463A4630
:105A200081B2691A012910D01BE0F018119B19806E
:105A3000078808040FD0500040008019001F02881A
:105A4000084681B2691A01290BD1A80030181199B2
:105A50000D80078826E00020024681B2691A0129DC
:105A6000F3D00A9989B2079B4B43BB421AD30699DC
:105A70008A4217D80599002914D0401C82B289188F
:105A800003E0401C82B291420CD983B2AB42F8D8F9
:105A90009200B35EBCB2A342F3DDB218119B188032
:105AA0001788EEE712970B980580119800882B1A3B
:105AB000002B16DD02210F9A1143032942D10E93C8
:105AC000411C421E10B281420EDA0E98032824DBDC
:105AD0000C98808C012820D019A818A9FFF736FD52
:105AE0001FE0002018902BE00026F443374608E022
:105AF000B8B2400019AD2B527F1C521C10B281422B
:105B0000E3DB13B2A3423346F2DD159B98423346E2
:105B1000EEDA8000149B1B5AEAE719A818A9FFF7D0
:105B2000E1FD149E139D0F9A012A13D0032A11D070
:105B3000022A04D111980088281A02280ADA0020C3
:105B4000179034E0022A01D1022BB8DA0020189015
:105B5000012AEBD1681C691E0FB2B84208DA0C9812
:105B6000808C01281DD119A817A9FFF7BBFD1CE0E7
:105B70000022D343144608E0A5B26D0019AF7E534E
:105B8000641C491C0FB2B842E9DB0DB29D421646B7
:105B9000F2DD159DAF421646EEDABD00149E765B2F
:105BA000EAE719A817A9FFF7D1FC149E139D249FBB
:105BB000189C17992046FAF71FFC0F99012900D865
:105BC000204638600D98002800D1CBE01199088854
:105BD000109FB8860888281AB880129880B2FAF701
:105BE0009EFE7921CC052146FAF70EFC2146FAF7F4
:105BF0000BFCB863119F3888002849D081008919AF
:105C0000091F0988129C0C191599884203D280003B
:105C100080198088041915984300534916AA304604
:105C200006F04CFE169810994864FAF7D0FEA4B21C
:105C3000A04201D14D480FE0001BFAF770FE1C9006
:105C40001CA81BA9012206F0B7FE2046FAF767FE42
:105C500001461B98FAF7D8FB109908603988491B50
:105C60004A1C92B2032A02D20021159F17E009B202
:105C70000229159F12DB3F210906FAF7FDFD0028D6
:105C800002990CD10998810709E0C04640210040E3
:105C90000020129C15998842B9D3BCE7344910986A
:105CA00001610898800E5DD0002F1CD000221146A3
:105CB000144610464B1B1DB2ED135B196B40139D30
:105CC0001BB29200B25E53431818A418491C8AB242
:105CD000BA42EFD3FAF723FE06462046FAF71FFE34
:105CE000002C03D100E000260398C0051C901CA8DE
:105CF0001BA901252A4606F05FFE1B9C2046314663
:105D0000FAF782FB014610988160002F119422D08F
:105D100000242746264613951291B8B2FAF7FFFDE4
:105D20001299FAF769FB0546A0001499085EFAF784
:105D3000EBFD01461398C00785432846FAF764FB3C
:105D400001463046FAF707FB06467F1CBCB21598A1
:105D50008442E2D300E0002611983146FAF754FB62
:105D60001099C8601DB0F0BD38A7010200002041A5
:105D700000004040F0B58FB00692F74A09AF70CAF4
:105D800070C770CA70C70328079320D88800F3A192
:105D90000858F649FAF7DFFA0446F549FAF7DBFA4C
:105DA0000D90F4492046FAF7D6FA0C90F2492046B5
:105DB000FAF7D1FA0B90F1492046FAF7CCFA0A909B
:105DC000EF492046FAF7C7FA0990EE4969E004283E
:105DD00022D0062820D88800EBA10858EE49FAF70F
:105DE000BAFA0446ED49FAF7B6FA0D90EC492046A6
:105DF000FAF7B1FA0C90EB492046FAF7ACFA0B909F
:105E0000E9492046FAF7A7FA0A90E8492046FAF746
:105E1000A2FA0990FD4944E00838022821D88800F8
:105E2000FBA10858D149FAF796FA0446FC49FAF75B
:105E300092FA0D90FB492046FAF78DFA0C90FF205C
:105E400081052046FAF787FA0B90F7492046FAF7C2
:105E500082FA0A90CA492046FAF77DFA0990FE496B
:105E60001FE08800F1A10858F449FAF774FA0446D3
:105E7000F349FAF770FA0D90F2492046FAF76BFAF7
:105E80000C90F1492046FAF766FA0B90EF4920464C
:105E9000FAF761FA0A90EE492046FAF75CFA09909F
:105EA000EC4900942046FAF756FAEC4909680E903E
:105EB000EB480468EB4801684808EB4F05463D4055
:105EC0000022002D08922DD0CA01120E07D0280CF6
:105ED000E90D12D14000E649085AE6490AE0C90333
:105EE000090E0CD0280AE90B10D14000E049085AED
:105EF0008F2189004018E4300DE0DC490AE081B2CE
:105F00007F2905D84800DA49085A04E0D94901E058
:105F10008F218900401800B2FAF7F6FCD649FAF74B
:105F200073FA02460292039507252606D34B1A6898
:105F3000002A089840D0791C8A420BD21102090E1F
:105F400013D0110C1F46D00D1FD14800C849085A64
:105F5000C84907E01F46110E002A13D44800C4495F
:105F6000085AC2494018E4301FE011041F46090EC8
:105F70000ED0110AD00B12D14800BD49085A8F210A
:105F80008900EFE7BE4808180FE0B84808180CE091
:105F900091B27F2906D84800B549085A05E0B548AE
:105FA000081802E08F218900501800B2FAF7ACFC03
:105FB000B149FAF729FA3B460590159F2C40F50E9A
:105FC0005B69B0491940089810D0DA02D20E34D07B
:105FD000C80B3E210140A648405AA6494018E4306B
:105FE00000B2FAF791FCA449FAF70EFA0490149E55
:105FF0006800A5A1085EFAF787FC0146A00009AA7F
:106000001058FAF7A8F90146B8B20128089F019183
:1060100002D1022C0AD9A74F052C24D11898089038
:106020000C2D20D80B2D16D3A44918E00027022CE4
:10603000089718D08120C70515E01A04120E00D168
:10604000CAE0080AC90B00D0CDE040008849085AD0
:106050008F218900C2E7092D00D2C7E09649089830
:10606000FAF779F9089001200021B542034600D3E0
:106070000B46052C00D308461799169A1A9C199DB1
:106080001843069B012B12D1079B402B22D10028DD
:1060900040D03846FAF75FF901460198FAF75BF904
:1060A00001460098FAF7A8F9059A04998AE0079B37
:1060B000402B1FD1002838D03846FAF74CF901465A
:1060C0000198FAF748F901460098FAF795F9059A08
:1060D000049977E0002833D03846FAF73CF90146B6
:1060E0000198FAF738F901460098FAF785F9059A08
:1060F000049967E000285BD03846FAF72CF901468E
:106100000198FAF728F901460098FAF775F9059A07
:10611000049957E002981146FAF76EF9039900299D
:1061200000D16748059A04994CE002981146FAF7A5
:1061300063F90399002900D16148059A049941E067
:1061400002981146FAF758F90399002900D15C48E2
:10615000059A049936E0C0460C2D0100000068C184
:10616000000088C166665EC1000084C100008441F1
:106170000000B44100004841000020400000F0C091
:10618000000084C10000F841333323C1000050C136
:106190009A9929C19A9949C19A9949413333CB4176
:1061A00066667641CDCCAC40333393C09A9949C1F1
:1061B00002981146FAF720F90399002900D14048C6
:1061C000059A049928601046FAF716F90899FAF723
:1061D00013F920600FB0F0BD99B27F2911D84800A3
:1061E0002349085AFCE623494018F9E6C120010674
:1061F0000898FAF7B0F80890062D00D933E7002088
:1062000030E78F2189005818EAE6C0463333F3415E
:10621000000058C19A9961C19A9969C1000084C16E
:106220000000AC4100003841000008C1CDCC80C165
:10623000CDCC88C133338FC1333397C133339741CA
:10624000CDCC8C413333F3409A9919C0666646C170
:10625000333397C1CDCCB4410000D4410C00004091
:106260005030004068400040FFFFFF007C08000005
:10627000183101005C050000919AF63C6420004052
:106280009C0B0000FFFF1F00FAFFFCFFFEFF000059
:1062900002000400060008000A000C000E001000B6
:1062A00012001400160018001A001C001E00200026
:1062B00022002400000080BF0000A0C0000040C0F9
:1062C0000000DCC2F0B5FFB0ECB017460E460D90F2
:1062D0000021E991E891DC9199919891979196919B
:1062E0001491139112919AA8F49DF39CF29A002EA6
:1062F00000D1E6E10B938030F09B11800995296075
:106300002546DBAC218095AC21800C952980DA9163
:106310007F24E405B994B894B794B694B594B49432
:10632000B394B294B194B094AF94AE94AD94AC9451
:10633000AB94AA94A994A894A794A694A594A49481
:10634000A394A294A194A0949F949E949D949C94B1
:106350009B949A94046644668466C46604674467A2
:106360008467C467046444648464C46404654465E5
:106370008465C465046244628462C46204634463E5
:106380008463C463046044608460C46004614461E5
:106390008461C461B0090B250B2800D3AE011095B0
:1063A000012B0B9D00D070E12B89012B00D06CE1FB
:1063B000298C00290E9200D18BE16B8C002B00D12F
:1063C000FAE1AA8C3021695C002900D188E10892A9
:1063D000109F5F431196304639460F93F9F77AFEC6
:1063E0000590FAF791FA01462046FAF74AF8832118
:1063F000C905FAF709F8064696A8021D11988742C2
:106400000A9200D879E155A811909AA9069196AF01
:1064100015463A46059C234606F042FA15A80F9009
:1064200006992A46234606F03BFA02230D93384686
:1064300031463A4606F080FA012308930093E8AA11
:1064400010923846394606F04DF8E898DD901198DC
:10645000069D29463A46234606F022FA0F98294619
:106460000A9A234606F01CFA384631463A460D9BF6
:1064700006F062FA089B009338463946109A06F0F7
:1064800031F8E898DE9011982C4629463A46059D49
:106490002B4606F005FA0F9821460A9A2C462B4601
:1064A00006F0FEF9384631463A460D9B06F044FAAE
:1064B000089B009338463946109A06F013F8E8987E
:1064C000DF901198069D29463A46234606F0E8F9E2
:1064D0000F9829460A9A2346254606F0E1F93846E0
:1064E00031463A460D9B06F027FA089B0093384642
:1064F0003946109A05F0F6FFE898E0901198069C4E
:1065000021463A462B4606F0CBF90F9821460A9AC7
:106510002C462B4606F0C4F9384631463A460D9BC8
:1065200006F00AFA089B009338463946109A05F09F
:10653000D9FFE898E1901198069D29463A462346EE
:1065400006F0AEF90F9829460A9A2346254606F02A
:10655000A7F9384631463A460D9B06F0EDF9089BFF
:10656000009338463946109A05F0BCFFE898E2904F
:106570001198069C21463A462B4606F091F90F9851
:1065800021460A9A2B4606F08BF9384631463A46A0
:106590000D9B06F0D1F9089B009338463946109AB6
:1065A00005F0A0FFE898E390119821463A462B4663
:1065B00006F076F90F9821460A9A2B462C4606F0EB
:1065C0006FF9384631463A460D9B06F0B5F9089BFF
:1065D000009338463946109A05F084FFE898E49015
:1065E0001198069D29463A46234606F059F90F9818
:1065F00029460A9A2546234606F052F9384631467E
:106600003A460D9B06F098F9089B009338463946A8
:10661000109A05F067FFE898E5901198069C2146CE
:106620003A462B4606F03CF90F9821460A9A2B462B
:1066300006F036F9384631463A460D9B06F07CF9AD
:10664000089B009338463946109A05F04BFFE898AE
:10665000E690119821463A462B4606F021F90F980C
:1066600021460A9A2B4606F01BF9384631463A462F
:106670000D9B06F061F9089B009338463946109A45
:1066800005F030FFE898E7907AE010880C9A1080C7
:1066900099919891DA9E08460F46099DF59CF9F765
:1066A000ABFE2860DC9827606060A6600C34DDA833
:1066B0000EC80EC42EC82EC42EC82EC47FB06CB017
:1066C000F0BDFF2010800021296020807FB06CB0D9
:1066D000F0BD002201233021695C002900D076E65C
:1066E000DDAA1ACF1AC23ACF3AC23ACF3AC20B2128
:1066F0003046F9F7EFFC054642E000200690059D84
:106700000796089F1190069801460D9C0F9A4A43E0
:10671000D219109B5A43119BD218D200A35889005A
:106720002E4655AD6B503546121DA25815AB5A502A
:10673000401C01B28E42E9DC55A89AAE96AC3146B7
:1067400022462B4606F0ACF815A831460A9A2B468D
:1067500006F0A6F8022320460799224606F0ECF838
:1067600001230093E8AA2046214605F0BBFE119BB9
:106770009800DDA9E89A0A505B1C0B2B1846C1D182
:10678000F19EDDA89AA9DCAA0B2306F089F809215D
:106790000E980F9101800B98C168DC9C2046F9F798
:1067A00033FE0146A8B2E69F0F281BD808280DD358
:1067B0000846F9F7D0FD14E0FF2010800021099A67
:1067C00011600C9908807FB06CB0F0BD042803D331
:1067D00081220846D10502E0412208461106F9F758
:1067E00013FE01462B20C04386420D9704DB08466A
:1067F000F9F7B1FD014603E04020C043864244DD85
:106800000E9A0C9C0B98408A002811D00B98038A92
:1068100095A80390DBA80290DAA801900094DDA867
:106820000D4603F029FF29462488DA9E099D68E079
:1068300011910F98208000273D46109705E00E9893
:1068400004887F1CB8B2A04211D8B8B28000DDA97C
:106850000C5820461199F9F7F3FF0028EFD1002DCD
:10686000EDD10C98078001250F971094E7E7DBA87E
:1068700005800F9A90B2201A012811D10C9804803B
:106880000D9FDA973E46099D3AE04920C043864273
:1068900000DA8BE0FF2208469105F9F7B5FDA9E77C
:1068A00010200B990E5E012E00DA90E0551CABB261
:1068B0001846A1B2AAB28A4217D805E00E990C88F0
:1068C000A1B2AAB28A4210D88000DDA90C58204695
:1068D00010991F46F9F7A6FF3B46002805D10C98F2
:1068E00005800B98068A0F95109430B2C1186D1C64
:1068F000A8B28142E2DC109EDA960F9C099D0D9FA2
:1069000011993046F9F7BDFDFAF748F8052800D38C
:10691000052095A90880A0B20E990988814218D94E
:10692000401C611E0CB2A04218DA12A898A9FEF70A
:106930006DFE0E980188481C491E0CB2A04221DA57
:1069400012A899A9FEF762FE99999898099D0D9F42
:10695000A4E600219891999108469FE600221346EB
:1069600008E09CB2A40012AF3D515B1C491C0CB264
:10697000A042DADB8DB20A2D1546F2D8A400DDADB7
:106980002D59EEE70022134608E09CB2A40012AF96
:106990003D515B1C491C0CB2A042D1DB8DB20A2DCB
:1069A0001546F2D8A400DDAD2D59EEE75320C043C3
:1069B000864200DB1BE70E460B9881692046F9F7FB
:1069C00031FF00280C9C08D10B98808B07E01446FF
:1069D000099D0D9F1199109E93E70B98C08BF9F7B5
:1069E0009EFF01463046F9F70FFD119021E70000A8
:1069F000F0B58BB01C4609930E46034600200A9062
:106A000040480088224F05970AA9049103940292F6
:106A1000109C0194012500950B21414389B230332C
:106A20001C4A3046FFF74EFC38680790786808909B
:106A3000B868069033480088334F00950194029758
:106A4000324E30363249334A3346FEF76BFB0698F6
:106A5000F8620798386308987863099800882E4987
:106A600005912E4904912E490391029701900096B9
:106A70002C4B284629462A46FEF74CFC43200106AB
:106A80000A98F9F7C1FCF9F789FF0BB0F0BDC046D1
:106A900000A70102F8DF0102F0B589B00F9F0E9C3C
:106AA000002815D01098079016480088164E01252A
:106AB0000095019102960893144B30331449154AFE
:106AC000FEF730FB089BF76207983063746303E0BE
:106AD0000D484763C462002518880F4905910F4986
:106AE00004910F4903910849029101900748303001
:106AF000009001210B4B28460A46FEF70BFC09B01B
:106B0000F0BDC046A4AD0102BCD4010268A00102E0
:106B1000F09E01028CD2010230A40102A0AD01025C
:106B200040AD010248AD010230487047004870474F
:106B3000E4AD0102800037490918C86B0022CA631E
:106B40007047C046800033490918886C00228A6467
:106B50007047C04680B52F4AD369002B01D0126A16
:106B60009847002080BDC0460249087800220A707C
:106B70007047C04654C901020020704780B51829EB
:106B800005D803468A1E03481946F9F7F3FA002090
:106B900080BDC046A8AD0102B0B502460020022962
:106BA00001D2C043B0BD8C1E0F2C07D8044D28461F
:106BB00011462246F9F7DEFA00202855B0BDC0463E
:106BC000C4AD0102B0B502460020022901D2C04383
:106BD000B0BD8C1E0F2C07D8044D28461146224606
:106BE000F9F7C8FA00202855B0BDC046D4AD01025F
:106BF0000849087800220A707047C046B0B50446BC
:106C0000044DAA68002A02D0E968204690472C610A
:106C10000020B0BDC497010210B5C64CA078002872
:106C200006D00020607118480121C170417010BD6C
:106C3000BF48808F0028F4D0E07821790143F0D05C
:106C4000114800214170C278002A0ED06279037980
:106C50009A4207D30122427002716171C1700AF039
:106C60008DFF6279501C607110BD01224270637902
:106C7000142B05D361714170C2700AF07FFF6379F4
:106C8000581C607110BDC0461C90010280B51248AE
:106C900001681F220A40026003200840022812D126
:106CA0000E480268D30D02D0FF231B06D2180C4BEE
:106CB0001A600C4A12680C4B1A6080680B4A1080EC
:106CC000000C0B4A10801A488268002A02D08268A1
:106CD0000020904780BDC0467420004064400040C2
:106CE000A0D2010278300040A4D20102CCA001025F
:106CF000B0D4010280B50D48016889070FD5052180
:106D000001600B48C178002908D00021C170C1681A
:106D1000002903D0C26841680020904780BD054823
:106D200005A10B4A0BA308F041FFC0462C0400400C
:106D300038940102114B01005048595F54494D45A8
:106D4000525F49525148616E646C657200000000E8
:106D50008D0A0000556E65787065637465642069FE
:106D60006E746572727570740000000070B5044630
:106D7000401E012814D80320084011D13F204003B1
:106D80000818050B281980280AD8164E31780120DA
:106D90004840294604F09AFC641E6D1C002CF5D175
:106DA00070BDC04680B50020014604F0B3F900284C
:106DB00000D080BD0B480121017080BD70B5164622
:106DC0000C460546FF22F9F7E7F905483118054852
:106DD0000278012050402A46234604F01FFB70BD74
:106DE00000E0070438A901020120000370470120D8
:106DF00040037047F0B585B04B484C49016006F040
:106E0000B3FC4B4DAB884B48C363A97A0173A98986
:106E10000183A98A4183EA8A8283474C6283218362
:106E2000A98D21810493A3804A1E9141490081626A
:106E3000E98E002901D10121E9860022EA833C2262
:106E40004A433E490A803221695C4173288B3C49A0
:106E500008800120000268806C8C0F2022460240CE
:106E60007D21C900260B4E43B6182205170F642258
:106E70005743F6192406270F0A246743F619314FA2
:106E80003E80AE8C374607402B46350B4D43ED19FF
:106E900037053F0F5743ED193606360F6643AD19D8
:106EA000294E3580DD8C2E4606402F0B4F43BE19F0
:106EB0002F053F0F5743F6192D062D0F6543751902
:106EC000224F3D801D8D28402E0B4E433018290542
:106ED000090F514340182906090F614340181C4E01
:106EE000308003241BA220462146049B09F0BAFEF1
:106EF0000F484088C1B20091030A1AA220462146D9
:106F000009F0B0FE0F4803880F480088398832889E
:106F10000B4D2D8800AE27C61DA22046214609F044
:106F2000A1FE05B0F0BDC0460896010281880000B0
:106F30003AA901029898010278D4010286960102CA
:106F4000849601027C9601027E96010280960102DF
:106F500082960102C9E8B1B849443A202578202E2A
:106F60000D0A0000B9CCBCFEB0E6B1BE3A5557429E
:106F70002D3447B3B5D4D8CAD6BBB7B2E2CAD4B958
:106F8000CCBCFE205625642E25642E200D0A000060
:106F9000B7FECEF1C6F7B5D8D6B73A2025642E2570
:106FA000642E25642E25643A25642E0D0A00000007
:106FB000F0B581B0244F3B78002B0CD0234D4035E9
:106FC000002214462E8886420AD0AD1C641C521C36
:106FD0009A42F7D301E0002422469C4203D006E007
:106FE000D4B29C4203D1172B01D8631C3B705300D1
:106FF000164CE318402558530020A0547981B889D5
:1070000000281ED0FC6A124884421AD00846F9F7BC
:107010008DFC00250F4B2A46F9F724FB07460E4648
:107020002046F9F783FC2A460A4BF9F71BFB024678
:107030000B463846044F3146F9F762FAF9F7DCFCA3
:107040000146F96201B0F0BD30990102009A0102D7
:10705000FFFF01000000E03FF0B583B0304800685A
:10706000C16B0901890F01D003B0F0BDC16BC06BCA
:107070002C4D05404800400F082602968640022706
:10708000384603F041F801907043C10B4A1B264873
:107090005043F9F735F8044608F050FC032123A2C9
:1070A00038461F4F0091234609F0DCFDF88A00287E
:1070B00017D0019840012946F9F70CF846431822E9
:1070C000324001200F2A014600D8002173095B18C5
:1070D0001B4CA3420DD8194DED1A6D050F2A0CD883
:1070E0000CE038680021C160112002F0FDFF03B000
:1070F000F0BD5D1C6D050F2A00D956422A0C029D79
:107100002E4009018919A34202D80098000400E02A
:107110004004081880183968086303B0F0BDC04601
:10712000C8940102FFFF1F0040420F0052434F333B
:10713000324B2070706D2025640D0A00FF0700009F
:10714000FE7F0000B0B582B0154908688269D20799
:107150000CD00122C2610D69002D07D000686C4679
:10716000214608F07FF900212046A84702B0B0BDB3
:10717000B0B582B00A490868026C92070ED5026C5D
:10718000012313430364CD68002D07D000686C46CB
:10719000214608F067F900212046A84702B0B0BD9B
:1071A000C894010206480168032291430160016806
:1071B00001220A43026000F01DFC08F0E5FBC04616
:1071C0002800004080B50D490868002810D52248E5
:1071D00002680423032A01D01A4300E01A460A6019
:1071E0001E490A68002A02D041680020904780BDED
:1071F00003A00CA19E2211A308F0D8FC2C10014082
:10720000696E636C7564652F647269766572732F3D
:107210006D6B5F736C6565705F74696D65722E630D
:1072200000000000534C4545505F54494D45525FA6
:1072300049525148616E646C65720000556E657804
:1072400070656374656420736C65657020696E7425
:1072500065727275707400000C900102B8D401025E
:10726000F0B581B0224F387A411C39723D280AD3DB
:10727000002038720C2004F0FFFF3846383001211E
:107280001C4A02F07FF900F0DDFD1B480124047068
:10729000B878002810D1FDF7DBFB002804D0174890
:1072A00000218170797207E0787A1E2800D30024CB
:1072B00012498C70401C7872FCF748FE1048448FCD
:1072C0002046F9F72CFB01467D6A2846F9F7D4FAE7
:1072D00006467F20C1052846F9F73DF80546601CA3
:1072E000F9F712FB002E00D12846786201B0F0BDFC
:1072F00098980102F5930000C69601021C900102C5
:107300003AA90102B0B582B004460078002811D035
:10731000094D01A908702868416A0029FCD101A91A
:107320000122002003460AF05FFA611C6078002801
:107330000C46EED102B0B0BD0495010270B50C78D8
:107340004D782D022C198D78C97809024919090444
:1073500009198000094C21509178D4781578527819
:10736000074E3350074B069E1E501202521923023D
:10737000591809048918044A115070BDA09F0102D0
:10738000A0E001023CE0010204A0010210B5C04CE3
:10739000216806290FD8012002468A4058210A4256
:1073A00009D020600020A0602369002B03D062690F
:1073B000002002219847DB482258062A12D80121D2
:1073C0000B469340582213420CD021502018002124
:1073D00081600369002B05D0AD20C0002258012038
:1073E0000221984747482258062A11D801210B4606
:1073F0009340582213420BD0215020180021816065
:107400000369002B04D00348225802200146984704
:10741000002010BDBC0A0000F0B581B00024022895
:1074200003D9E443204601B0F0BD17460B46094E90
:10743000464309488519284618302A2107A2FCF737
:10744000B1FE42202F52032003498851204601B04B
:10745000F0BDC0465405000064AE01022573000073
:10746000F0B585B0C14D2C68002C0CD0C04FBF4C7E
:10747000E659002E0CD0C04FE659002E0DD000204A
:10748000C04305B0F0BD01AC0FC400272E4608E094
:1074900001AE0FC6E619012703E001AE0FC6E619DB
:1074A0000227D84C30462146FCF762FD02203060AE
:1074B0007C432919029D4D60CF60039808610498B0
:1074C000486108464430CC3101225602102332462E
:1074D000FCF744FFCC480019B32189004118012D65
:1074E00005D1B83001233246FCF723FB04E07430A9
:1074F00010233246FCF732FF01980760002005B0E8
:10750000F0BDC046A80A000001460020022901D9AA
:10751000C0437047DB4A4A43DB4988507047C04646
:10752000022806D8E6494143E64840180249401877
:1075300070474B2080007047D4040000022802D915
:107540004B2080007047E6494143E64840184D21F2
:10755000090140587047C046032801DB03487047C3
:10756000DF494143DF484018183070471E49010089
:10757000022806DCDA494143DA4840184221405AE1
:10758000704700207047C046032801DB0020704789
:10759000D3494143D348401844307047022804DCA3
:1075A000CF494143CF484058704700207047C046FC
:1075B000022805DCCA494143CA4840184068704760
:1075C0000020704780B5022801D9002080BDC44941
:1075D0004143C44840184430FCF77BFE014640421A
:1075E000484180BDB0B50024E14302280FD8BC4A11
:1075F0004243BC4B9D58042D09D0991801220A60C2
:107600000B69002B05D04A6902219847214608469C
:10761000B0BD2046B0BDC04610B50024022801D937
:10762000E04310BDAE494143AE4A072353505118C1
:107630000B69002B03D04A69002421469847204655
:1076400010BDC04610B50024022801D9E04310BD8A
:10765000A3494143A34A0623535051180B69002BF9
:1076600002D04A6901219847204610BD10B5002478
:10767000022801D9E04310BD99494143994A511864
:107680000B69002B02D04A6903219847204610BDA0
:1076900064AE0102F0B583B017460024E24302282D
:1076A0001AD8002B18D00D468D4941438D484618F5
:1076B00070680128029312D1002F0AD0B836002436
:1076C00029193046FCF73DFA002825D1641CA74251
:1076D000F6D1029807600022104603B0F0BD019277
:1076E00074363046FCF7F5FD002811D00346426899
:1076F000BA4209D2196828461D46F8F73BFD2B46C9
:10770000686802990860019430461946FCF7B7FD95
:10771000019A104603B0F0BD0298046000221046A2
:1077200003B0F0BD540500006E480168062909D079
:107730006B49415806290BD00F49415806290ED0F4
:107740000020704701218160654941580629F3D125
:10775000084901224250084941580629F0D1AB217D
:1077600009010122425000207047C04664AE010268
:10777000540500005C050000A80A0000F0B581B0C7
:1077800004460020C343022C02D9184601B0F0BDC4
:1077900015460E461B4A62431B498F18796801291A
:1077A00010D1002D28D01C460090B83738463146FD
:1077B000FCF7A0F9002821D1761C6D1EF6D10098A7
:1077C00001B0F0BD0090743738462946FCF79CFDA7
:1077D00000280CD00446006831462A46F8F7CAFC57
:1077E00038462146FCF760FD009801B0F0BD07A0C7
:1077F0002146FCF73DFA009801B0F0BD204601B0EB
:10780000F0BDC0465405000064AE0102536F636BC7
:1078100065745B25755D20526563762042756666EA
:1078200065722046756C6C0D0A000000F0B583B0DF
:10783000154607460022D043022F19D8002D17D035
:1078400000AB07C30F4878430F490E184436304643
:107850002946FCF759FD00280CD004460068019920
:107860002A46F8F787FC30462146FCF71DFD0298B2
:1078700003B0F0BD05A03946FCF7FAF9009803B053
:10788000F0BDC0465405000064AE0102736F636B27
:1078900065745B25645D2073656E64206275662087
:1078A00066756C6C0D0A000002460020022A04DC9A
:1078B0000B4B53430B4AD1507047C0437047C046EF
:1078C0005405000064AE0102022801D9002070476F
:1078D0000349414303484018034940587047C04694
:1078E0005405000064AE0102CC040000F0B581B084
:1078F000354CA06A0025002828465ED0334E3278E9
:10790000012A11D1E548808A314909680122814262
:107910000ADA0020A0716178002905D0A07160709A
:10792000022001F00DFC3278DC4FB98A284800684B
:10793000884201DC002A0ED1A279531CA371152ABA
:1079400009D36278002A06D10120607001F0F8FBAB
:10795000B98A1F48006888420DDA2078002801D0D3
:107960000020207000202071E0621A4908703078F1
:1079700000280CD118E001212171E26A531CE36256
:10798000FB8A9842132A04DA307800280CD001B020
:10799000F0BD2078002800D121700020E0620D4861
:1079A000017030780028F2D12078002801D1012020
:1079B00020700948064908600120E56220710549E8
:1079C000087001B0F0BDC0469898010230990102DC
:1079D0005C990102C5960102FFFF010080B50448D1
:1079E0000168491C01600069002800D0804780BD03
:1079F00024E00102014802490160704784900102BD
:107A00000026B80310B5F448002484611030022128
:107A1000024A2346FFF724FD204610BDC97A000024
:107A200070B584B0FDF724F8012815D1FCF74EFAA3
:107A30001F4D6861A969022914D0002909D129784C
:107A400000291ED0E969411A062902D300212970B4
:107A5000E861002004B070BD15480021816100205C
:107A600004B070BD13492A6A904202D10A78002AF4
:107A7000EFD028620020087000F018F9002004B050
:107A800070BD0126AE61AB88E88829896A8900AC9F
:107A900007C4B102084C09A22046FCF783FB286901
:107AA000AA892146FFF7B8FC2E70002004B070BDF3
:107AB000789601024893010250C5010225752E25D2
:107AC000752E25752E257500F0B58FB0032909D8C0
:107AD0007944097949008F4401070F15624881698B
:107AE00001290AD00FB0F0BD5F4881690129F9D1A1
:107AF000022181610FB0F0BD5B48002181610170FE
:107B00000FB0F0BD00250295574C20695749584ADF
:107B100002ABFFF7BFFD0028E4D1032055A20146C8
:107B200009F0A0F8514856A10A22F8F758FB00289E
:107B300013D04E4855A10F22F8F751FB0028D1D1A0
:107B40004A482C2103AA0C23FCF73DFB0498FCF7C0
:107B500013FA422160520FB0F0BD44482C2103AA11
:107B60000C23FCF730FB0698FCF706FA4221605222
:107B700080B2984989888142B4D10498FCF745FBCA
:107B80006063059801794279120251188279C379AC
:107B90001B029A18120451188278C378067840782C
:107BA000000280191B029A1812041018A062E162E8
:107BB0000798FCF7E1F94421019160520898FCF71D
:107BC00024FB4626A0530998FCF71FFB4827E053E7
:107BD0000A98FCF71AFB4A216054616B491E06297A
:107BE00001D80122A270062932D8C0467944097909
:107BF00049008F44031E14181B232A00A05B7549FB
:107C00008882E05BC8820198205A898D81421FD00A
:107C1000244902220A606F498885234800E02048F1
:107C20000121017014E06B48858711E00120E070AC
:107C30000EE01C4805606748858509E0C0B26549CB
:107C4000C8863C214143E18102E0012061498887E7
:107C50000120A07000F02AF807F0ECFDA562E562B3
:107C6000A5700FB0F0BDC0467896010250C5010264
:107C7000FF030000CAD5B5BDCAFDBEDD0D0A000078
:107C800024696E7374727563742C0000246D6573BF
:107C9000736167655F7265706C792C003AA90102A7
:107CA000C4960102C09801023C900102F0B5CFB029
:107CB000484CA0881490484D68781C90FBF7ACFDA8
:107CC0001B90A08D1A9068781990444800781890FD
:107CD000A08A1790E08A1690414801681591436880
:107CE000404903C9AA78404E3768404E3678283557
:107CF000089009910A950B920C970D961B9800908D
:107D00001A98019019980290189803901798049067
:107D1000169805901598069007931C98012801D095
:107D2000344A00E0324A2C4E149B1DA8C8210AF0A8
:107D30008FFA0246F078002842D0A0881C90FBF70A
:107D40006BFD1B904020205A1A90A08D19902A4854
:107D500000781890214800781790A08A1690E08A41
:107D600015901F48076843681E4806C8B0781490ED
:107D70001D480668E08E13906488E0B2240A1094CF
:107D80001190089709930AA826C014980D900E9692
:107D9000114E13980F901B980090199801901A9803
:107DA00002901898039017980490169805901598CB
:107DB00006901DA8C821114A1C9B0AF049FA0246E8
:107DC0000020F0700949087030691DA9FFF72EFDE9
:107DD0004FB0F0BD3AA9010278960102AB980102BA
:107DE00010990102089901025C9901029F98010211
:107DF000B23F0100F63F0100C7960102633F010058
:107E000080B582B00E4908680022C2600192CA683B
:107E1000002A02D0016801A8904702B080BDC04688
:107E200080B582B0064908690022C2600122019231
:107E3000CA69002A02D0016801A8904702B080BD3B
:107E400020930102F0B583B01348007800281ED0BB
:107E500000224024114B1146009003E0A41C521C48
:107E6000824215D29F5C7E1C9E54092FF6D81D5B62
:107E70000295C8B2019141005D1819464023029F46
:107E8000EF520B4601991E540098491CE6E7002169
:107E90000148017003B0F0BD30990102009A01025F
:107EA000F0B589B00AF0F8F8EA4C607809F09AFE6B
:107EB000E9498A8807A882800A88498809048918BC
:107EC000079105F0D3FC6078052804D00222E3492D
:107ED000092804D104E00122E049092800D08918CA
:107EE00049792078621C09F041FF607A07F0C0F8F8
:107EF000DB48DC4904F0FCFEDB4C2078002600283F
:107F000006960AD0D9491A31D94A034610CA0C80BC
:107F1000891C5B1EFAD14600D34CD64DA872D648B8
:107F200000886871D549097829706178E970000A7C
:107F3000A871481C607028460B30CC4F39464C3134
:107F400003913246F8F716F970190B3039461A3199
:107F50003246F8F70FF92020687206982071E08801
:107F60006870000AA870C320840106F045FD03195B
:107F7000BD48C362BC48007881000D31012228460B
:107F800006920AF007F9B8498862B748C46A06F051
:107F9000C9FC0019B44C07F0CDF905460E46AD48B2
:107FA000007B07F053F881B2C90B401800B2C1172B
:107FB00040102818A0657141E16506F01DFDA06123
:107FC00004F006FE0028FBD106F016FDE0617D20DE
:107FD000060100273846394632460AF08FF8A0627B
:107FE000677106F009FD2178A54A4A438118A64821
:107FF0000818421C01D1A3480818206306F0FCFCB5
:108000006063216B884204D3A04A8918884200D853
:1080100097E006F0F1FC606306F0EEFCE06104F02E
:10802000D7FD0028FBD106F0E7FC2062607902282A
:108030004FD001287DD100206071954D697A2129AA
:1080400071D16979AA79120251188B4A128891422A
:1080500069D18A4909782A788A4264D16978AA78EC
:1080600012025118A181E278002A40D02278002A19
:108070000BD07E4B4C3300201C888C4204D09B1CC0
:10808000401C8242F8D11046774CC0B2E081236E8A
:10809000A16BA26D7E4D2C4622340094724C01914E
:1080A000029229461A311E352A46FFF747F9E08920
:1080B000E178884208D341006C4A5118A2894C23C8
:1080C000CA522178491C21700521684A1154704810
:1080D00024E000206071014632460AF00FF8A062E9
:1080E00006F08AFC206206F087FCA06121E04C20AB
:1080F0005E4A11520698207005201070236EA06B06
:10810000A16D2A46223200920190029129461A312D
:108110002A461E320020FFF711F928469621F8F76B
:1081200042F80020208200200146324609F0E6FF96
:10813000A062226B606B55495118904200D365E7ED
:1081400067E70126304602F0AFF830460AF000F843
:10815000A06DE16DFBF7EAF8A770207800282FD01A
:1081600043484C213D463C46404B05E0891C001DE0
:10817000FAB26D1C95421AD25E5D002EF6D0761EC4
:108180005E55A3000693F6B22246424CE650374BAA
:108190005E5A5300404CE6527F1C334B9F7003687D
:1081A0003E4C069EA3511446304B541CDEE705920C
:1081B0002D48C77007700497F8B2022806D228E04D
:1081C000E77805970497F8B2022822D30598441E51
:1081D0000021069403E0491C069CA14219D02F4AB5
:1081E00010682D4B2B4F0FE0156050605D881E8886
:1081F0005E801D8060CF083F3E607D60641E121D62
:108200009B1C3F1D002CE6D05568A842ECDC28469C
:10821000F4E704980006059C10D062001E490398FC
:10822000F7F7A8FFA20012481C49F7F7A3FF0F4A6F
:10823000184802C81170521C641EFAD10A4883897A
:108240000B4800680090032015A2014608F00AFDC3
:1082500009B0F0BDCA900102242D0100D0A0010296
:108260009D0E0100B1F70000C896010218980102A6
:1082700028D2010216EA0102D4980102A498010250
:108280008024010001CF030000CF03000026B803C3
:1082900078D301021CE90102E4E9010280E901024C
:1082A000BBF9D5BE4944A3BA25582CBEE0C0EB3A71
:1082B0002025640D0A00000080B5002008F04CFF66
:1082C00080BD80B5012008F047FF80BDF0B581B0CA
:1082D00003F05AFF164CE060A178002901D001B0EC
:1082E000F0BD21790029FAD10121217100281BD08C
:1082F0008D02281AA168814216D0604E2F46A068D0
:10830000305C21698847A068401CA060681EA16895
:10831000814201DD0020A060E168A068022F03D344
:10832000691A7F1E8842EAD10020207101B0F0BD99
:10833000F8950102B0B5284C2368002B07D0022B1A
:108340001CD0012B38D109F073FE00F03BFC09F082
:108350004DFE2368012B2BD0022B2DD11F48017815
:10836000002929D122494A8A531C4B820223152A0B
:1083700022D301220270002048821DE0174D287888
:1083800000281FD0032016A2014608F06BFC002035
:10839000287009F04DFE00F041FD144D2870FBF7E8
:1083A0008DF809F023FE28780028D2D00120206023
:1083B0000F48002141820123032014A2014608F046
:1083C00051FCB0BD0A48408A14210B1A032009A2AF
:1083D000014608F047FCBCE7C09801023C9001024E
:1083E000BFAAC6F4CBD1CBF70D0A0000A6980102B4
:1083F00030990102B5C8B4FDBDF8C8EBCBD1CBF7BD
:10840000C4A3CABDA3BA25640D0A0000555742D7BC
:10841000B4CCACA3BA25640D0A00000080B50548B1
:108420000068022805D809F003FEFFF739FD09F0BE
:10843000DDFD80BDC098010270B50E2500242846E0
:10844000214604F001F80D20214603F0FDFF012430
:10845000204608F089FD04262846314603F0F4FF43
:108460000920314603F0F0FF204601F06DFBA20227
:108470000249034B204609F075F870BDE8CD0102B2
:108480009D17010080B5032810D800290ED07C224A
:108490004243BF488018C268012A07D12030FBF749
:1084A00050FB002801D00020C04380BD0020C04305
:1084B00080BDC046F0B589B00022D543032800D95D
:1084C000ABE00C46002900D1A7E00095216A072700
:1084D000534DA9420EDC574DA9421ADD564A91422E
:1084E0002FDC4B22D501A9423ED0120291424BD142
:1084F000042246E04B4A914217DD4B4A91422ADC66
:10850000E1221203914231D0494A91423CD10C22DE
:1085100037E04B252E01B14233D06A01914227D07A
:10852000AA01914230D102222BE0E1225502A94258
:1085300020D09502A9421FD0D202914224D1092213
:108540001FE04B225202914218D0E12212029142C6
:108550001AD1062215E0E1225203914210D0334A8B
:10856000914211D10D220CE003220AE00A2208E018
:10857000012206E0072204E0082202E0052200E0D2
:108580000B22D1002D4A57587C214143804A50503C
:1085900056182068B0606068F060A1683161E268D8
:1085A00072610025059503230493039502950197B5
:1085B0000695079501231B020893012807D0002880
:1085C0000AD18818009A8018B161F06104E0304641
:1085D00020300123FBF7ADFA206970636069B06356
:1085E000E069B067A069F063706801A908F0E6FE71
:1085F0002068012806D830464030234610330ECB81
:10860000FBF7ACFE6068012807D1301D70360068AA
:1086100001220B4B314608F0A5FF284609B0F0BDFA
:10862000FFC10100FF0F0E00FF1F1C0080841E0011
:1086300040420F007F250000FF950000542D0100EF
:10864000B5170100B0B50C467C214843504A1518B7
:108650002846FBF78DFC6C600020B0BDF0B583B000
:108660000024E743032800D98EE00E46002900D1FC
:108670008AE01546002A00D186E07C214143444827
:1086800041188868022832D001283AD000282BD11E
:10869000EFF31080C00702D1EFF3108072B60291A1
:1086A0000846403001902946FBF72EFE002863D093
:1086B000014601980F46FBF7F7FD386831462A4618
:1086C000F7F758FD0198FBF704FEEFF31081C90797
:1086D00003D1EFF3108172B662B602994D6806C8F5
:1086E0002C4B284609F080F8204603B0F0BD4868BE
:1086F000002431462A46234609F076F8204603B086
:10870000F0BDEFF31080C00702D1EFF3108072B616
:1087100002910846403001902946FBF7F5FD0028FC
:108720001ED0014601980F46FBF7BEFD3868314662
:108730002A46F7F71FFD0198FBF7CBFDEFF31081F9
:10874000C90703D1EFF3108172B662B602994D6882
:1087500006C8104B284609F047F8204603B0F0BD84
:10876000EFF31080C0070FD1EFF3108072B662B63E
:108770003C46204603B0F0BDEFF31080C00703D1A4
:10878000EFF3108072B662B63C46204603B0F0BDEF
:1087900060BE0102B91A0100B0B582B0602833D0C2
:1087A000622843D0642854D101A82F490180EFF3F7
:1087B000108072B600242046214602F0ABFC2B4DFF
:1087C000002805D1012002030020294602F0FCFB0D
:1087D000103501AA02232046294603F0F7F862B6B5
:1087E00023A0FEF78FFD64201B490C5207F022F8EE
:1087F0001A4801F059FDBFF34F8F1948194901601C
:10880000BFF34F8F00BFFDE76020134900220A52DB
:1088100007F010F8114801F047FDBFF34F8F1048E3
:1088200010490160BFF34F8F00BFFDE762200A4986
:1088300000220A520A8006F0FDFF084801F034FDCC
:10884000BFF34F8F064807490160BFF34F8F00BF4A
:10885000FDE702B0B0BDC0463AA90102A086010002
:108860000CED00E00400FA05AAAA000000D0020402
:10887000BDF8C8EBC9FDBCB6C4A3CABD0D0A000053
:10888000F0B5D1B0AC490A78002A24D0A94EF28BB9
:10889000002A20D1A94DAA68082A75D8930001A4FE
:1088A000E3589F46C9880000898900008989000033
:1088B00099890000C3890000CD890000D789000094
:1088C000A7890000E1890000552800D0A1E001201F
:1088D000A86051B0F0BD4978002900D19DE0974EC5
:1088E00072799B498854B179B071F171521C7271DF
:1088F0000A2800D091E00D2900D08EE003A8019055
:1089000037A8009034463834914892491DAB22462E
:10891000F7F782FCF06090A105222046F7F75FFC94
:10892000002800D0A7E01DA8002421460AF059F92C
:10893000B061F16137A821460AF053F930627162E3
:1089400022462346F7F7B4FF002800D085E0B0693F
:10895000F16900221346F7F7ABFF00287DD180486C
:1089600000F0FCFF1DA8002529460AF03AF9B06284
:10897000F16237A829460AF034F93063716303A81D
:10898000F7F7DCFC306169E0AA2838D1012A36D13A
:108990000220A86051B0F0BD0421A9600021A97097
:1089A000687051B0F0BD2979654A5054481C28714F
:1089B0006978491FC0B281422FD10820A86051B008
:1089C000F0BD0522AA60887051B0F0BD0621A960F3
:1089D000A87051B0F0BD0721A960287051B0F0BD5A
:1089E0006A78062A02921AD3531F0025544A2C464D
:1089F000575DE419A4B26D1C9D42F9DB10E0032819
:108A000007D1022A05D10120E8700320A86051B0E7
:108A1000F0BD0020A870A860687051B0F0BD0024BF
:108A20002018029A821888781118444FBD78491985
:108A30003C780919FA78002A00D0C91CC9B2FF296C
:108A400059D101282DD0022855D11E2D5AD1FFF71A
:108A5000F3FC0120F08351B0F0BD306900280AD04A
:108A60004048047040480470404804804048047006
:108A700009F084F8346136489621F7F794FB1DA875
:108A800064242146F7F78FFB37A82146F7F78BFBC5
:108A900003A82146F7F787FB00207071F08051B0E2
:108AA000F0BD284A9471032010719070AA20507074
:108AB0005520107068085071651DD5704000311840
:108AC0001646D01D2246F7F755FB301DE11CEAB2D1
:108AD000D21C037892B2D218401C491EF9D1A019B9
:108AE000D143C171090A01720934012000233146C2
:108AF000224608F079FE0020B870B86038717870AE
:108B000051B0F0BD70190E4E31462246F7F732FBD8
:108B10003078012802D12846FFF73EFE06F08AFE93
:108B2000BFF34F8F084809490160BFF34F8F00BF63
:108B3000FDE7C0463AA9010218900102E09801023F
:108B400084CD0102EC9A01020CED00E00400FA056C
:108B5000ECCC0102F13E0100474E474741000000C6
:108B6000A1AD010230940102C7960102A2AD01023B
:108B7000C696010210B5042003F086FB0446FBF7FD
:108B8000A5F9002C05D00E4C2063FBF79FF960631C
:108B900010BD0B4C216B401A042806D30120E07154
:108BA000FBF794F92063FFF781F8FBF78FF9616B0E
:108BB000401A0B28ECD360208A4901220A5210BDCA
:108BC00098980102F0B585B009F066FA7E487F49B1
:108BD00004F08EF87E4C00252571E57005F00CFF41
:108BE00060627C4E726828460495294609F086FA30
:108BF000607105F001FF0546A06327204101706800
:108C000048430A21F7F766FAE0634119481C00D08F
:108C10000846206405F0F0FE6064216C6E4D8842C9
:108C200002D34919884237D96C4E6D4F05F0E4FEE6
:108C3000606403F0CDFF00280ED0FBF7D7FEFFF7EE
:108C400099FFFBF7F7FD05F0D7FE6064216C8842C1
:108C5000EFD949198842ECD2E07801280ED130785A
:108C6000397881420AD1707A202807D17079B17998
:108C7000090208185B49898D884234D055484268FA
:108C80000020014609F03AFA6071216C606C88425C
:108C9000CCD349198842C9D80125284601F004FBE4
:108CA000284609F055FA2079002802D0002005B0A6
:108CB000F0BD4D4806F046FE4F4E3378032050A2DB
:108CC000014607F0CFFF3078411C31700628EDD304
:108CD0005148022101600498307060823D4805705F
:108CE000002005B0F0BD012020713F48623006F041
:108CF00029FE05F081FE2062B27A0392A27070799B
:108D0000B17909020818E08131460B315500374F1F
:108D1000384602912A46F7F72DFAA9190B31384641
:108D200032302A46F7F726FA039A002A049835D0FB
:108D300000262F4D03E0BF1C761C964210D23888C7
:108D400029688142F7D1788EA0812649898908183F
:108D5000788601B2E0890022FEF72AF9A278EAE7D4
:108D6000002A10D029680020029D16462A786B78C8
:108D70001B029A18914209D0AD1C401C3246864213
:108D8000F3D1104608E00020024605E0C5B22846AF
:108D9000FAF750FA2A46A078824202D1C0B2FAF716
:108DA00049FA14480B494860134800210170062015
:108DB00020560C498B8DE16A0091019003200F4AE7
:108DC000014607F04FFF67E7750E010001F700004D
:108DD000309901023C900102007C3125E0D2010271
:108DE000A49801023AA901021A3F0000749A0102F4
:108DF000D498010288130000DED201023A4001003B
:108E0000B2E2BEE0CAA7B0DCA3ACBCC6CAFDA3BA3E
:108E100025640D0A00000000C0980102F0B587B07B
:108E200009F03AF97F4C607A08F0DCFE7E498A88C6
:108E300005A882800A88498809048918059104F0E8
:108E400015FD607A052804D002227849092804D14A
:108E500004E001227549092800D089184979207A4F
:108E60002246093208F082FF607C06F001F9704862
:108E7000704903F03DFF704F0024FC7005F0BCFD0D
:108E800078626E4D2046049421462A4609F036F950
:108E9000787205F0B1FDF8646949B863F963411867
:108EA000481C00D00846386405F0A6FD7864396C8B
:108EB000644E884202D3891988423BD9624C03F040
:108EC00087FE002810D0FAF7F9FAFBF78FFDFFF7BD
:108ED00051FEFBF7AFFC05F08FFD7864396C8842DA
:108EE000EDD989198842EAD205F086FD3862F87812
:108EF00001280FD120785549097881420AD1607A3A
:108F0000202807D16079A179090208185049898D74
:108F1000884218D005F070FD7862002001462A468C
:108F200009F0ECF87872396C786C8842C7D38919EB
:108F30008842C4D8022001F0B7F9012009F008F9ED
:108F4000049807B0F0BD434806F0FCFC42483549A0
:108F5000486005F051FD3862A27A0492BA706079D7
:108F6000A17909020818F88121460B3156003B4DC2
:108F7000284603913246F7F7FDF831190B312846A0
:108F800032303246F7F7F6F8049A002A29D0002446
:108F9000334E03E0AD1C641C944210D22888316823
:108FA0008142F7D1688EB881294989890818688675
:108FB00001B2F8890022FDF7FBFFBA78EAE7002A40
:108FC00011D031680020039D14462A786B781B026B
:108FD0009A1891421DD0AD1C401C22468442F3D108
:108FE00002E0002203E000221446944202D1D0B2F3
:108FF000FAF720F90620385615498B8DF96A009149
:1090000001900320174A014607F02CFE012007B00B
:10901000F0BDC4B22046FAF70DF9BA789442E9D10E
:10902000E5E7C0463C9001022A2D0100D0A00102D4
:10903000750E010001F700003099010280841E00C6
:10904000004C7007007C3125E0D20102A498010297
:109050003AA90102D23D0000204E0000749A01029C
:10906000D49801023A40010080B582B000200190FE
:109070000448C268002A02D001A80021904702B02B
:1090800080BDC04694950102F0B583B0002420460F
:10909000FDF788FEFDF7ABFE274EB060FDF7A4FE9E
:1090A0007060264F0BE001A8C1888088084319D161
:1090B00001A8408824180834B068844235D201AD34
:1090C000082128462246FDF779FE28880028EAD0A4
:1090D000B8422AD001AD0421284601F0CFF8A98872
:1090E0008842E5D03460B06884420CD201AD0221E0
:1090F00028462246FDF762FE2888B84203D0A41C09
:10910000B0688442F2D370682118491E404208407A
:1091100030600DD00024254601202946FDF726FEAB
:1091200003CE4D19083E8542F6D3346003B0F0BD3E
:109130000024346003B0F0BD30970102FFFF00004F
:1091400010B5054C6070FEF7B1FD6078022801D1C2
:109150000020607010BDC04678960102C8480149E1
:109160004181704701030000F0B585B01F460492AD
:109170000646C8170C1844400A2C039114D3012545
:109180000A212046F6F7A6FF6D1C632C0446F7D88B
:1091900004998D4200D329460A9C002F09D00398D8
:1091A000002808D4002207E0012504998D42F2D25C
:1091B000F2E7002205E00122042323409B08134329
:1091C000FA1A0223234004980028029412D1002B9B
:1091D00010D0F468002C62D40398002825D402989B
:1091E000400734D57068B5686F1C87422FD8306847
:1091F0002B2423E0E407ECD1002A0AD1E9E7376801
:1092000020203855B560F068441CF460521E002CD4
:10921000DFD49142DDD27768B468651CBD42EED9D7
:10922000F468521E002CF4D5D3E7404203907068D6
:10923000B5686F1C87420AD830682D244455B76042
:10924000F068441CF4600025ED43A84227DB002BA6
:109250001CD00120029B1840049B184316D1002A01
:1092600003D113E0521E002C0ED491420CD2706830
:10927000B3685D1C8542F5D830683024C454B560AD
:10928000F068441CF460EDE7002C08D400920298CA
:1092900001900A2230460399049B00F003F805B0C0
:1092A000F0BD0000F0B587B01F46154602900124BE
:1092B00006919142009407D3012406982946F6F7B7
:1092C00009FF641CA842F9D20D980C9ABC4203977E
:1092D00000D3039400990140002A009109D000298D
:1092E000029C25D12021800705D40846002F11D0EB
:1092F00004E0029C1CE03020002F0BD0084609E05F
:1093000023685854A260E168491CE1603246721E2D
:1093100000290DD4039991420AD216466368A168C8
:109320004A1C9A42ECD9E1683246721E0029F1D5F6
:10933000E068002859D40590012401E07F1E6C43A9
:10934000022FFBD2069821461646F6F7C3FE324698
:10935000A842F4D2029880680490069F019506976F
:1093600038462146F6F7B6FE049D691C029F7A68CE
:10937000914206D9069F059A019D0592002A0ED5B5
:1093800016E01B4A125C3B685A55B960FA68521CD9
:10939000FA600491069F019D0592002A08D460435B
:1093A0003F1A20462946F6F795FEAC420446D6D22F
:1093B00000980028029C059B049D16D0002E14D016
:1093C000701C01E0002B10D4401E039981420CD286
:1093D000691C62689142F5D8226820235355A16028
:1093E000E268531CE3600D46ECE707B0F0BDC046F1
:1093F00030300100F0B583B001900291002923D0F4
:1094000000251F4E2F460AE01F480818410F40183C
:10941000C010F0747F1CB8B20299884214D201982F
:1094200000884B24210100B200F05AF8400061018D
:109430004018308401B2114881422846E9DB1148C6
:109440008142E1DD6420E4E70C2002F025FF2021C9
:109450000B48415E094A914201DA0CA207E0002163
:10946000817015480078012102F098FF13A20320B3
:10947000014607F0F7FB03B0F0BDC046E40C000066
:1094800098980102041000001CF3FFFFB5E7B3D861
:10949000B5E7D1B9B5CDD3DA332E3356A3AC3447C3
:1094A000A3AC4750532CC2EDB4EFCDA3D6B9B9A4A9
:1094B000D7F70D0A00000000C6960102B5E7B3D841
:1094C000B5E7D1B9D5FDB3A32C3447A3AC4750536E
:1094D0002CC2EDB4EFD5FDB3A3B9A4D7F70D0A00A4
:1094E000074A904201DD054A801800B24143C8177F
:1094F000400D0818C00A00B27047C04600F0FFFFD8
:10950000FF07000010B50078012819D1AC480269A6
:10951000012A04D1614A13680124A343136003297B
:1095200005D080214161C269002A05D107E00121EF
:109530004161C269002A02D001898069904710BD4B
:10954000FF222E32024803A107A306F02FFBC046DC
:10955000E43B01006164635F646D615F63616C6C37
:109560006261636B00000000556E6578706563741E
:10957000656420646D61206368616E6E656C0D0AC0
:1095800000000000F0B58DB00D460124EFF310810E
:10959000214002D1EFF3108372B6894E73690F2B0D
:1095A00006DD102B37D0402B2FD0802B2DD005E09F
:1095B000002B2AD0012B01D110237361B581358195
:1095C000B061F261002900D162B63179002929D059
:1095D0000294304C05A90A4604950390E8CCE8C2F1
:1095E000E8CCE8C2029C204600F0CEFE2A4800905B
:1095F0002A4D294608312046039A049B00F034FF87
:109600002C60002420460DB0F0BD0029FAD162B6CE
:1096100020460DB0F0BD02240029F3D162B62046E9
:109620000DB0F0BD3178002907D01C4807218161B9
:109630000460002420460DB0F0BD3269B38917499B
:10964000002B15D0B5693089012A02D0002A03D039
:1096500003E09FB2874200D10C604F68FF07FCD047
:109660008F6880C55B1E1F04EED10023B381B561F6
:10967000012A02D10A68A2430A607461F2690024D7
:10968000002ABFD0B36931898800181A9047204654
:109690000DB0F0BD703001000595000008D001400C
:1096A000F0B581B0002856D00446424EF0688007DD
:1096B00054D41325284600F01FFD284605F0C4FEAB
:1096C00027686168012538462840CA07920F10189C
:1096D000227C1207120E8018627C1207120D80186D
:1096E000A27C1207120C8018627D13071B0AC01897
:1096F00012091206801830607D20060200293046CB
:1097000000D12D48E3681A0A7D2A1A4629D22B4E29
:10971000B3422AD200292BD0002A2946254E00D058
:109720001146F6F7D7FC401E80B2706024480761EE
:10973000E27C0270237D0371224F3E686902A468B7
:10974000012C1BD02C0226433E60002B1ED0012191
:10975000184A116329E0012001B0F0BD022001B0D8
:10976000F0BD3246154EB342D4D333460029D3D18F
:109770001A46002A29460F4ED2D1D2E73F242401AF
:10978000A6437618F0363E60002BE0D1002A0CD0BC
:10979000FF2212020C4B1C6894430122D203A21830
:1097A0001A60304A1160304A116001214161002085
:1097B00001B0F0BD00D001400026B80380841E0037
:1097C000A89501022C06004008E400E070B50028CE
:1097D00001D0012070BD0C461625284600F08CFCF7
:1097E000284605F031FE002C05D01B481830142205
:1097F0002146F6F7BFFC28211748415C002915D007
:109800004168002916D403220B469343144A9C58FE
:109810008D07ED0EFF26AE40B4439C501F220A4038
:10982000012191400F4A11600F4A1160012101612D
:10983000002070BD8A07D20EFF2393400F220A40FA
:10984000083A03218A43054954589C435450012146
:109850000161002070BDC046889001021CED00E04F
:1098600000E400E080E200E000E100E080B568484C
:109870000021017061480078C001614909788901BF
:10988000014360480078400108435F4909780901B5
:1098900001435E480078C00008435E4909784900EA
:1098A00001435D4800780843C0B2FAF7DBFF80BD92
:1098B00080B55748012101705148007880014F4917
:1098C0000978C90101434F480078400108434E49D7
:1098D0000978090101434D480078C00008434D490B
:1098E0000978490001434C480078084304210143AA
:1098F000C8B2FAF7B7FF80BD5A21014A50527047EB
:1099000068A00102F0B581B013490A78002A13D08B
:10991000052A01D104220A709300CD18561C002399
:109920001C462F686F60F917DB194C412D1F761EFE
:10993000012EF6DC084902E0002213461446486076
:10994000521C0A70C11718186141D2B20023F6F7F1
:10995000EBFB01B0F0BDC046C8950102F0B581B087
:109960000446007841424141217024480078C001FA
:1099700023490978890101432248007840010843BE
:10998000214909780901014320480078C0000843B3
:109990001F4F3978890001431E4D28784000084345
:1099A0001D4E31780143C8B2FAF75CFF7D20C0003C
:1099B00000F07AFC20784142414121700F48007844
:1099C000C0010F490978890101430E480078400120
:1099D00008430D490978090101430C480078C0008B
:1099E00008433978890001432878400008433178DA
:1099F0000143C8B2FAF736FF01B0F0BDEC9E010298
:109A0000C69601021D900102ACEA0102A1AD01025D
:109A1000ED9E0102DFD20102AC98010270B58B4EBF
:109A20003060112400252046294602F00DFD204615
:109A300029462A4602F038FC03222046294602F035
:109A40002BFD32680221204602F0A6FB2046294663
:109A500005F0DEFA70BDC046B0B57C4DA8600224AA
:109A6000002120460A4602F01FFC01210522204663
:109A700002F012FDAA680321204602F08DFBB0BD62
:109A80005C21C5480022425282847A2141840284AA
:109A9000C2830283C2820282114941608260C26035
:109AA0003D21490441834182090C818381827047B1
:109AB0005C21B9480022425282847A214184028486
:109AC000C2830283C2820282054941608260C26011
:109AD0003D21490441834182090C81838182704781
:109AE0004C37373770B5AD484C21016001252C0249
:109AF000601C00F081FA322000F0D6FB00F094F9EF
:109B0000284600F09BF9284600F0AAF800F086F9F4
:109B10000C4800F071FA00263046314600F07CFB1C
:109B20002846314600F078FB204600F065FA022016
:109B300000F062FA4834204605F0B0FF06F00EF857
:109B400070BDC0460102000010B50446072106F0B2
:109B5000E7FE3E48446010BDB0B50C250024284601
:109B6000214602F071FC012128460A4602F09CFBC6
:109B700002212846224602F08FFC04252846214671
:109B800002F062FC28462146224602F08DFB0522A7
:109B90002846214602F080FCB0BD70B505200424A3
:109BA000214602F051FC0620214602F04DFC0E2019
:109BB000214602F049FC0D20214602F045FC00241C
:109BC0000121204602F040FC02252046294622467B
:109BD00002F062FC0B2630462146224602F064FB6E
:109BE00030462946224602F057FC70BD80B507205A
:109BF00002F042FB80BD0000B0B50120104907F023
:109C0000DDFBF9F71FF90F48FFF74AFD0E48002169
:109C100001600E4D2A6811200224214602F0BCFA90
:109C2000AA680321204602F0B7FA0724204602F072
:109C300033FB05F093FF6868214606F071FEB0BD66
:109C4000E09401022490010200960102689601024C
:109C500002480168012291430160704758000040AA
:109C600002490A6802408242FBD17047046000400A
:109C7000B0B5494D28688107484C0ED528797F2119
:109C8000084022688A431018206023680B40022095
:109C90000321434A06F0E6FF286880040ED55E20C3
:109CA000285C7F21084062688A43101860606368FE
:109CB0000B40022003213B4A06F0D4FF172000F09E
:109CC0001BFA3948016802220A4301218A430260D3
:109CD00036483749016037480021C17181791F2515
:109CE00029408171817A427C837C1B029A18C37C53
:109CF0001B04D218037D1B06D2182F4B9A4218D191
:109D0000427B837B1B029A18C37B1B04D218037C03
:109D10001B06D218294B9A420BD1C27A037B491EEB
:109D2000122906D819028918254A914201D1202109
:109D300001720178CA0602D11022114301701C3C45
:109D400020682021884320601E481F490160416827
:109D50000029FCD503F0EEFC0446022003211BA2DF
:109D6000234606F07FFF0A20C441032C05D80220B9
:109D700003211DA206F076FFFEE71848C1680F22F6
:109D80009143C1600168164A0A400260192000012F
:109D9000144948600D60B0BDD0A0010248000040E9
:109DA0002C3C0100163C0100040200400C0600405F
:109DB000AF6B100A6B0001404D383650312E3236F1
:109DC0000734000000600040FE1C0080436869709A
:109DD0002049443A20253038780D0A00C8600040F8
:109DE000FEFFC3FF0C0400404F6C64206368697081
:109DF000206D6F64656C206973206E6F74207375BD
:109E000070706F7274656420627920746869732061
:109E100053444B2121210D0A0000000080B517207A
:109E200000F062F9002080BD10B51724204600F034
:109E300063F9204605F008FB002010BD0121C90789
:109E400001430148016070470060004080B56348ED
:109E50000021017062480078C001624909788901D7
:109E600001436148007840010843604909780901CD
:109E700001435F480078C00008435E4909788900C3
:109E80000143554800780843C0B2FAF7EBFC80BDA7
:109E900080B5524801210170524800788001504934
:109EA0000978C901014350480078400108434F49EF
:109EB0000978090101434E480078C00008434D4924
:109EC000097889000143444800780843022101438E
:109ED000C8B2FAF7C7FC80BDF0B581B00B2002F024
:109EE000D3F93B49097800282AD03A480022027069
:109EF000643948424841384A10704A1E9141374AF5
:109F000011704900081836490978C90140183549C7
:109F100009788901014334480078400108433349F6
:109F200009780901014332480078C00008433149EB
:109F3000097889000143C8B2FAF794FC01B0F0BD7A
:109F4000102940D324480024047025480078C0011B
:109F500024490978890101432348007840010843D6
:109F60002249097809010143214F3878C00008438C
:109F7000204D297889000143184E3078400008436D
:109F8000C0B2FAF76FFC347015480078C00115496B
:109F900009788901014314480078400108431349B6
:109FA0000978090101433878C000084329788900FD
:109FB0000143094800780843C0B2FAF753FC05484A
:109FC000047001B0F0BD03480121017001B0F0BD83
:109FD000AB980102AD980102AC980102DFD20102F8
:109FE000EC9E0102C69601021D900102ACEA01023C
:109FF000A1AD0102ED9E010210B5C1B2000AC2B2CC
:10A0000002290CD0012913D0002930D1911E7F489C
:10A0100002291BD20121032A2AD0490429E07B48C6
:10A020004168002A1FD00246203A1143416010BD0A
:10A0300076480168D31E022B10D3012A29D0002AAA
:10A0400041D1012292079143016010BD002A16D12F
:10A050000121490702688A43026010BD0123042AD6
:10A060001FD05A041EE0012292079143416010BDA7
:10A070000904194A7F32C36A13405918C16217494B
:10A080008A699207FCD50121490702680A430260E8
:10A0900010BD0522120791430246203A0A4302608E
:10A0A00010BD1A04836A0C4C1C40A21882620B4A31
:10A0B000131F00241C600A4B0A4C1C600D235B021A
:10A0C00014681C431460054A93695B06FCD505229D
:10A0D00012071143016010BD80FFFCFF1402004015
:10A0E00004010040FF0F0000012181404748026841
:10A0F0008A4302607047C04601218140434802689C
:10A100000A4302607047C04610B5052811D8C04602
:10A110007844007940008744020E192434393B49C1
:10A120000A680868C0003CD53A4820390A425DD028
:10A130003BE0002010BD35490A680868C00035D5ED
:10A1400034480B46203B1A4237D134E02F490A6885
:10A150000868C00036D52F480B46203B1A424CD128
:10A1600035E02A494C680120C0030A680B46203BB1
:10A170001C421AD00C68E4003BD5264C1A423CD055
:10A180003AE0224800680120C00310BD1F490A6858
:10A190000868C0001ED51F480B46203B1A4220D13C
:10A1A0001DE01B4820390A4220D010BD18480B463C
:10A1B000203B1A4201D10120C00349688900890F60
:10A1C000C84010BD12480B46203B1A4215D1012051
:10A1D000C00312E00E480B46203B1A4201D1012079
:10A1E000C00349680903890FC84010BD0120C0039E
:10A1F00010BD074C1A4200D020464A689200920FC8
:10A20000D04049680901890FC84010BD20000040B6
:10A21000006CDC020026B80304282CD8164AC0467D
:10A220007844007940008744020A121A2100032072
:10A230000007136883438807800818181AE0032072
:10A2400080061368834388070009181812E003206A
:10A250008004136883438807000B18180AE0FF2066
:10A260000002136883430802181803E01068FF23F4
:10A27000984340181060704724000040B0B5002299
:10A2800000290CD0074B047895B22D0A65406C006C
:10A290001C5B12026240491E401C0029F3D190B29F
:10A2A000B0BDC046302E010000280AD030B40725CA
:10A2B0002C02CD256419604340091238001FFDD8D7
:10A2C00030BC7047F0B583B01F4616460D460146B8
:10A2D000E8680291F6F798F804460F2E11D8082E78
:10A2E00004D320462146F6F736F809E0042E02D3BF
:10A2F0008120C10501E0412001062046F6F784F8DF
:10A3000004460999089E2B20C043874205DB20465E
:10A310000F462146F6F71FF80DE03F20C043874265
:10A320000BDA4920C04387420CDBFF200F46810532
:10A330002046F6F769F839460446688A0880346092
:10A3400003B0F0BD01915320C043874206DB204695
:10A350002146F6F700F80446688A10E0A8690299D9
:10A36000F6F77CFA002801D1A88B00E0E88BF6F71D
:10A37000D6FA01462046F6F747F804460020019930
:10A380000880346003B0F0BDF0B581B0054601200F
:10A39000072D66D80C46002963D04A4F38680169FA
:10A3A000C90736D105263046FFF7A6FE304605F030
:10A3B0004BF803CF0369012213430361002918D42A
:10A3C00003200B4683438E481E588807C00EFF2784
:10A3D0008740BE4340278740374389481F501F208E
:10A3E000084082408748026087480260354800681C
:10A3F0000FE08A07D20EFF2696400F230B40083B42
:10A4000003218B437D495F58B743402696403E4326
:10A410005E5069014018012109024218E369DB0618
:10A420009B0CA569ED00EDB2EB1853606268520712
:10A43000520B23685B075B099A18A3685B079B0CA8
:10A44000D218E3685B075B0DD21823695B01DBB2AE
:10A45000D21863699B07DB0ED21880231343435045
:10A46000002001B0F0BDC046F0B581B0002A23D075
:10A4700005460835134C2668F668EE40F50702D00D
:10A48000022001B0F0BD069D8600A619B56040010E
:10A4900024682018009301231D02461977680724B9
:10A4A000A7437760F16032610099B1604159194367
:10A4B0004151002001B0F0BD03A00AA174220DA3F8
:10A4C00005F074FBD8920102696E636C7564652FA8
:10A4D000647269766572732F6D6B5F646D612E6354
:10A4E00000000000646D615F7472616E7366657276
:10A4F00000000000496E76616C6964207472616EC0
:10A500007366657220647374206164647200000075
:10A5100000015849085840687047C046F0B581B0FE
:10A5200005460120012D4CD80C46002949D0002DAC
:10A5300003D0012D04D10F2000E00E20FFF7DCFD39
:10A54000A668012E04D0002E4FD1E08900284CD1FE
:10A550002901294843580020D860F507AD0F276826
:10A560006668B607360F76192569EA07920EB6189F
:10A57000022F04D0012F03D10122164300E0403600
:10A580001D4F9E60E2681A6079188D606269CA602A
:10A590004968002917D403220B469343184A9C5854
:10A5A0008D07ED0EFF26AE40B4438026AE40264315
:10A5B0009E501F220A4001219140124A1160124A06
:10A5C000116001B0F0BD8A07D20EFF2494400F2322
:10A5D0000B40083B03218B4308495D58A543802469
:10A5E00094402C435C5001B0F0BD08A00FA149225B
:10A5F00012A305F0DBFAC046209301021CED00E037
:10A6000000E400E080E200E000E100E0696E636CDD
:10A610007564652F647269766572732F6D6B5F6404
:10A6200075616C5F74696D65722E63006475616C31
:10A630005F74696D65725F6F70656E00636F6E66E3
:10A64000696720697320696E76616C696400000037
:10A650000001084A10580160816880220A43826024
:10A660007047C04600010349085881688022914321
:10A670008160704720930102F0B58DB001931546BB
:10A680000E460A901298002408900480149F3C8083
:10A69000139809900460159804900480FF208105A8
:10A6A0003046F5F7B1FE0290304603963146F5F795
:10A6B00052FE2B463D460690274607950B9311E028
:10A6C0001180188880002858099908600120079D8A
:10A6D00028800520049908807F1CBCB21888844219
:10A6E00000D9A0E028880028F6D1A0000A9D2E58A5
:10A6F00030460699F6F7A4F8002817D0304603999B
:10A70000F6F79EF800280B9B079DE5D1089A178065
:10A71000099D2E601888011B012934D110801988E9
:10A7200089000A9A51582960059035E0089A1780E7
:10A73000099806600B9B1988081B0128C0D00C964D
:10A74000019825187E1CB0B28542BFD389B2B2B23F
:10A750008A420ED880000A990C5820460C99F6F7C8
:10A7600061F80B9B002804D10998046008980680C2
:10A770000C94761CB0B28542A8D3198889B2B2B2C3
:10A780008A42E7D9F5E70C96019962187D1CA9B2B7
:10A7900016468A4205972CD2059884B2A5000A9ED7
:10A7A0007259002C104609D0A819001F01681046E4
:10A7B0000C92F5F7D0FD0C9A062C07D80446A81980
:10A7C00041681046F5F7C7FD0C902046079D029999
:10A7D000F6F744F800280B9B07D10C980299F6F77E
:10A7E0002FF80B9B002800D076E70120288003205B
:10A7F00070E780B2AAB282420FD888000A990C583A
:10A8000020460C99F6F70EF80B9B002805D1099805
:10A8100004600898058005950C946D1CA9B28E42C1
:10A82000BAD31888E5E70DB0F0BD0000F0B585B0EB
:10A8300001273904494D6868049188436860286895
:10A84000474901432960390746480160464803915A
:10A8500001600024204600F0BDFD4448017849B263
:10A86000002902D480220A43027068690290A86914
:10A8700001903F4803683F4E7360C36833603346BE
:10A88000143B1B68F3603346103B1B68336133464F
:10A890000C3B1B6873613346083B1B68B361331F75
:10A8A0001B68F3616C62FB052C460C3C20689843E6
:10A8B000206078046A6882436A6030BF6A68024335
:10A8C0006A602068184320602B4C029804400029DD
:10A8D00001D42648017007206862002000F08CFD3A
:10A8E000264803990160BFF34F8FBFF36F8F1D4858
:10A8F000016070681E4908603068C860002C08D08C
:10A900008C622046019A1040086320469043C8623A
:10A91000CC611B4801688906FCD50A242046FFF754
:10A92000C3FCF8022968814329602046FFF7BCFC7C
:10A9300038032968814329602046FFF7B5FC286861
:10A94000B8432860284614380068C002FAD5686801
:10A9500004990843686005B0F0BDC0462C00004073
:10A96000011C000080E200E000E100E0670001401F
:10A97000042000501C010040FFFF030080E100E0C4
:10A980002C0200400A490A680A4802400A60FD2178
:10A990004900094A1268515C002908D007490A6C2D
:10A9A00002400A64012000060A6882430A60704778
:10A9B00000040040FFFFFF7F489401022000004098
:10A9C00000207047F0B583B00D4604467C26464310
:10A9D00050488719F869396AF5F77CFBA84200D816
:10A9E00092E0019502940121EFF31080084002D11A
:10A9F000EFF3108272B63C4610343B690025062BFB
:10AA00000CD80A469A40D3065B0F06D161231A423E
:10AA100075D00D46002803D003E00225002800D1A0
:10AA200062B6002D02D0284603B0F0BD00943C462B
:10AA30002034384880591021C1613E46143605F053
:10AA400087F805463868C069C00605D505F080F866
:10AA5000401B31888842F5D90621029D284600F026
:10AA60002FFF206801994143B8690918386881604F
:10AA7000172179563C461734002909D5C16920228F
:10AA80000A43C2610121F966890502680A4302602E
:10AA90000521284600F014FF207840B20025002848
:10AAA000C1D42B4800687D24E100F5F713FB610158
:10AAB0004143029800F0D6FE05F04AF80446386893
:10AAC000C069C00705D005F043F8001B31888842F3
:10AAD000F5D905F03DF804463868C169890706D5FF
:10AAE00005F036F8001B31888842F5D93868012115
:10AAF000009A116053498161284603B0F0BD0321DB
:10AB0000216000288CD08CE7034804A1084A09A3DF
:10AB100005F04CF84C9301025C3C0100666C6173DB
:10AB2000685F626C6F636B5F6572617365000000E4
:10AB30005D020000626C6F636B206964782069734A
:10AB4000206F7665722072616E67650D0A000000E5
:10AB500038E00102F0B583B002907C214143934A72
:10AB60005418E56EEAB2511E02291FD229040126AB
:10AB7000090E18D001960092022100F0A1FE27468E
:10AB8000143704F0E5FF06462068C169890606D43B
:10AB900004F0DEFF801B39888842F5D92068007DEB
:10ABA000C007019E08D0304603B0F0BD032A36D15D
:10ABB00000922804000E36D020466C302D0C002167
:10ABC000019101602746143704F0C2FF0646206851
:10ABD000C069C00705D004F0BBFF801B39888842DC
:10ABE000F5D904F0B5FF06462068C169890706D586
:10ABF00004F0AEFF801B39888842F5D920681149DE
:10AC00008161E9B20120002911D003290099019E38
:10AC100000D006202061226F002A0ED1C3E7002653
:10AC2000304603B0F0BD0126304603B0F0BD0099B8
:10AC3000019E2061226F002AB5D002A890473046BD
:10AC400003B0F0BD000093EB70B5002801D00120E7
:10AC500070BD7825CD4E705D00280ED000240921EE
:10AC6000204600F02DFE0F20FFF71EFB1520FFF7FA
:10AC70003BFA74553461204670BD042070BDC04657
:10AC8000F0B581B00C460078484EF16881422CD175
:10AC9000032C54D1706EB16E884261D90024062114
:10ACA000204600F00DFE3068F16D8160204621469F
:10ACB00000F006FE354660352CCDF0683168B48C66
:10ACC000414F00975B1BA34200D81C46A3081431D8
:10ACD000FFF7CAFBB06E0019B066306E001930661F
:10ACE000F06D0019F06501B0F0BDB168814255D139
:10ACF000032C45D1F08CF16D0918F165316E0918FE
:10AD00003166B16E0818B066716E814238D9002480
:10AD10000621204600F0D4FD3068F16D81600121EC
:10AD2000204600F0CDFD316EB068F38C3268264CC1
:10AD3000009414329B08FFF797FB01B0F0BD306818
:10AD40001021C16104F004FF05463068C069C006E7
:10AD500016D504F0FDFE401BB18A8842F5D90FE0FC
:10AD600030681021C16104F0F3FE05463068C06907
:10AD7000C00605D504F0ECFE401BB18A8842F5D927
:10AD80000120C107326813688B431360F16E2204FF
:10AD90000A4300021043F06601B0F0BD4D200201ED
:10ADA000034804A1844B04F001FFC0464C93010208
:10ADB0005C3C0100666C6173685F646D615F636138
:10ADC0006C6C6261636B000081AC0000F0B581B017
:10ADD00000786E4DAA68824200D0D0E00126300291
:10ADE000032942D16A6DAA66AB6DAC6AA418EB6503
:10ADF0002C66AB6C5B1CAB646B6E934235D95E30DA
:10AE0000FFF752FA686CA96C02293AD3814238D113
:10AE1000E88C696D081868650020062100F050FD77
:10AE20002868E96D81602F6D04F092FE0446286861
:10AE3000C069C00705D004F08BFE001BA98A8842B8
:10AE4000F5D904F085FE04462A68D069800706D546
:10AE500004F07EFE001BA98A8842F5D92A68742076
:10AE6000285C012841D0F10440E0F2072B681C68FF
:10AE700094431C60EA6E090411430143E96601B082
:10AE8000F0BD0229FBD38142F9D2E88C696D091823
:10AE90006965A96D0818A8650020062100F010FD5D
:10AEA0002868E96D8160EF8C04F052FE0446286842
:10AEB000C069C00705D004F04BFE001BA98A884278
:10AEC000F5D904F045FE04462A68D069800706D506
:10AED00004F03EFE001BA98A8842F5D92A68742036
:10AEE000285C012822D0F10421E03105334B3B409E
:10AEF0005918012802D01920400601E00720C00699
:10AF000008182F4940185060002F0DD004F020FE83
:10AF100004462A68D069800706D404F019FE001B95
:10AF2000A98A8842F5D92A682B6D1FE03105234B89
:10AF30003B40C918012802D01920400601E0072033
:10AF4000C00608181E4940185060002F0DD004F0AC
:10AF5000FFFD04462A68D069800706D404F0F8FD96
:10AF6000001BA98A8842F5D92A68EB8C296EA8684B
:10AF7000144C00941432FFF777FA01B0F0BD044886
:10AF800004A10C4A0C4B04F011FEC0464C93010284
:10AF90005C3C0100666C6173685F646D615F777231
:10AFA0006974655F6E62797465735F63616C6C620E
:10AFB00061636B0072040000433C0100FF3F00002E
:10AFC00000808000CDAD0000F0B587B004460126BA
:10AFD000880E14D01546002A11D00F468120C004D7
:10AFE000401B88420BD37C206043F0490818059031
:10AFF000818C38460691F5F76DF8002902D030466D
:10B0000007B0F0BD28460699F5F764F80029F6D197
:10B01000059880693E1A30460699F5F75BF80746B1
:10B02000039670190190069E3146F5F753F80546D0
:10B03000C01B04900598006A02903146F5F74AF863
:10B04000049981420FD20026BD42D8D92046394604
:10B0500000F03CFB2046FFF77DFD0028FAD17F1C65
:10B06000AF42F3D3CBE700900398029D2946F5F752
:10B0700031F80646284670430399081A019800D013
:10B08000761C2946009D7543F5F724F80590029932
:10B0900041430198401A03900699F5F71BF8049074
:10B0A000AF420BD22046394600F010FB2046FFF796
:10B0B00051FD0028FAD17F1CAF42F3D30598864298
:10B0C000069D009F0CD220463146FFF77BFC2046B0
:10B0D000FFF740FD0028FAD1761C05988642F2D38E
:10B0E0000398A84203D20026304607B0F0BD059869
:10B0F00047430025E919204600F0E8FA2046FFF70B
:10B1000029FD0028FAD16D1C002604988542F1D350
:10B1100075E7C046F0B585B0002803D0012420466D
:10B1200005B0F0BD7822A14FB85C002803D0002400
:10B13000204605B0F0BD0492002905D038461430F1
:10B140000CC90CC01CC91CC00020F8661524204680
:10B15000FEF7D2FF204604F077F938681021C1616C
:10B1600004F0F6FC04463868C169C90607D504F046
:10B17000EFFC001BB98A8842F5D9386800E0B98A2B
:10B18000BA7D1207120B5218F97DCB07DB08D218D3
:10B190008B07DB0F5B05D218CB06DB0FDB05D21864
:10B1A0004B07DB0FDB06D2188B06DB0F5B07D218D1
:10B1B0000907C90F89071143016000240A212046AD
:10B1C00000F07EFB3220FFF76FF80821204600F0E8
:10B1D00077FB04F0BDFC05463868C169890606D4D2
:10B1E00004F0B6FC401BB98A8842F5D93868017D65
:10B1F0000A46C23A5342534174257B550904027DE5
:10B2000012025118007D0B180220032668A2314655
:10B2100005F028FD785D0128039619D1F87D02908C
:10B2200000260621304600F04BFB0721304600F097
:10B2300047FB012102988143785D012847D1386896
:10B240008901017506757521795C012938D048E0BE
:10B250000020032100F034FB04F07AFC0646386835
:10B26000C169890606D404F073FC801BB98A884240
:10B27000F5D93868007D46080122F87D0146314342
:10B280001640C90701D0304036D00295002506216E
:10B290002846019200F014FB07210095284600F093
:10B2A0000FFB019846400298385C012813D138689A
:10B2B000B1010175009901757521795C012910D1E1
:10B2C00014307621795C4A424A41510008E03868DE
:10B2D0000675490003E03868009901757100143063
:10B2E0000170374800687D21C900F4F7F3FE28217A
:10B2F0004143002000F0B6FA7720385C012803D1E2
:10B3000002200021FEF788FF04F022FC0646386880
:10B31000C069C00705D004F01BFC801BB98A8842B5
:10B32000F5D904F015FC06463868C169890706D5C9
:10B3300004F00EFC801BB98A8842F5D93868E249CE
:10B34000816117203856002829D57868002816D43E
:10B350000146039A91431C4A8B588507ED0EFF2640
:10B36000AE40B3438026AE401E438E501F210140A5
:10B370000120884015490860154908600FE08107E1
:10B38000C90EFF228A400F230340083B03988343E2
:10B390000C481D58954380228A402A431A500120A8
:10B3A000049978543861204605B0F0BD4C930102F1
:10B3B0006A656465635F69642025780D0A00000092
:10B3C00038E001021CED00E000E400E080E200E073
:10B3D00000E100E080B57C214143A6484218782373
:10B3E000D25C002A05D04058024941600F20FEF788
:10B3F0005BFF80BD008020B980B57C2141439D4822
:10B4000042187823D25C002A05D040580249416096
:10B410001E20FEF749FF80BD008020ABF0B593B041
:10B420007C270A9047439348C619980704D0F07DBB
:10B430004024044000D017E10125880E2ED0002BB7
:10B440002CD08120C004C01A884227D3099201223F
:10B45000EFF31084144002D1EFF3108072B630463F
:10B46000103005903069002506280891069310D801
:10B47000079414468440E106490F04D161210C422F
:10B4800003D0154604E0022502E00221059B196065
:10B49000079C002C00D162B6002D02D0284613B0C4
:10B4A000F0BD344617347348C05910210491C1616E
:10B4B0003746143704F04CFB05463068C069C006B7
:10B4C00005D504F045FB401B39888842F5D9207822
:10B4D000400665D40297B78C069C20463946F4F79F
:10B4E000F9FD079039464143601A039035462435EB
:10B4F000A74200D894E0039800281CD006210A9C9B
:10B50000204600F0DDF9288807994843089940183B
:10B510003168886000272046039C394600F0D0F946
:10B52000079B099A28885843C0193168097D11542E
:10B530007F1CA742F6D330680499C16104F008FB70
:10B540000446029D3068C069C00605D504F000FBC2
:10B55000001B29888842F5D904F0FAFA04463068BD
:10B56000C069C00705D004F0F3FA001B298888429F
:10B57000F5D904F0EDFA04463068C169890706D5AB
:10B5800004F0E6FA001B29888842F5D930680121C9
:10B59000059A1160B24981610025284613B0F0BDBB
:10B5A00003200025089FF7650999316606997166A1
:10B5B000B566F0660120C00731680A6802430A6078
:10B5C00006210A9C204600F07BF9306887602046FF
:10B5D000294600F075F93A4F0BAA0A921BCF1BC2FD
:10B5E0001BCF1BC2B48CF0680A99FEF7CDFEF06841
:10B5F0003168344A0092069A944200D31446A30854
:10B600001431099AFEF730FFB06E0019B066306E43
:10B6100000193066F06D0019F065284613B0F0BDD2
:10B62000002404E0641C0798844200D363E70621E9
:10B630000A9800F045F92888604308994018316855
:10B64000886000270A98394600F03AF928880028CF
:10B65000099AE7D0604310183168097DC1557F1CF5
:10B6600028888742F6D3DDE7034804A1064A07A3EA
:10B6700004F09CFA4C9301025C3C0100666C61731F
:10B68000685F726561640000C6030000546865204D
:10B69000444D412072656164206C656E677468205A
:10B6A00073686F756C6420626520746865206D75C1
:10B6B0006C7469706C65206F6620340D0A000000A0
:10B6C000D030010081AC0000000093EBF0B583B0F6
:10B6D0000D4604467C26464351488719F869B98CC3
:10B6E000F4F7F8FCA84200D894E0019502940121F7
:10B6F000EFF31080084002D1EFF3108272B63C469F
:10B7000010343B690025062B0CD80A469A40D30614
:10B710005B0F06D161231A4277D00D46002803D073
:10B7200003E00225002800D162B6002D02D0284691
:10B7300003B0F0BD00943C462434394880591021B0
:10B74000C1613E46143604F003FA05463868C06904
:10B75000C00605D504F0FCF9401B31888842F5D9B4
:10B760000621029D284600F0ABF82088019941434C
:10B77000B869091838688160172179563C46173432
:10B78000002909D5C16920220A43C2610121F96655
:10B79000890502680A4302600421284600F090F8F7
:10B7A000207840B22C4600250028C0D42B480068E1
:10B7B0007D21C900F4F78EFC20492D3141432046FC
:10B7C00000F050F804F0C4F904463868C069C007B6
:10B7D00005D004F0BDF9001B31888842F5D904F08A
:10B7E000B7F904463868C169890706D504F0B0F98D
:10B7F000001B31888842F5D938680121009A116010
:10B8000017498161284603B0F0BD0321216000285B
:10B810008AD08AE7034804A1084A09A304F0C6F9BC
:10B820004C9301025C3C0100666C6173685F736558
:10B8300063746F725F657261736500002B020000B4
:10B84000736563746F7220696478206973206F7602
:10B8500065722072616E67650D0A000038E00102B2
:10B86000000093EBF0B583B001917C22029042433B
:10B8700053498C182546143504F06AF9064602210E
:10B88000029800F01DF804F063F907462068C169CA
:10B89000890606D404F05CF9C01B29888842F5D9D2
:10B8A0002068007DC00708D06420FEF7FDFC04F08E
:10B8B0004FF9801B01998842E1D903B0F0BDC04621
:10B8C000F0B585B0049104467C2060433C490F18D4
:10B8D0003D46143504F03CF906463868C069C00797
:10B8E00005D004F035F9801B29888842F5D904F089
:10B8F0002FF906463868C069800705D504F028F995
:10B90000801B29888842F5D91421049B5943DC20E7
:10B9100060432C4A1018039002914018018A8268F3
:10B92000C47C7426BE5D012E0DD10191012B0299BC
:10B930000CD0012B0DD07526BE5D012E0ED0019EC0
:10B94000072B0ED10EE00E4602990BE00222012BCE
:10B95000F1D138247526BE5D012EF0D10326072BC8
:10B9600000D0019E184B334024069207D20A1219C8
:10B97000D218039B5958C907490C52184168CB0784
:10B980001B0CD218837C5B075B0BD218C068400786
:10B99000000A10183A685060002E0ED001290CD110
:10B9A00004F0D6F804463868C069800705D404F06E
:10B9B000CFF8001B29888842F5D905B0F0BDC046F4
:10B9C0004C93010218320100FF3F0000F0B59DB01A
:10B9D0000D460126890E2FD0002B2DD011928121EA
:10B9E000C9041093C91AA94226D30121EFF3108488
:10B9F0000C4002D1EFF3108272B67C220F904243CA
:10BA0000E74814928718384610303B690026062B09
:10BA10000DD80A469A40D3065B0F07D161231A421C
:10BA200000D16FE30E46002C03D003E00226002C69
:10BA300000D162B6002E02D030461DB0F0BD02909B
:10BA4000BD650021139179651098401E1290401930
:10BA5000B964B9690D916E1A1199B962FD623863C2
:10BA60007E63F98C0E913046F4F734FB0446B863DC
:10BA7000129830180E9E3146F4F72CFB109B011BD8
:10BA80004A1CF86339647A64139A0029194608D06D
:10BA9000704359190D9BC91A0A1A7443581B80190F
:10BAA0000119384648300E90384644300D903846DB
:10BAB00040300B9038462630059038465830139069
:10BAC000384654301290F9643A651498B4490858CD
:10BAD0001021C1613846143014903846503004901B
:10BAE0003D464C3504F034F804463868C069C00659
:10BAF00006D504F02DF8001B149909888842F4D962
:10BB0000F87D40060C9500D574E201230E98036081
:10BB10000D98016800290F9800D1CDE23A467432A1
:10BB20000A92DA0407921A0509921922520606921D
:10BB30000722D206089216E09A4800687D21C900C3
:10BB4000F4F7C8FA109941430F9C2046FFF78AFE8C
:10BB500020460C9D0E9A11684B1C13600D990968C4
:10BB60008B4200D9A8E20B9A1268012A55D0002A0C
:10BB700000D0A8E02E6812990C6813990D68062170
:10BB80001091FFF79DFE386885601198051903F044
:10BB9000DFFF04463868C069C00706D003F0D8FF4D
:10BBA000001B149909888842F4D903F0D1FF044698
:10BBB0003868C169890707D503F0CAFF001B1499CB
:10BBC00009888842F4D938680A990A78012A0899BC
:10BBD00000D00699012A099A00D0079A3346724C80
:10BBE000234013430B4371490B434360002EA3D002
:10BBF00003F0AEFF04463868C069800706D403F03E
:10BC0000A7FF001B149909888842F4D9386829785D
:10BC100001756D1C761EFAD18EE7012B00D0C7E0AE
:10BC20002E6812990C6813990D6806211091FFF780
:10BC300047FE386885601198051903F089FF0446AE
:10BC40003868C069C00706D003F082FF001B149952
:10BC500009888842F4D903F07BFF04463868C1693B
:10BC6000890707D503F074FF001B149909888842DF
:10BC7000F4D938680A990A78012A089900D00699F7
:10BC8000012A099A00D0079A3346474C23401343B0
:10BC90000B4346490B434360002E69D003F058FF25
:10BCA00004463868C069800706D403F051FF001BC2
:10BCB000149909888842F4D93868297801756D1C6F
:10BCC000761EFAD154E0012B00D0C9E02E681299FB
:10BCD0000C6813990D6806211091FFF7F1FD386883
:10BCE00085601198051903F033FF04463868C06970
:10BCF000C00706D003F02CFF001B14990988884266
:10BD0000F4D903F025FF04463868C169890707D5CF
:10BD100003F01EFF001B149909888842F4D9386883
:10BD20000A990A78012A089900D00699012A099AE5
:10BD300000D0079A33461C4C234013430B431B4946
:10BD40000B434360002E13D003F002FF0446386813
:10BD5000C069800706D403F0FBFE001B1499098814
:10BD60008842F4D93868297801756D1C761EFAD19D
:10BD70000C4800687D21C900F4F7ACF910994143E3
:10BD80000F9C2046FFF76EFD20460C9D2A68139BF2
:10BD9000196889181960129B196889181960D9E601
:10BDA0004C93010238E00102FF3F00000080800058
:10BDB0008B4200D0CEE604990E6812990C68139954
:10BDC0000D6806211091FFF77BFD3868856011989A
:10BDD000051903F0BDFE04463868C069C00706D0E7
:10BDE00003F0B6FE001B149909888842F4D903F0C9
:10BDF000AFFE04463868C169890707D503F0A8FE7D
:10BE0000001B149909888842F4D938680A990A787D
:10BE1000012A089900D00699012A099A00D0079AA8
:10BE20003346D44C234013430B43D3490B43436065
:10BE3000002E00D180E603F08BFE04463868C0690E
:10BE4000800706D403F084FE001B149909888842F9
:10BE5000F4D93868297801756D1C761EFAD16BE625
:10BE6000129A1268119CA618139A15688B425FD11A
:10BE700004990C6806210391FFF722FD386885605C
:10BE800003F066FE05463868C069C00706D003F0B7
:10BE90005FFE401B149909888842F4D903F058FECC
:10BEA00010900C9D3868C169890708D503F050FED1
:10BEB0001099401A149909888842F3D938680A9968
:10BEC0000A78012A089900D006991091012A099A46
:10BED00000D0079A2346A7490B40134310990B4300
:10BEE000A5490B434360002C14D003F031FE1090A1
:10BEF0003868C069800707D403F02AFE1099401AF9
:10BF0000149909888842F3D9386831780175761C0C
:10BF1000641EFAD19A4800687D21C900F4F7DAF866
:10BF2000039941430F9C2046FFF79CFC204611E6F5
:10BF300005990C8806210391FFF7C2FC38688560DB
:10BF400003F006FE05463868C069C00706D003F056
:10BF5000FFFD401B149909888842F4D903F0F8FDCD
:10BF600010900C9D3868C169890708D503F0F0FD71
:10BF70001099401A149909888842F3D938680A99A7
:10BF80000A78012A089900D006991091012A099A85
:10BF900000D0079A234677490B40134310990B436F
:10BFA00075490B434360002C14D003F0D1FD109071
:10BFB0003868C069800707D403F0CAFD1099401A99
:10BFC000149909888842F3D9386831780175761C4C
:10BFD000641EFAD16A4800687D21C900F4F77AF836
:10BFE000039941430F9C2046FFF73CFC20460599EE
:10BFF0000A88CCE65E4815A90A4678C878C278C88F
:10C0000078C20125E8073A68136803431360B868EB
:10C01000FEF7BAF902200026139C2168BA6AF96576
:10C020003A6610997966BE66F8660C980068129AAE
:10C030001168091811600E9B19684A1C1A60226861
:10C0400010182060002900D0F6E4109538466030C2
:10C0500013903C465C3438460830129006210F9805
:10C06000FFF72EFC3868216881600C9800681190F9
:10C0700003F06EFD04463868C069C00706D003F0BF
:10C0800067FD001B149909888842F4D903F060FD0C
:10C090000446109D3A68D069800707D503F058FD23
:10C0A000001B149909888842F4D93A687420385CD6
:10C0B00001282DD0E9042CE003F04AFD044638683D
:10C0C000C069C00706D003F043FD001B149909881E
:10C0D0008842F4D903F03CFD04463868C1698907F9
:10C0E00007D503F035FD001B149909888842F4D95F
:10C0F00038680121029A1160224981610026304688
:10C100001DB0F0BD04210160002C00D191E491E448
:10C110002905119C174B2340591801280C9D02D06A
:10C120001920400601E00720C006081812494018EF
:10C130005060002C0ED003F00BFD04463A68D06925
:10C14000800707D403F004FD001B14990988884276
:10C15000F4D93A682B681398016812980068074C64
:10C1600000941432FEF780F930461DB0F0BDC04691
:10C1700090300100FF3F000000808000CDAD000046
:10C1800038E00102000093EB3920C0000149096842
:10C1900008587047D8920102F0B5032920D8C0464C
:10C1A0007944097949008F4401080F150121814024
:10C1B0004F4B1B685963D96212E0012181404C4BFF
:10C1C0001B681963D9620BE001218140484B1B6851
:10C1D000596304E001218140454B1B681963996252
:10C1E00083004349CB18DA608A68002A29D14A685B
:10C1F000002A16D4032314469C43174BE558960790
:10C20000F60EFF27B740BD438027B7402F43E750C6
:10C210001F23134001229A40104B1A60104B1A60E2
:10C220000FE09307DB0EFF259D400F241440083CD0
:10C2300003229443074AA658AE4380259D403543C8
:10C24000A550012282400868026288681043886015
:10C25000F0BDC0461CED00E000E400E080E200E03C
:10C2600000E100E010B501242046FDF745FF20461F
:10C2700003F0EAF8002010BD012181401C4800684D
:10C2800042688A4342607047194909680968C14099
:10C29000012008407047C0460121814014480068D1
:10C2A00042680A4342607047012907D0002910D133
:10C2B000012181400F4802680A430FE001218140BB
:10C2C0000B4800684368002A0DD00B4343600161AE
:10C2D000704701218140074802688A430260044890
:10C2E0000068416170478B43436001617047C046FD
:10C2F000DC9301020801004070B5144E307800282C
:10C3000023D0134D2846FDF7CFFF032411A220466A
:10C31000214604F0A7FC2846FDF7C6FF12A22046DE
:10C32000214604F09FFC2846FDF7BEFF13A22046DD
:10C33000214604F097FC2846FDF7B6FF14A22046DC
:10C34000214604F08FFC0020307070BD3194010252
:10C35000C0C62D00244346474D53472C302C342C67
:10C36000302C310D0A000000244346474D53472C22
:10C37000302C332C302C310D0A000000244346476A
:10C380004D53472C302C322C302C310D0A0000003C
:10C3900024434647534156450D0A000080B5114AD3
:10C3A0001170114A10708001C90101430F480078D3
:10C3B000400108430E490978090101430D480078FE
:10C3C000C00008430C490978890001430B480078F4
:10C3D000400008430A4909780143C8B2F8F742FA15
:10C3E00080BDC046EC9E0102C69601021D9001026E
:10C3F000ACEA0102A1AD0102ED9E0102DFD2010211
:10C40000AC98010210B5054804680548006860430F
:10C410000449F3F775FE201A10BDC04674000040B1
:10C42000B4D4010240420F00012282400548002995
:10C4300003D00168114301607047016891430160B6
:10C440007047C04600010040124A072809D8800002
:10C450000F238340814019401068984308431060BF
:10C4600070470F280AD8800020380F23834081406E
:10C470001940506898430843506070478000403826
:10C480000F2383408140194090689843084390608F
:10C490007047C04634000040F0B54307DC0E072665
:10C4A000A640C3089D000E4BEF187D68B5433E1DA6
:10C4B000002908D035600122824001290CD118687A
:10C4C00010431860F0BD012181401868884318604E
:10C4D000A24015433560F0BD186890431860F0BD68
:10C4E0000C01004010B582B014460A46014604987B
:10C4F000009301900820234600F092F802B010BD8E
:10C50000B0B584B014460A46014608980225009545
:10C51000019302900720234600F052F904B0B0BD09
:10C5200070B500285BD031490A783149002A03D11F
:10C530004A68012313434B60428803881B049A18FE
:10C540000B46183B1A60828883891B049B180C4693
:10C550000C3C23600B46083B84681C604469032341
:10C560002340057CAD00EB188569AD072D0D5B19E7
:10C57000457C2D035B19C569AE07B60A9B19867CFD
:10C58000B6059B190E1F3360036A122B04D10724D2
:10C590000C60541EA2410AE0032C05D1012D03D8E2
:10C5A00007220A60012202E006220A600122114CE1
:10C5B000002525700F2464012034C57C6D022540C0
:10C5C0001B069B0BD218C3791B07DB0ED218807990
:10C5D0000007C00D101840191439086070BD0648D6
:10C5E00006A1862209A303F0E1FAC046E4CC0102C9
:10C5F00018100050E6CC0102CE4901006C73705F48
:10C60000656E67696E655F72756E0000506172617C
:10C610006D65746572206973206E756C6C00000026
:10C62000F0B58BB0109E34043ED00D46D64C214060
:10C63000012701977F06B9423CD111462140B942FA
:10C640003FD11C40BC4243D1119902AC0027E78185
:10C65000E780668027802782A774E1749908A1810A
:10C66000A908A1800A90099708970797900880B2B7
:10C6700004902046FFF754FFAA480078002801D014
:10C680000BB0F0BDAB480168C90708D10168C90704
:10C6900005D10168C90702D10168C907F3D07F48F5
:10C6A000019901700BB0F0BDB8480D49AF22C14BE4
:10C6B00003F07CFA0095B5480949B022754B03F0A8
:10C6C00075FA0092B1480649B122724B03F06EFA36
:10C6D0000093AE480249B2226E4B03F067FAC0469F
:10C6E000A4490100F0B58DB00392139E340446D0E6
:10C6F0000A46A54C2140012502956F06B94244D156
:10C7000003992140B94247D11C40BC424CD11499F5
:10C71000129D04ACE174294921820027E781E7805A
:10C72000668027809908A1819108A1800B95012D31
:10C7300001D16121CF43A7740C9002200A90099087
:10C740000398800880B206902046FFF7E9FE7548FE
:10C750000078002801D00DB0F0BD76480168C90707
:10C7600008D10168C90705D10168C90702D101686C
:10C77000C907F3D04948029901700DB0F0BD834854
:10C780000D49FB228B4B03F011FA00927F480A49B6
:10C79000FC22404B03F00AFA039800907B480649BC
:10C7A000FD223C4B03F002FA009378480249FE2236
:10C7B000384B03F0FBF9C046B14901008E8E0000F2
:10C7C000F0B58BB0119E340447D00D466E4C21401D
:10C7D000012701977F06B94245D111462140B94250
:10C7E00048D11C40BC424CD11299109F02ACE1745C
:10C7F000294921820021E181E18066802180990818
:10C80000A181A908A1800997012F01D0712100E021
:10C810006121C943A1740A900320089007909008F1
:10C8200080B204902046FFF77BFE3E480078002847
:10C8300001D00BB0F0BD3F480168C90708D10168BD
:10C84000C90705D10168C90702D10168C907F3D03A
:10C850001248019901700BB0F0BD4C480C49D5222B
:10C86000544B03F0A3F9009548480949D622094BD7
:10C8700003F09CF9009245480549D722054B03F087
:10C8800095F9009341480249D822024B03F08EF9F2
:10C89000C0490100EE49010086860000E6CC010295
:10C8A00010B582B014460A4601460020009301905C
:10C8B00004202346FFF7B4FE02B010BD10B584B0CB
:10C8C00014460A460146002000900193029004207D
:10C8D0002346FFF707FF04B010BD000070B50D46FA
:10C8E000064604242046FDF707FC204602F0ACFD76
:10C8F0000B4805600B480670002E0ED00A480168F0
:10C9000080220A437F218A430260012000030749F5
:10C9100008600749086007480460002070BDC046F1
:10C92000E8CC0102E4CC01020CE400E080E200E08B
:10C9300000E100E01C100050B0B582B01446024681
:10C940001148204001256D06A8420DD1180413D0CE
:10C9500017480160002000930190062011462346ED
:10C96000FFF75EFE02B0B0BD0094FF228C32074894
:10C97000074908A303F01AF9FF208C30421C034832
:10C9800003490C4B03F012F90300FCFFCE490100F0
:10C990009649010044737420616464726573732066
:10C9A000257820697320696E76616C6964000000E7
:10C9B000081000500C4A010080B582B00B460146B9
:10C9C00000200092019003200A46FFF729FE02B0E2
:10C9D00080BD0000002801D0042100E00221C64AE9
:10C9E0005172411E8841800103490A6840239A43DD
:10C9F000101808607047C04650A00050F0B583B0D2
:10CA000002912E49CD7A0E7B771987424FD908992A
:10CA10000191182545434126F604BF00BE19745BF9
:10CA200034490C4057033C199B07D90C6418324B0E
:10CA30001B681B7A745375196C880326B60326404D
:10CA40009B079B0C9B193F2404401819029CA306CA
:10CA50001B0DC0186880012A184E13D8707B142251
:10CA60004243307B5023434324011B199A18F37A25
:10CA7000C0181C234343D01880081E4A10400743A7
:10CA80000F432F800198686001F0B6FFA860E86846
:10CA90001A4908403030E860286908402721715C55
:10CAA0004018286100F008FF686103B0F0BDFF2264
:10CAB0008832034803A108A303F078F8ECD10102FF
:10CAC0005D4A01006D61635F63735F636F6E7374D2
:10CAD0007275637400000000435320696E646578CA
:10CAE000206973206F7665722072616E67650D0A2A
:10CAF00000000000FF070000489401020000F0FF62
:10CB00002820F04900220A547047C046F0B581B091
:10CB1000009314460D46074606263046FDF7ECFA0C
:10CB2000304602F091FC26211D4847540021017037
:10CB300041708171017181704171C170C1710222B6
:10CB40004272C16201634163816304734273C572BF
:10CB5000009A561C134A168001724120C00401211C
:10CB60004903F3F720FB502060432901081861199D
:10CB70008A00801818224A438018B2B24A438018AB
:10CB8000094940180949884204D200F0B7F800204A
:10CB900001B0F0BD064807A19A2209A303F006F8E8
:10CBA000ECD10102E8D101022800080201200802AC
:10CBB0005D4A01006D61635F696E69740000000089
:10CBC000454D206F766572666C6F770D0A00000028
:10CBD000BC48C179002901D001207047007A411E6C
:10CBE00088417047F0B583B002912A494B7B83425C
:10CBF00048D9CB7A0C7BE31818245C439B00E318DC
:10CC00004124E4041A1914240190054665430026C2
:10CC1000565100925519EE882E4F0B467A1C324021
:10CC20002D4E3688497A711A2C4E0E40B618EE8079
:10CC30003740997BEF80AA88294F17404A424A41E2
:10CC400091007918274A8918A980274F0F402D1D78
:10CC5000029801280AD125490E400921C9027118FC
:10CC600069800121C9037918298000E02F8001988B
:10CC7000444300980019074A918C4182118C01822B
:10CC800003B0F0BD3520C200034804A109A302F09F
:10CC90008DFFC046ECD101025D4A01006D61635F0A
:10CCA0006C696E6B5F646573635F636F6E737472E0
:10CCB000756374004C696E6B206465736320696EE4
:10CCC000646578206973206F7665722072616E6783
:10CCD000650D0A00FFFBFFFFE8D10102FF03000022
:10CCE00003D0FFFFE80F0000EF1F0000FF830000EC
:10CCF000D54A506391637047ECD10102F0B581B021
:10CD00004348CC21016003214160CF490A7BD30411
:10CD1000404C1B19CC7AA218541E1C4318235343B1
:10CD200092009A184B7B14255D43521992012243BD
:10CD3000012463061343436100228262C2620263DC
:10CD400042638263C26342650267334B1A605A6072
:10CD50009A60324B1A601A619A61DC61304C1C6235
:10CD6000304C251D1D6325460C3D5D632546283D41
:10CD70009D632D4EDE631C645C642C4D2F461C3776
:10CD80009F642746143FDF64103C1C65284C5C659B
:10CD9000284C9C650C369E67274CA5634035E5639F
:10CDA000DA651A665A669A66DA661A67234DDD678F
:10CDB00002258561224DC561C325AD03CD620A639D
:10CDC000D2435A601F4A1368FF25AB4326254D5DA9
:10CDD000AD072D0EEB1813601B4A102313601B4A7E
:10CDE0001360272260238B5419498160C16001615F
:10CDF00021607D210901016641661649C164164919
:10CE000041641649016400F047FD01B0F0BDC04621
:10CE100004A000500000F8FF94A0005034A100507E
:10CE2000FF185A0030040040041000401C2000404D
:10CE30005430004060400040B8A10050140014007D
:10CE4000FF3F3FFF04E400E080E200E000E100E09B
:10CE5000DC05DC053F0270020133D007D007D007A4
:10CE600070B5182002F0F0FA192002F0EDFA06244D
:10CE7000204602F0E9FA2046FDF73EF9D54C0025A0
:10CE800025706570A5712571A5706571E570607B71
:10CE900014214143207B50224243E37A1E01921920
:10CEA0005118C0181C22424389184120C004F3F7CE
:10CEB0007AF9E5712572FFF721FF70BD2921C54A76
:10CEC00050547047ECD10102F0B58BB00792089135
:10CED0000146C04FB8780991FFF784FE78793A7B14
:10CEE00079790691824200D89FE0FB7A9A1818233C
:10CEF000534392004124E10404915218D2187B7BE1
:10CF000014214B43D21850246043155801230A932F
:10CF1000DB022E469E4316504E4B2B4005937D7BE5
:10CF200003914D433E7B7443F97A0B011B195B1946
:10CF300071181C24029461435918A74B1B88069C46
:10CF40005C430919C904490D059BC91811501018F3
:10CF50000799416038787979089A00920322099BF1
:10CF6000FFF74CFDF87A397B09183878814263D98C
:10CF700083000993049AD45C0894F7212140D1548A
:10CF8000D1184D788E7836027619CB781B04F318B9
:10CF900007900A9886051E43330CCB70FB7A387BCA
:10CFA000BC784D709E4D3540039E6643C018029B71
:10CFB0004343981940029B4B03405C19200A887038
:10CFC000200CC870F023089D2B401B1D3D7B08954D
:10CFD000FE7A099D5355C8700620079A5043801960
:10CFE000089A801848701F22D20222400243100A79
:10CFF00088707879401C7871387B7979814201D3C7
:10D00000002179713978491C3970F97A0818397812
:10D01000884201D80020387028200A993954387A7B
:10D02000401C3872387A0BB0F0BDA7204200D148BE
:10D030000649074B02F0BAFDA72042007A32CD48DC
:10D040007249734B02F0B2FDECD101027D4A01003E
:10D05000264A010000F0FFFF0320000605490A6888
:10D0600082430A600A6802430A60034801210160A2
:10D070007047C0461C0000401CA0005080B5012035
:10D08000FDF7F0FA80BD0000F0B587B006930646C4
:10D09000504C607A504B1B88181A0C9DA84200DC3B
:10D0A00089E00F460592012E06D156480021C16243
:10D0B0000169554A89180160A0783146FFF792FD51
:10D0C000E078E178069A2B4600F0AEF82078E17817
:10D0D0000097002206923346FFF790FCE07A217B0E
:10D0E0000818217888426ED94120C2040491880032
:10D0F000815C0391F7250D40029285544549455CBA
:10D100004549465C360276194449475C3F04F619A6
:10D110000127BF0537433E0C4654E67A217BA378AE
:10D120003C4A85543E4D3D4014275F4389191C23DA
:10D130004B43D91949023B4B0B405D19290A364B29
:10D14000C1542E0C35494654F02703990F400599D8
:10D15000002900D13F1D217BE37A029A87542F4A90
:10D1600086540622049E7243D2185118294A8154CB
:10D170001F22D20215400D43290A274A8154E07824
:10D18000401CE070E07AE178814201D30699E170B9
:10D190002178491C2170217B08182178884201D808
:10D1A00006982070E079401CE071A07A401CA072C3
:10D1B000E07907B0F0BD3920C2001632074808A157
:10D1C00009A302F0F3FC3920C20004480F49104BB8
:10D1D00002F0ECFCECD10102E8D101025D4A010051
:10D1E0006D61635F747800004D4143205458206C9A
:10D1F000656E206973206F7665722072616E676557
:10D200000D0A00000804004090D00300934A01007A
:10D21000444A01000100080202000802030008025B
:10D22000FF07C0FF00F83F00F0B589B008930192F6
:10D2300004914F4DEF7A874200D891E0297B502628
:10D2400032464A434124E3040693D218CC19A10084
:10D2500051181822059254430A19697B1423079325
:10D260005943531802900001195804460390504A3C
:10D270000A40A97AC902511808988205D2088A186A
:10D280001A514C4911402A7B00965643384CE57A96
:10D290002C0106982418A719354E5419A5007D199C
:10D2A000059844432819747B079D6C430519049F16
:10D2B000D2194148048854432A19089CD204520DBB
:10D2C00051181D460398195000F000FB0146707A72
:10D2D000001902043E460CD080B2C000002900D1E3
:10D2E000801E029FA5214900F2F7F4FE1F21014094
:10D2F00001E00021029F38012818427983791B023E
:10D300009A18C3791B04D2182C4B1340437109049B
:10D310005918090CC171002C20D015483546064615
:10D32000007B009B4343F17A0A01069F3A43D218DF
:10D3300041188B00D218059B4B43D118727B079B79
:10D340005343C91840191C4A12884243881801994E
:10D35000884203D001992246F2F70CFF09B0F0BDD4
:10D36000FF225C32034804A109A302F01FFCC0465F
:10D37000ECD101025D4A01006D61635F74785F6406
:10D380006573635F636F6E7374727563740000001E
:10D390005458204445534320696E6465782069736E
:10D3A000206F7665722072616E67650D0A0000005D
:10D3B000FF0700E000F8FFFFE8D10102EFFFE00007
:10D3C0000168044A11604168516081689160C068D9
:10D3D000D060704780A0005082B0FCF783FB05202E
:10D3E00000252946FFF730F806202946FFF72CF8DC
:10D3F0000A202946FFF728F809202946FFF724F8D4
:10D400000124204603F0B0FD284603F0ADFDFCF7F3
:10D41000C4FB2046FCF798FB01F096FF01F08EFF5D
:10D420009748016897480068890308D403210907D1
:10D4300008402107884202D0FCF722FB06E0FBF7F8
:10D4400023FEFCF735FB0020FDF7FEFBFCF710FC8C
:10D450000025284604F0C8FE03268BA2304631463C
:10D4600003F000FC30462946FBF7ECF8F7F7F8FA32
:10D47000FAF7C8FAFEF7F6FEFCF76EFB88480830AC
:10D48000FCF70EF9F6F7CCFFF5F79AFEF7F775FA09
:10D4900020462146FEF782FFF9F7ACFCA202814943
:10D4A000814B2046009204F05DF801F02BFDFEF761
:10D4B00023FF03F033FD7D4A2046214602F012FA95
:10D4C0007B4802F03FFA0C20FEF7D6FE2146A54C21
:10D4D00020463830774A0191FCF754F87648FCF73B
:10D4E000BBFA7648FCF79AFACB4E08E0002001F030
:10D4F000B9FC01206B49009A6B4B04F033F80C2007
:10D50000FEF7C2FE2064A07800281AD16448807813
:10D51000002803D1F7F79CFA002812D0A07A01283E
:10D5200003D10220A072FAF7FFF8FCF7C1F9F7F770
:10D53000A3FAF6F79DFAF6F7CDFCFAF771FAFCF7C5
:10D5400095F9E07B002802D0E573F9F789FE0B20FE
:10D55000FEF79AFE5249097800280BD0002915D110
:10D560000198574908704E4908705648057003F0F5
:10D57000D5FC0BE0012909D149480570F5835048D5
:10D58000057001984F49087003F0A8FCFAF79EFE59
:10D590000420FEF779FE0746F6F798FC002F04D02A
:10D5A0002063F6F793FC606313E0216B401A0428B4
:10D5B00006D30198E071F6F789FC2063FAF776FB51
:10D5C000F6F784FC616B401A0B2802D360200199A6
:10D5D0003152708FF3F7A3F90146606AF3F722F92D
:10D5E000002808D1F08F012805D10220012101F087
:10D5F0000FFD00F06BF8F7F72BFA2074F5F796FCA7
:10D6000060740020F9F7DEFFA074E07A2E490978F3
:10D61000014300D073E70B20FEF736FE002800D050
:10D620006DE7F7F715FA002808D0F5F77FFC00281A
:10D6300004D00020F9F7C6FF00280BD118488078E5
:10D64000002803D1F7F704FA002803D0A0780028B7
:10D6500000D154E702F004FFEFF31080C00700D0C0
:10D6600044E7EFF3108072B6002001F0FBFB0120CD
:10D670000C49009A0C4B03F075FF62B63FE7C046B9
:10D6800018000040300001405557422073696D700A
:10D690006C65206578616D706C650D0A0000000096
:10D6A0001C900102E8CD01029D17010081F80000E5
:10D6B0007C3F0000F59300005DD700005D91000005
:10D6C0001890010219900102C6960102B0B502F04D
:10D6D000C7FEEFF310800124C00716D1EFF31080CE
:10D6E00072B60320124A014603F0BCFA0025284610
:10D6F0002946FEF753FE02F041F9204601F0B2FB45
:10D70000284602F055F962B6B0BD0320084A01462A
:10D7100003F0A8FA002528462946FEF73FFE02F04E
:10D720002DF9204601F09EFB284602F041F9B0BDDC
:10D73000543F0100014800687047C0460C0000409B
:10D7400081B080B581B0039303AB009302F004FF76
:10D7500001B080BC02BC01B00847000001480021B4
:10D760004162704798980102F0B581B000263046BA
:10D770003146FDF7CFFC0125AC022649264F304645
:10D780003A462346FDF74AFE3888244988423FD06E
:10D7900040203D5264203E5262203E5260203E5264
:10D7A0004422BE52BE83FE811D4ABA817E810A2276
:10D7B0003A81C822FA801B4ABA803980FD87BD872A
:10D7C0007821798702213987FD86FE8350217E5298
:10D7D00006213985F884FF20123078843A83873017
:10D7E000B884EFF3108072B630463146FDF792FCF4
:10D7F00000280CD12A0300263046064D2946FDF7A5
:10D80000E3FB054A304629462346FEF7DFF862B6B9
:10D8100001B0F0BD00E002043AA90102AA550000DF
:10D82000E1FF0000341200000020704710B5002412
:10D83000002809D0002905D003464A0003481946AC
:10D84000F2F798FC204610BDE04310BD4093010262
:10D85000014600200A2901DAC0437047014A1180BD
:10D860007047C046C89301020020704780B5018808
:10D87000064A11808178064A1170C178054A1170F4
:10D880000079FCF739F8002080BDC04632940102CF
:10D89000349401029CD2010204480549016015211B
:10D8A00009044160034981607047C0469C300040D4
:10D8B00041000800340007000748006840697047CD
:10D8C000FD20400004490968085C70470248006870
:10D8D0006221405C7047C0464894010210B506487A
:10D8E0000468064800686421F2F70AFC0221C94373
:10D8F0004143081910BDC046A0D20102A4D20102C2
:10D900000A491A220A600A4948704878FF21090228
:10D91000084A13688B43800380B2C0181060064821
:10D920002021016005480160002070477020004000
:10D930003894010204E400E080E200E000E100E04D
:10D94000F0B5A9B016460F460546C648002B02465C
:10D9500000D01A463921CC003D21C900511811913F
:10D960008242189206D001204202BE491898F2F76E
:10D9700001FC189A6120111913910E21119C0A9132
:10D98000A170002F0D9501D00A2100E00921592333
:10D9900017938300E17078427841139908703078CA
:10D9A00010901070F17AE17471785170B7789770B7
:10D9B000F178D1703579157174795471B1799171AB
:10D9C000F179D171317A1172717A5172B17A9172A1
:10D9D0007E1EF0B200210328169106D870B2800096
:10D9E000A1A210586A00805A1690179882001898C1
:10D9F000C0181490F81E022804D3012E084604D83B
:10DA00009D4800E09D48031918781290189DA818A9
:10DA100017902846303015902C4656346D208000E3
:10DA20002950974A974B149E33627262B362F26236
:10DA30003176F182139B597009229A70281841603F
:10DA40008160C1600161109880008F490858F3F728
:10DA50001FF8012F10900F9104D0022F05D17F21C4
:10DA60007E2004E07C217B2001E05B215A20159D73
:10DA7000A984207003200C90A080012666701F20CE
:10DA80000B90A8821820A8740A46083A179BDA76E9
:10DA9000169B129AD2184A439100189A9163B702C2
:10DAA000791E8B420E9109D97848608034206884B1
:10DAB0007748288277481399088339E07F2B10DD57
:10DAC000802B18D031028B421BD071028B4227D1A0
:10DAD0006E49618068846F4813990883CF20C00025
:10DAE00025E0202B17D0402B1AD1684860800420F5
:10DAF000688469481BE06548608006206884674840
:10DB000015E0624860801020688462481399088399
:10DB1000C520C0000BE0624860800220688404E0F9
:10DB200004206884812040006080FF200230288229
:10DB3000104600F005FF1298102806D0402808D1A2
:10DB400008201499C876072000E0042017998870EF
:10DB500002E017980C9981701898169A8078C11E67
:10DB600002290CD3022811D001280CD12672BA4206
:10DB700000D900266672BA4213D8F44812E00D208C
:10DB80000002119908800120800201E00C98000237
:10DB90002081BA4201D8EE4800E0FA201799886047
:10DBA0000EE0FA20179988601398007800281199E0
:10DBB00001D0E8484880E848139A1083E748088075
:10DBC000A88CF2F7C7FE0026E54B3246F2F74AFD75
:10DBD00002460B46E3493046F2F7ACFDE24B3246D3
:10DBE000F2F740FDF2F708FF0746E080DF493046D4
:10DBF000109A0F9BF2F79EFDDD4B3246F2F732FD95
:10DC0000F2F7FAFE78434042800B608116990E9835
:10DC1000814208D90C20149FB872D648179988837E
:10DC20001220189A0EE0480A189A149F01D00D206D
:10DC300003E0080A00D1DBE20A98B872CE481799CF
:10DC400088831220F872D078052844D87844007967
:10DC5000400087440227402C3339C848B881C8485F
:10DC60002FE0C046D8900102403001004030010052
:10DC70005030010050300100302D0100372D0100DF
:10DC80003075000010270000F02D01000502000093
:10DC9000FF060000040800000A040000360400002B
:10DCA00003020000B748F881B748388013E0B7484E
:10DCB000F881B7483882B74838600CE0B448B8817A
:10DCC000B5481799C88306E0B4487882B448B8804C
:10DCD0000B9800069064AE483881A748F880B14898
:10DCE00002882A84B0480078E874B0480078119F10
:10DCF0007875387D139000285ED0AD490A681023EE
:10DD0000DA413A600A794B79CF8867801B029A180A
:10DD10006A840A7A4B7A8F7AC87A0D7B65701B0207
:10DD20009A183B04D21800061018179FF860487B19
:10DD30008A7BCB7B3B77120210186081087C787756
:10DD4000487C149A9072887CD072C87C159B187499
:10DD5000087D5874487D11909874C87D0A7E12021F
:10DD600012181A84887DD87418464B7EC375887E35
:10DD7000CD7E2D022818B880087F4D7F2D022818EF
:10DD8000F880887FB877C87FF8772020085C149DDA
:10DD900028732120085C68732A20085C2A314D789A
:10DDA0002D0228188D782D044019C97809064018CD
:10DDB00018998864119801E0EB7DA87C7D498B70EF
:10DDC0000A8080001F38C882C883139800281FD09B
:10DDD00022227748825C034622335B781B029A1822
:10DDE0000A842422825C034624335B781B029A183F
:10DDF000CA842622825C034626335B781B029A186B
:10DE00008A832822825C2830407800028018888427
:10DE10006948032569A2294602F024FF189F387833
:10DE200014907B78B8780F90FA78B8791390F879D5
:10DE30001190387A1090787AB97A08900991009305
:10DE40000F980190029216980390129804901398DC
:10DE500005901198069010980790FAA2F848294664
:10DE6000149B02F0FFFE3D46643580212846F2F700
:10DE70009AF9B878C11E02290ED3012800D18FE18A
:10DE8000022800D0ABE11691149078787F2250439D
:10DE9000F7494018F74907E01691149078785B220B
:10DEA0005043F1494018F14941182846F2F762F908
:10DEB0000D9D1898C6870E34324602E0641C0F2A66
:10DEC0000ADA21780029F9D0491C8907C90F914045
:10DED0000E43C687521CF1E71699022907D31499FD
:10DEE000491E012900D97DE14279D24901E04279F8
:10DEF000CF4989180C78002D00D177E1C1790E91B6
:10DF0000032900D94AE14279062A00D979E1492159
:10DF1000890041181191E43010900E98401E129023
:10DF200019A800190F9000231392149403E0189875
:10DF3000290600D15AE1052A5AD8C0467A441279F6
:10DF400052009744455C728598ABC0468813000028
:10DF5000E20400000C080000060A0000040F0000A4
:10DF60000000104130C1BD41000070400000F04091
:10DF70000000D041120C0000140B0000121200002F
:10DF8000140E00000E160000130D00001216000003
:10DF90000E120000140B0E0A1208000010160000EA
:10DFA0000E0B000032940102349401029CD2010253
:10DFB000A8D20102A0940102010800004361736528
:10DFC00020706172616D65746572733A200D0A008C
:10DFD0001693DFB2002F04D019A801223946F2F7B8
:10DFE000DBF8002C00D191E019A8C019BB498AE0E8
:10DFF000E8B2022867D00027022867D06BE00E98AD
:10E00000022872D1E8B2022800D103461693DFB28B
:10E01000002F04D019A801223946F2F7BDF8002CD0
:10E0200074D019A8C019ACA16DE0E8B2022800D1E3
:10E0300004231693DFB2002F04D019A80122394619
:10E04000F2F7AAF8002C61D019A8C0199FA15AE0D4
:10E05000E8B2022800D106231693DFB2002F04D0C5
:10E0600019A801223946F2F797F8002C4ED019A8CA
:10E07000C01992A147E0E8B2022800D10C23169300
:10E08000DFB2002F04D019A801223946F2F784F834
:10E09000002C3BD019A8C019874934E0E8B2811E92
:10E0A0004A424A419700022804D119A80122394660
:10E0B000F2F772F8002C16D019A8C0197CA12246DC
:10E0C000F2F758F80FE00627022804D119A8012218
:10E0D0003946F2F761F8002C05D019A8C01980491B
:10E0E0002246F2F747F8169710E01693DFB2002F9A
:10E0F00004D019A801223946F2F74EF8002C05D0B9
:10E1000019A8C01973492246F2F734F83C193F2C7C
:10E1100005D80F98C0194021091BF2F744F812984E
:10E120000228189801D2002002E0C078411E8841E0
:10E1300015990870611E2E46E8B202280CD1179A74
:10E14000517019A9119AB8C9B8C2B8C9B8C2B8C92A
:10E15000B8C2B8C9B8C20DE0179A117019A9109ABF
:10E16000B8C9B8C2B8C9B8C2B8C9B8C2B8C9B8C2C3
:10E17000C10709D180073546149C139A169B00D419
:10E18000D5E602208543D2E6FE20354605401898A4
:10E19000149C139A169B290628D0CCE637A231E0AE
:10E1A0001691149078780B994143334808181F381A
:10E1B0006F21C9430D9D7A180378D427D35543782E
:10E1C000D827D3558378DC27D355002900D170E6B2
:10E1D000C378E027D3551031001D189FEBE70120CD
:10E1E000404A10E00024002D00D087E629B0F0BDA1
:10E1F00080290ED30F20B8721048179988831020F9
:10E2000020E525A20120014602F02CFD189829B036
:10E21000F0BD1020402904D3B8720849179B998398
:10E2200010E5B87204481799888314200AE5C0469F
:10E23000372D0100302D0100150F0000140B0000D8
:10E240000108000025642025642025642025642021
:10E25000256420256420256420256420256420254C
:10E26000642025640D0A0000195401001DF7FFFF0A
:10E27000314B010089FBFFFF215301007472785F6D
:10E280006D6F646520706172616D65746572206583
:10E2900072726F720D0A00004E73666420706172B4
:10E2A000616D65746572206572726F720D0A00008F
:10E2B000FFFFFFFF01FF0000F0300100FFFFFFFF45
:10E2C000FF0101FFFF01FF01FFFF01FFFFFFFF0152
:10E2D000FFFF01FFDC360100FFFF01FF10310100ED
:10E2E00060300100CF4A0100002800D101481D49DB
:10E2F00008607047D890010210B5002801D004468C
:10E3000001E018480468204600F006FC204600F0B2
:10E3100021F80B4841780B4A1A231360417040786A
:10E32000FF210902084A13688B438007000CC018BC
:10E3300010600648202101600548016010BDC046FC
:10E34000389401027020004004E400E080E200E024
:10E3500000E100E0F0B586B0002805D10148006872
:10E3600002E0C046489401023121C90004914118DD
:10E370008A791F231A40CD79ED06AD0DAA180D7AC2
:10E38000ED066D0C52194D7AED062D0B52198D7A52
:10E39000ED06ED095219CD7AED06AD0852194D7C06
:10E3A000ED075219BD4C22600A7B1A404E7BF606DF
:10E3B000B60DB2188E7BF606760C9219CE7BF60659
:10E3C000360B92190E79F606F60992194E79F60671
:10E3D000B608921962604A6AB14D2A40A2608A6A00
:10E3E0002A40E2602D22D20087183A7E1A40039319
:10E3F0007E7EF606B60DB218BE7EF606760C921933
:10E40000FE7EF606360B92193E7FF606F609921945
:10E410007E7FF606B60892190E7CF60792192261E5
:10E42000BA7F1A400597FE7FF606B60DB218049B18
:10E43000C35CDB065B0CD2184B78DB061B0BD218D7
:10E440008B78DB06DB09D218CB78DB069B08D21869
:10E450006261CA692A40A2610A6A2A40E2618A7C32
:10E4600001252A40CB7CDB079B0F9A180B7DDB072D
:10E470005B0FD2184B7D9B07DB0ED2188B7DDB0721
:10E480009B0ED218CB7D1B079B0D9A180B7E1B078A
:10E490009B0CD2184B7E5B06DB0A13438A7E520626
:10E4A00012091A43CB7E5B075B0813432362CA6AD7
:10E4B00062620A6BA2624A6BE2628A6B2263392251
:10E4C000D200835C1E462E4066635E425E41B3040A
:10E4D000AE04744F3C68B443E3183B6083185A7829
:10E4E0002A409C782407E40EA2188C8F6401A2189D
:10E4F0006D4C1440C98FC905490A0919DA78D20749
:10E50000120A89181A791207120989185A79D2073A
:10E51000D2088918FB4EB1639968F1639979049523
:10E520002940DA79D207920F51181A7B5207D20E7E
:10E5300089185A7BD206920D51189A7B5207D20C39
:10E540008918DA7BD206920B89181A7CD206520AF5
:10E5500089185A7C520792090A43997CC9064908CE
:10E5600051183164D97C039A11401A7DD206920D5C
:10E5700051185A7DD206520C89189A7DD206120B78
:10E580008918DA7DD206D20989187164197E0F24A0
:10E5900021405A7E120151189A7E12038918DA7EA0
:10E5A0001207120A51181A7F1207120989185A7F86
:10E5B00012078918B164997F01942140DA7F12070C
:10E5C000120E51183D22D200835C5B075B0D591877
:10E5D000841862781207520C8918A278D206120B9E
:10E5E0008918E278D206D2098918F16421790722C4
:10E5F0000A406179C9008918A2795206920B511814
:10E60000E2799207120B8918227AD2078A18BF4939
:10E610000A60627AA37A1B029A18E37A1B04D21862
:10E620004A60E289BA4B13400394228AD2049209C9
:10E63000D2188A6003463033598CB64A114002938F
:10E640009A8CD205D20A51185622825C1206891879
:10E65000B14D2960014656314A788C782402A218BF
:10E660008C8864056409A218CC78240712196A60A2
:10E67000CA880C7AA407A40BA2184C7A6407E40A8F
:10E680001219AA604989E960492189004118FF22CD
:10E690006632821800921035002207E000300040F8
:10E6A000FFFFFF0004040040FF3F000084186427C0
:10E6B000E65D03273E406523E35C9B071B0F9B1928
:10E6C0006626A65DB607B60EF3186726A65DB601E8
:10E6D000F318DBB26826A65DB607B60DF3186926F7
:10E6E000A65DB607360DF3186A26A65DB607B60C0A
:10E6F000F3186B26A65DB607360CF3186C26A65DDC
:10E70000B607B60BF3186D26A65DB607360BF318E1
:10E710006E26A65DB607B60AF3186F26A65DB60785
:10E72000360AF3187026A65DB607B609F3187126E7
:10E73000A65DB6073609F3187226A65DB607B608B9
:10E74000F3187326A45DA407E31808C51032802AC5
:10E75000ACD1019AD243704EB4180B783B404D783F
:10E76000AD072D0FEB188D78AD07AD0EEB18CD78FA
:10E77000AD01EB18DBB20D79AD07AD0DEB184D799E
:10E78000AD072D0DEB188D79AD07AD0CEB18CD79DC
:10E79000AD072D0CEB180D7AAD07AD0BEB184D7ACC
:10E7A000AD072D0BEB188D7AAD07AD0AEB18CD7ABE
:10E7B000AD072D0AEB180D7BAD07AD09EB184D7BAE
:10E7C000AD072D09EB188D7BAD07AD08EB18CD7BA0
:10E7D000AD07EB18A3641031121DBDD1009B197851
:10E7E0005A785207520D51189A78D207120D89188B
:10E7F000B164059B1968F164D97D5A6812025118F9
:10E8000031659968454A0A40998A490589187165B0
:10E81000D9683D4C2140B16519692140F165029EDE
:10E820003178049D294082785207120F5118C2791D
:10E830009207920E8918427A9207920D5118827AA5
:10E840009207120D8918C27AD207920C89189A7D04
:10E85000D207520C891872789207D20B8918B278B5
:10E860001207D20A8918F2781207D2098A182C499D
:10E870000A60327C737C1B071B0D9A18B37C9B06C5
:10E880009B0BD218F37C1B079B0AD218337DDB0647
:10E890005B09D218737DDB071B09D2184A60B27D71
:10E8A0002A40C38F5B009A188A60826CCA60C26C6F
:10E8B00022400A61F27D7F231340328C5204520AB7
:10E8C000D2184A6102698A614269CA6182690A6230
:10E8D000C2694A62026A8A62426ACA62826A0A63D8
:10E8E000C26A4A63039A927CD201121D0A64027AB8
:10E8F0003A40CA65808F074A10400866002006B07B
:10E90000F0BDC04600300040FFFFFF009C300040DB
:10E91000FF1F0000FF03000000400040FFFF1F003A
:10E920000020004004480068806B800803490968A3
:10E930004900401809307047489401021004004013
:10E9400010B52D21C9004118027A032A04D100799B
:10E95000002807D0082006E08378DA1E022A05D2B4
:10E96000032412E0142088601C203DE0012B02D11A
:10E97000C8228A6012E00479042C01D3462404E002
:10E98000032C01D1322400E014248C605B1E022B86
:10E9900004D3022A10D24279154B01E04279154B7B
:10E9A0009B181B78402B04D0102B06D11423442431
:10E9B00005E02A233E2402E04279342348244B8098
:10E9C0000C80022A06D0062A08D0052A08D118226F
:10E9D0004C2301E0142250230B8000E01C224A80CB
:10E9E000C078042803D1142048806420088010BD1A
:10E9F000372D0100302D0100424800687047C046A5
:10EA000010B53F4A107091703E49002813D05068ED
:10EA10000861042048619078FF2212023A4B1C687A
:10EA20009443800380B20019186001204007054A12
:10EA30001060364A106000200860354901220A60E3
:10EA400010BDC04680E200E03148002101602D4841
:10EA5000016802688A420BD0016802688A4207D0C6
:10EA6000016802688A4203D0016802688A42EFD1D5
:10EA70007047C046F0B581B021480178214D00298A
:10EA800011D08178FF2212021F4B1C689443890326
:10EA900089B209191960012149071C4A11604068AF
:10EAA0002861042068610127EFF31080384000904E
:10EAB00002D1EFF3108072B6154807602E682868FF
:10EAC000B04208D12868B04205D12868B04202D1CE
:10EAD0002868B042F3D0FDF795FC0446F1F71FFF1C
:10EAE0000C49F1F791FCF1F772FF3018B843286038
:10EAF0000098002800D162B6204601B0F0BDC046A3
:10EB000038940102180400401CE400E000E100E039
:10EB10007000004080096E45F0B591B0002801D129
:10EB2000C04800688778F91E022913D3012F21D02D
:10EB3000022F3CD11021CA43447821461939914211
:10EB40003DD800970125B94A28462946234602F0B8
:10EB500089F853E10821CA4344782146213991427A
:10EB600018D800970125B14A28462946234602F0C5
:10EB700079F843E10821CA43447821460939914292
:10EB800034D800970125A94A28462946234602F091
:10EB900069F833E1032F3CD0042F43D1C37801251A
:10EBA000042B00D02DE106462A02042343E0012570
:10EBB000A6A2284629463B4602F054F81EE1C37837
:10EBC0000125052B0AD806462A02284698401B2113
:10EBD000084230D10021052B08462ED0022000909B
:10EBE000914A2846294602F03DF807E10646C378D7
:10EBF0000021022B1ED3032B1CD0042B08460A46EF
:10EC00001BD001250095884A2846294602F02AF89B
:10EC1000F4E0C3780125032B00D0FAE006462A026F
:10EC2000032308E0012583A2284629463B4602F03B
:10EC300019F8E3E00A46012148020F9159218900A1
:10EC40007518FD21490071180291314662313F0566
:10EC5000D219641E1F2727405C013C19144304434A
:10EC600032795207D20C22432B789B065B0BD218C9
:10EC7000B379DB071B0B13436D4D2B60F279032334
:10EC800010931A40737A9B079B0E9A18B37A5B070E
:10EC9000DB0D9A18F37ADB079B0DD218337BDB0769
:10ECA0005B0DD218737B1B075B0CD218AA6032690C
:10ECB000EA6072692A61B2696A61F269AA61326ABC
:10ECC000EA61726A2A62B26A6A620F980870F06A30
:10ECD000A8623F20C4432C353046E4300F903046C4
:10ECE000E5300E903046E6300D903046E7300C901F
:10ECF0003046E8300B903046E9300A903046EA3032
:10ED000009903046EB3008903046EC3007903046A2
:10ED1000ED3006903046EE3005903046EF300490EE
:10ED20003046F03003903746F1373046F230F33654
:10ED30000F990A194021525C109B1A400E9B1B1917
:10ED40005B5C9B071B0F9A180D9B1B195B5C9B0759
:10ED50009B0E9A180C9B1B195B5C9B019A18D2B2F4
:10ED60000B9B1B195B5C9B079B0D9A180A9B1B193D
:10ED70005B5C9B071B0D9A18099B1B195B5C9B072F
:10ED80009B0C9A18089B1B195B5C9B071B0C9A1821
:10ED9000079B1B195B5C9B079B0B9A18069B1B1917
:10EDA0005B5C9B071B0B9A18059B1B195B5C9B0705
:10EDB0009B0A9A18049B1B195B5C9B071B0A9A18F9
:10EDC000039B1B195B5C9B079B099A183B195B5CB7
:10EDD0009B071B099A1803195B5C9B079B089A18F1
:10EDE0003319595C8907891802C51034A0D10298DB
:10EDF0000078042101430E48C1630025284611B064
:10EE0000F0BD04200090084A2846294601F02AFF58
:10EE1000F4E703200090044A2846294601F022FF27
:10EE2000ECE7C04648940102A44A0100EA4A010006
:10EE300000100040556E646566696E6564206D65FE
:10EE4000616E205052462025640D0A00496E76619D
:10EE50006C6964206D65616E205052462025640DFA
:10EE60000A000000B0B584B00446FAF7BFFE1F48A0
:10EE7000016800914168019181680291C068039026
:10EE8000FFF7E2FD00F0B4FD1948016804220A43CF
:10EE90000260184D6868A021002C01D1884300E071
:10EEA00008436860FF200230FBF7A6F8FBF7BEFCC2
:10EEB0000020FFF721FAFDF7D3FF6846FEF780FA3E
:10EEC0000D480168C907FCD00120800229688143F0
:10EED00029600A48FBF790F8FFF7CCFD4B49086022
:10EEE00000F0A4FDFAF788FE04B0B0BD80A0005089
:10EEF00010ED00E02C0000402C0200400102000058
:10EF00007047704780B50E490E480246083A1268AD
:10EF1000920000D4603142680A4342600A490A689C
:10EF200008239A430A60091F012252040A60032140
:10EF3000890402688A430260FAF78AFE80BDC046EF
:10EF4000200000802800004004020040B0B50320EB
:10EF500000072D490A6882430125680710180860D8
:10EF600000242046FFF7CDFF2046FFF7C9FFEFF34F
:10EF70001080284002D1EFF3108172B68021C9437E
:10EF8000224A53680B40536093680B409360D368E8
:10EF90000B40D36013690B40136153690B405361FD
:10EFA000002800D162B6B0BD70B50C460321090738
:10EFB000154A13680B4313600122EFF310811140CF
:10EFC00002D1EFF3108272B68025EA430F4B5E68E0
:10EFD00016405E609E682E439E60DD681540DD60D1
:10EFE0001D6915401D615D6915405D61002900D1F5
:10EFF00062B6002802D00120FFF783FF002C02D068
:10F000000120FFF77DFF70BD00040040E095010284
:10F010000D4A002907D001290BD101218140106838
:10F020008843106007E001218140106808431060A8
:10F0300001E001218140101F02680A430121C90734
:10F04000114301607047C04644000040032804D8C3
:10F0500040000649085A00B27047002000B27047CD
:10F06000032802D84000014A11527047D6D201024B
:10F070009E4908707047C04670B58AB00C46054678
:10F08000FF20FC30A8490E68315C59208000335CB9
:10F09000B278307808AE069609AE05960C4E049606
:10F0A0002126760603960B4E0296012601960E2621
:10F0B00000965B1CDBB2F6F75DFE0998F1F76EFC7B
:10F0C00028700898F1F76AFC20700AB070BDC0463D
:10F0D0000000204100000443F0B58BB00446457C9D
:10F0E000824800788249002822D000200880814A86
:10F0F0001080814B01269E761E830A907F480078FF
:10F100007F4E36786DB205957E4D04957E4D039504
:10F110000AAD02957D4D01950096F6F769FB0A9DB3
:10F12000112020567A497B4A00F032FC064626E040
:10F1300000260E806F4A16806F4B01209876188348
:10F1400009966E4800786E4F3F786DB205956D4D0B
:10F1500004956D4D039509AD02956C4D0195009791
:10F16000F6F746FB099D112021567F20C00500902F
:10F1700001900296664A674B3046F7F78DFC4320B4
:10F1800001062846F1F740F9F1F708FC08906248BB
:10F190000078002824D05120800060494A7D4243F5
:10F1A0008D185F480068A8642F46403750480078A3
:10F1B000B87450480078F874554800783875554848
:10F1C0000078787557480078F87550480069F1F76D
:10F1D000E5FBB87552484069E8644C4800686864CB
:10F1E000FF20FE3050490968085C3922D200891896
:10F1F000022812D303D04E48007801280DD14B4885
:10F200000660434800883A4A108042480088394ADC
:10F21000108009200790089605E04448089A02608B
:10F220003548C08B07900B780022002B01D0114687
:10F2300000E0D1430125002B01D0042300E0EB4383
:10F24000A67AAD1BEE175B1971416568AE0F277A80
:10F25000AD00ED195641677A3F1FF817ED1970415F
:10F260004000EE0F80196D00EB1848418001990EA7
:10F270004118980127239B02C31A91411D48058814
:10F280001B480088854201D00798421B1020205659
:10F29000C001194D2D8C032D07D1E468E5176D0AC7
:10F2A0006419E4150519EC170FE0E468E5176D0A19
:10F2B0006519EC17ED15C6174519744197B2002F63
:10F2C00000D03446002F00D00546581BA14113043E
:10F2D00009D012B2D2015242D31780185941089B6B
:10F2E000DA17C01A91410BB0F0BDC046CA930102B3
:10F2F00044AD010242AD0102A0940102C990010295
:10F30000C890010230A3010230A1010248AD010200
:10F3100092AD010290AD0102FCA6010234A40102EB
:10F320006420004040AD0102489401023CAD01025E
:10F33000A0AD0102C10D4002803070470120C0071E
:10F340001B4908607047C04610B519480068C107DE
:10F3500010D1810711D4410712D4010713D4C1067B
:10F3600014D4810615D4410616D48021084016D045
:10F3700031A215E001240FA213E0022411A210E033
:10F38000032414A20DE0042416A20AE0052419A205
:10F3900007E006241CA204E0072421A201E0254A7C
:10F3A00004090220032101F05DFC204610BDC04687
:10F3B0005C000040526573657420627920504F52A2
:10F3C0000D0A0000526573657420627920424F5225
:10F3D0000D0A000052657365742062792050494E11
:10F3E0000D0A0000526573657420627920574454F9
:10F3F0000D0A00005265736574206279204C4F43FA
:10F400004B55500D0A0000005265736574206279F7
:10F41000205357205265626F6F740D0A0000000080
:10F420005265736574206279205359535245510DCA
:10F430000A000000BA3C01005265736574206279CD
:10F4400020445644440D0A0001218140044A1F28EB
:10F4500002D010688843106010680843106070473D
:10F460001C000040F0B583B0029104469949F0F7C2
:10F4700031FE0546984901942046F0F72BFE974946
:10F4800046189749714300956F18964944186421AE
:10F490002046F0F71FFE3818A108471A9249204667
:10F4A000F0F72EFE381891494518914F05D4642184
:10F4B0003046F0F70FFE0C4614E0A6B26421304649
:10F4C000F0F708FEB7204000A20701D1002907D1BC
:10F4D000884B73430422D341874A934200D3401E92
:10F4E0000C464519009847430298068019200101EF
:10F4F0003046F0F7EFFD2A461F3A284600DB10465B
:10F50000019BFF18B30705D1002C03D01F2D05DA8E
:10F510000120C5E01F2D0BDA0120C1E005461D3D8D
:10F52000034600DB2B461C2808DC02201546B7E00A
:10F5300000290CD01C21451A0CD50CE019461F39A6
:10F54000184600DB08461F2B1DDA0320A8E01D210A
:10F55000451A00D42846002D08D401461F3902461A
:10F5600000DB0A461F2804DA032099E00220154632
:10F5700096E015461E3D104600DB28461E2A0CDA92
:10F5800004200D468CE005461E3D024600DB2A465F
:10F590001E280BDA04200D4682E001461F39024680
:10F5A00000DB0A461F280ADA052079E011461F39D8
:10F5B000104600DB08461F2A0BDA052070E01546CE
:10F5C0001E3D104600DB28461E2A0CDA06200D469A
:10F5D00066E005461E3D024600DB2A461E280BDA81
:10F5E00006200D465CE001461F39024600DB0A4654
:10F5F0001F280ADA072053E011461F39104600DBA6
:10F6000008461F2A0BDA07204AE015461F3D13461D
:10F6100000DB2B461F2A0CDA08200D4640E0054689
:10F620001F3D024600DB2A461F280BDA08200D4644
:10F6300036E019461E39184600DB08461E2B0ADA4A
:10F6400009202DE011461E39104600DB08461E2A0F
:10F650000BDA092024E01F28054601DB05461F3D83
:10F660001F280CDA0A200D461AE01F28054601DB88
:10F6700005461F3D1F2806DA0A200D4610E01E2D04
:10F6800005DB0C2004E01E2D06DB0C2005E00B2022
:10F690001E2D05DB1E3D03E00B201E2D00DB1E3D55
:10F6A000029EB070681CF070E12001013846F0F74E
:10F6B00011FD3071C0B211494143CC193C212046A3
:10F6C000F0F708FD70713B21C94341430819B0713F
:10F6D00003B0F0BD805101008033E101B2070000AA
:10F6E00093FEFFFFB107000070FEFFFFA7FA0A00BC
:10F6F00080AEFEFF295C8FC20BD7A300F0F1FFFFA5
:10F70000F0B581B00446FFF721FCA08A00280FD095
:10F71000FFF772F92249886122481C302CCC2CC09A
:10F720002CCC2CC02CCC2CC00020888201B0F0BD89
:10F73000E08A1B4FB882A169BA8A1B48F0F71AFD0C
:10F74000184D1C35204629464CC84CC14CC84CC1EC
:10F750004CC84CC1FFF750F9B8611248066AFFF770
:10F76000E1F8301A38632846FFF7B6FC06460D4626
:10F770000E48007DFFF76AFC0121F970617CB971C8
:10F78000396D491C396581B2C90B401800B2C117E7
:10F790004010301A38668D417D6601B0F0BDC0461C
:10F7A00030990102009A0102E0D201023C9001026C
:10F7B00070B50446FFF7CAFBA08A1B4E7082718A9F
:10F7C000002908D0B0820220707100203082FFF73B
:10F7D00013F9F06170BDE08A3082A169328A134862
:10F7E000F0F7C8FC2046FFF777FC05460C461048AA
:10F7F000007BFFF72BFC81B2C90B401800B2C11788
:10F800004010281A30668C417466FFF7F5F8B06135
:10F81000F06C401CF064FEF761F8F063FAF772F8E0
:10F8200030640120707170BDC896010278D3010266
:10F83000CA900102F0B581B0EFF3108072B60020DB
:10F840000146FBF767FC0446002803D062B6204659
:10F8500001B0F0BD01273A030025074E2846314686
:10F86000FBF7B2FBBB02054A28463146FCF7AEF86F
:10F8700062B6204601B0F0BD00E002043AA90102E0
:10F8800010B5164C607D002803D000202075FAF7D3
:10F89000FFFA13480078002801D0F8F74BFDF8F77D
:10F8A000BDFDF8F723F8F7F7B7F902F067F9012083
:10F8B000A075E17D8843E073481CE075FAF70CFB06
:10F8C000607D002803D000202075FAF7BFFAE07AA7
:10F8D000002801D0401EE07210BDC0469898010279
:10F8E0000095010270B514460D4606461120FAF740
:10F8F00003FC2448042101600C4804601E48056094
:10F900008660002E0DD0FF20000609490A68824358
:10F910000120C00710180860064808210160064849
:10F9200001601A200221FFF773FB70BDB8D40102F9
:10F9300000E400E080E200E000E100E00C49086043
:10F940007047C04610B5044609480068604309493D
:10F95000F0F7D6FB0019084948600A480022026007
:10F9600002460C3A4B6813600968016010BDC0463E
:10F97000B4D4010240420F000C9001020148002162
:10F98000016070472C10014000480047C100000092
:10F9900080B582B013460A4600900348011D034813
:10F9A000F7F726F802B080BDF4D4010268A0010286
:10F9B00080B503460220032109A201F053F9002873
:10F9C0000AD030B407252C02CD25641960434009C4
:10F9D0001238001FFDD830BC1E20FFF735FD80BD5A
:10F9E00073797374656D207265626F6F742578002A
:10F9F0003B480021016081684068401C534A1368FD
:10FA00005B0104D40029024609D00A4607E04D49AB
:10FA10000B685B1C0B6001214906116002464949D5
:10FA20004860801ACA688018C860704770B5454E33
:10FA300071682748821C91422AD2491E284A516087
:10FA400028490B680340032084071B190B60002121
:10FA500091601060FCF7D6FC054674682146F0F70B
:10FA600039FBF168491922464243891AF160A142E3
:10FA700004D3091B401CA142FBD2F1603168091874
:10FA80003160002803D03069002800D0804770BD65
:10FA900010481149E622114B00F088F810B50C49C6
:10FAA0008A1C90420DD2401E0D4A50600D480368DA
:10FAB0000B4003218C071B1903600020906011602C
:10FAC00010BD04480449E622044B00F06FF8C0461C
:10FAD000FFFFFF00913C0100AB3C0100773C0100BF
:10FAE00010E000E020ED00E0B0B50120EFF3108160
:10FAF000014002D1EFF3108272B6124A1368124C21
:10FB0000226864688506114800682840850E5D19E2
:10FB10002923DB006B43002C1D4606D1002809D1A8
:10FB20001E20684300290AD0B0BD121BD218551CF4
:10FB30000028F5D01D461E2068430029F4D162B686
:10FB4000B0BDC04624E0010214E000E004ED00E096
:10FB500080B50020FAF7DCFC404280BDB0B586B02D
:10FB6000104869460A4638C838C238C838C2002426
:10FB70002046FAF7D3FC03992046FAF769FD01986D
:10FB8000012803D00824002804D102E0042400281E
:10FB900000D104460220FAF7B7FAE04002490860B3
:10FBA00006B0B0BD3C2D010038E0010290B01C460B
:10FBB00005AB07C3EFF31080C00702D1EFF310804D
:10FBC00072B6EFF310800B9068460E907046089066
:10FBD00010AB0F93CF4F3E1D01200490C50230465D
:10FBE0002946224600F0B8FC00213154EFF303808F
:10FBF0000990EFF308800C90EFF309800D90EFF37C
:10FC000014800A9000F02CFC3868012833D80028B2
:10FC1000C14F00D0C14F2A20C1497A69920703D54C
:10FC20000A783A60401E491C0028F6D1B948041DE4
:10FC30002046F0F7CDFA002807D079698907FAD570
:10FC400021783960401E641CF5E70220B5497A69C5
:10FC5000920703D50A783A60401E491C0028F6D165
:10FC60002A20AF497A69920703D50A783A60401E84
:10FC7000491C0028F6D1FFF737FF0346AA4A304651
:10FC80002946FDF75DFD04463018291B089F3B1FE0
:10FC9000049A9343A5A2FDF753FD9E4909680129E3
:10FCA00066D8001900299C4C00D09C4C00280AD032
:10FCB0009849091D6269920703D50A782260401E9F
:10FCC000491C0028F6D10A209F496269920703D592
:10FCD0000A782260401E491C0028F6D10598F0F7EA
:10FCE00077FA002809D061698907FAD5059A117851
:10FCF0002160401E521C0592F3E702208949626987
:10FD0000920703D50A782260401E491C0028F6D1CC
:10FD10000A208EA16269920703D50A782260401EEC
:10FD2000491C0028F6D10698F0F752FA002809D0AD
:10FD300061698907FAD5069A11782160401E521C24
:10FD40000692F3E7022077496269920703D50A78A1
:10FD50002260401E491C0028F6D10A207EA162695B
:10FD6000920703D50A782260401E491C0028F6D16C
:10FD70007CA230462946079BFDF7E2FC65490968ED
:10FD800001290E9B1BD80029634900D06349002834
:10FD90000AD0604A121D4C69A40703D514780C6080
:10FDA000401E521C0028F6D102205E4A4C69A4076E
:10FDB00003D514780C60401E521C0028F6D16AA2AC
:10FDC00030462946FDF7BCFC04463018291B694A19
:10FDD0003B46FDF7B5FC4F490968012911D80019C8
:10FDE00000294D4900D04D4900280AD0494A121D2A
:10FDF0004B699B0703D513780B60401E521C0028EB
:10FE0000F6D15D4A30462946099F3B46FDF798FCEE
:10FE10000446F800C00FB900C90F7A00D20F009253
:10FE2000019102903019291BFB0F544AFDF788FC01
:10FE300004193019291B3F233B40514AFDF780FC30
:10FE400034490968012911D820180029324900D005
:10FE5000324900280AD02F4A121D4B699B0703D54F
:10FE600013780B60401E521C0028F6D1454A3046DC
:10FE700029460B9BFDF764FC04463018291B424AB7
:10FE80000A9BFDF75DFC23490968012911D8001977
:10FE90000029214900D0214900280AD01D4A121DFD
:10FEA0004B699B0703D513780B60401E521C00283A
:10FEB000F6D1364A304629460C9BFDF741FC0446F4
:10FEC0003018291B324A0D9BFDF73AFC114909688D
:10FED0000129114A0DD80019002908D00F4A06E05F
:10FEE0005169890703D531781160401E761C0028BE
:10FEF000F6D128490E98091AA94200D32946890843
:10FF000000F03AFE24480068002800D0804700F046
:10FF100045F8C04608E101020090014000A0014000
:10FF2000EB3C0100603F0100D43C01000D0A23239B
:10FF300023204153534552542040203078253038F7
:10FF400058202323230D0A00AE3D010046554E43A1
:10FF500054494F4E3A2000004C494E452020202065
:10FF60003A200000256400000D0A53503D2530382A
:10FF7000580D0A00733D0100893D0100953D0100C7
:10FF80007D3D0100323D0100413D0100503D010039
:10FF90005B3D010000F8020204E10102F74800683D
:10FFA000012811D8002801D00B4800E0FC480C21A2
:10FFB0000A4A01E0002907D043699B07FAD5137864
:10FFC0000360491E521CF5E71E20FFF73DFA00BFF3
:10FFD00000BF00BF00BFFAE700A00140DE3C010007
:10FFE0008AB00646E448B06600F03AFAFFF77CFDB6
:10FFF0000346E248041D01200590C502E04A204660
:020000040001F9
:100000002946FDF79DFB074608942018DB4C09950F
:10001000E91BF36C3F2206921340DAA2FDF790FB36
:100020002168012910D8C0190029DD4900D0DD4917
:10003000002809D0221D4B699B0703D513780B605C
:10004000401E521C0028F6D1F36BD7A2089C204614
:10005000099D2946FDF774FB0746291A2018336CC1
:10006000069A134007D1D8A2FDF76AFBC34C21685A
:10007000012907D917E0CEA2FDF762FBBF4C21682A
:10008000012910D8C0190029C54900D0C549002848
:1000900009D0221D4B699B0703D513780B60401EC6
:1000A000521C0028F6D10027CBA5B800305800908C
:1000B000089809992A463B46FDF742FB2168012929
:1000C0000FD80029B64900D0B649002809D0221D12
:1000D0004B699B0703D513780B60401E521C002808
:1000E000F6D17F1C0D2FE0D1736BBFA2089C204678
:1000F000099D2946FDF724FB074620189F4CE91B64
:10010000B36BBC4AFDF71CFB2168012910D8C0194C
:100110000029A34900D0A349002809D0221D4B691A
:100120009B0703D513780B60401E521C0028F6D1A4
:10013000336CB14A089C2046099D2946FDF700FB17
:100140000746326CD000C00F9100C90F5300DB0F7F
:10015000009301910290E019E91BD30FA74AFDF724
:10016000EFFA3246C619A019A91B1546136C069A58
:100170001340A34AFDF7E4FA80490968012911D820
:1001800080190029864900D0864900280AD07B4A78
:10019000121D4B699B0703D513780B60401E521C40
:1001A0000028F6D12E466B6C964A089C2046099D85
:1001B0002946FDF7C5FA07462018E91B0796B36CD8
:1001C000914AFDF7BDFA6D4A1168012910D8C0198E
:1001D0000029734900D07349002809D0121D4B69CA
:1001E0009B0703D513780B60401E521C0028F6D1E4
:1001F0000798426E042360215C2004931A400B464A
:1002000000D003460693002A00D00846079E3358C4
:100210007E4A089C2046099D2946FDF791FA07462B
:1002200006983358E019E91B794AFDF789FAC6198F
:10023000A019A91B079A536E76A2FDF781FA4F49C0
:100240000968022911D280190029554900D0554961
:1002500000280AD0494A121D4B699B0703D5137821
:100260000B60401E521C0028F6D10798C36C06464E
:100270006DA2089C2046099D2946FDF761FA0746B4
:100280002018E91B336D6B4AFDF75AFAC619A019FD
:10029000A91B079F7B6D68A2FDF752FA8619A0196A
:1002A000A91BBB6D67A2FDF74BFA34490968012908
:1002B000059C11D880190029394900D039490028F6
:1002C0000AD02E4A121D4B699B0703D513780B6089
:1002D000401E521C0028F6D10798476B5D4A974292
:1002E00037D2032087430026059CB00039580246C8
:1002F000049B1A43BA5808230343FB580C250543B3
:100300007D5900910192029303953B180898099931
:10031000514AFDF715FA1949096801290FD8002932
:100320001F4900D01F49002809D0089A4B699B0734
:1003300003D513780B60401E521C0028F6D11B2EEB
:10034000444A06D80798406B361DB10040189042C9
:10035000CBD30798406B111A099A914201D88908AA
:1003600000E0610200F008FC3C480068002800D072
:100370008047FFF713FEC04622224B4D08E10102E1
:10038000D43C01000D0A0D0A232323204558434580
:100390005054494F4E202564202323230D0A00008A
:1003A0000090014000A0014050433D2530385800E6
:1003B0002C20457863657074696F6E4E756D62654B
:1003C000723D25640D0A00002C205468726561643A
:1003D0004D6F64650D0A000052252D32643D2530B5
:1003E00038580D0A0000000053503D253038580D94
:1003F0000A000000733D0100893D0100953D0100A8
:100400007D3D0100323D0100413D0100503D0100B4
:100410005B3D01004558435F52455455524E3D25C2
:100420003038580D0A000000494353523D253038FA
:10043000580D0A00663D01005343523D253038589F
:100440000D0A00004343523D253038580D0A0D0A6D
:100450000000000000F80202163D010004E1010264
:10046000F0B583B0344D2C68012C06D8601E844151
:10047000204601F073FB0028FAD10120EFF3108130
:100480000140019102D1EFF3108072B62B48285A37
:100490002B49695A814245D02A68002A01D02A4E48
:1004A00000E0284E1F23DB020293284C022A27D2A9
:1004B00005E01046214AA85282B2914232D087B25A
:1004C000B9420A4600D8621C131A21482B5218045C
:1004D0000DD0E819001D9FB201E0002F07D073690D
:1004E0009B07FAD5037833607F1E401CF5E7A242D4
:1004F000DFD902981018DDE7304683B299420CD05C
:10050000024680B281420E4600D8661CA642F3D94C
:100510000298301883B29942F2D108496852B01A51
:100520000B4968520B48002129540198002800D13A
:1005300062B603B0F0BDC04608E101020A0800003F
:10054000080800000090014000A00140FF070000E3
:100550000C0800000F080000F0B58DB00793174697
:1005600000240C9409AA13C215E006986849EFF715
:100570004BFFF0F713FAC117401848406549EFF7F1
:10058000A9FD009509A806223346F8F7EDFDBDE068
:10059000002C00D5BEE138787F1C25280DD000281E
:1005A00000D1B7E10B9A511C0A9B9942F0D8099BE4
:1005B0009854641C0C940B91EAE708940025397850
:1005C00023390D2914D801207944097949008F4431
:1005D000090F0F0F0F0F0F0F0B0F060F0F0D054316
:1005E0007F1CECE70820FAE70420F8E70220F6E792
:1005F0003878014630390024092902D9264639467F
:100600000BE000260A2171430E18303E791C7878E1
:100610000246303A0A2A0F46F4D32E2817D14A1C34
:10062000487801463039092905D911464F1C25382B
:10063000532811D96AE000240A2161430C18303C88
:10064000511C50780246303A0A2A0A46F4D34F1C0D
:100650002538532800D959E04000C04678448088A6
:1006600040008744A0005300530053005300530040
:1006700053005300530053005300530053005300E2
:1006800053005300530053005300530053005300D2
:1006900053005300530053005300530053005300C2
:1006A00053005300530060005300530053005300A5
:1006B00053005300530053005300530053005300A2
:1006C000530053005300530053009800530053004D
:1006D0005300530053005300530053005300530082
:1006E000AD00B600530060005300590053005300A2
:1006F00053005900530053005300DE0053005300D1
:10070000BD005300D3005300530098000C9C3FE7FA
:100710000024744940420F00791C38780F46253870
:100720005328F3D898E70799C91D07208143086823
:1007300007914968F0F7C0F900210690F0F78EF8AC
:1007400000280BD10B99481C0A9A904206D8099AA6
:100750002D2353540899491C0C910B90079808308D
:1007600007900698F0F71AF90095C21781185140C2
:1007700009A822463346F8F7F7FC0B98411C0A9A61
:10078000914200D9F1E6099A2E2313540B910C984B
:10079000401C0C90E9E6079802C807900096019566
:1007A00009A8102239E00B98411C0A9A9142ADD851
:1007B000099A252313540B910C98401C0C90A5E723
:1007C0000B9A511C079C201D0A9B994239D907900E
:1007D0009CE7079802C80790009509A82246D3E62F
:1007E000079901C9079109990A9A089E02E0401CDD
:1007F000002E8BD40378002B88D00B9D6C1C944268
:10080000F5D84B55761C0C960B94F0E7079802C868
:1008100007900096019509A80A222346F8F742FDA1
:1008200074E7079B10CB102C079308D300202146B8
:10083000401C0A09FF291146FAD806280AD80820C0
:1008400009E02368099CA354089A521C0C920B914E
:1008500007905BE7401C069009230C980B9D0999B3
:1008600005910A9E04940DE0202104463046059E21
:10087000715506462046049C401C154601460891C9
:1008800000290AD45B1E0699994206D26A1CB2421C
:10089000EAD9089908910029F4D50C900B9508988D
:1008A000002800D532E70126082501E06D1E36013B
:1008B000022DFBD220463146EFF70CFC0F28F6D86C
:1008C0000C980590099803900A9806900B9D204675
:1008D0003146EFF7FFFB691C069A914204D908994B
:1008E000089100290CD511E00C4A125C039B5A5563
:1008F000089A521C0D46059211460891002905D40C
:100900007043241A3009102E0646E0D205980C9048
:100910000B95FBE620460DB0F0BDC046303001001F
:1009200070B588B00022032803D9D243104608B01E
:1009300070BD7F4CC34D2A510F4B104EEE5081239A
:100940001E010123AB5528602C1962600128EDD8E7
:1009500007930022069205920492032303930292C6
:1009600001920091411E8841694600F027FD024630
:10097000104608B070BDC04604080000FFC0FFC0AC
:10098000F0B583B00C460023D943012C56DB074653
:1009900002910126EFF31085354002D1EFF310806C
:1009A00072B65849584A505C002800D0A3E056540B
:1009B0005E48115A5E48105A0196F202161A814298
:1009C00040D832465218A24240DB00930295A6421C
:1009D000354600DB25464C490818001D39462A4695
:1009E000EFF7C8FBA642484E04DA7919621B301DA6
:1009F000EFF7C0FB4E48305A001981B24D4A914280
:100A000001D94D494018029D009B4949705230461A
:100A10004A4E805D002865D1EFF3108501980540AE
:100A200002D1EFF3108072B6374A4048115A40485D
:100A3000105A884232D1424813524FE00C462046A9
:100A400003B0F0BD42425218A242BEDA3B4A2E4EDB
:100A5000B25C002A0CD03A4AB25A51188AB2354CCC
:100A6000A242284C029F01D9334A8918304A02E039
:100A7000244C2F4A029F3355B152421A89B2884200
:100A800002D22C488018421C93B22F4801212FA279
:100A900000F0E8F83C46002DD1D128E0019F9755A1
:100AA000884201D82348401C421A90B2800A01D0E3
:100AB000019882022248144F3A52386801280DD812
:100AC000431E9841104B5918091D92B21D4B00F05E
:100AD0008BFE009B002801D00B488355002D029D02
:100AE00000D162B6074808490B54002DA7D162B661
:100AF000204603B0F0BD21200201044804A108A350
:100B0000FFF754F80E08000008E101022A3E010038
:100B100074726163655F6F757470757400000000B6
:100B20005452414345204255535900000A080000E1
:100B300008080000FF07000000F8FFFF0F08000092
:100B40000C080000910D010002FF00000D0A547214
:100B500061636520627566666572206973206675DB
:100B60006C6C2C206469736361726473202575203A
:100B700062797465730D0A00F0B587B005460026EA
:100B800006960596049603960296800701D007B054
:100B9000F0BD019102A8142126A2FCF7D1FD29493C
:100BA0000968012911D80029274900D027490028C0
:100BB0000BD002AA01E0002807D04B699B07FAD5A9
:100BC00013780B60401E521CF5E701990029DED016
:100BD000204C3746B8002B58D80724D0581EA042C6
:100BE00004D31B4818181C4A90421CD802A8142190
:100BF0001AA2FCF7A5FD13490968012911D800299B
:100C0000114900D0114900280BD002AA01E00028A8
:100C100007D04B699B07FAD513780B60401E521C16
:100C2000F5E7761C01997F1C8F42B0D2322ED1D3CA
:100C3000ADE7C0460D0A4261636B74726163653A49
:100C4000200D0A0008E101020090014000A00140CF
:100C5000FFFFFFFCFFFF0200FEFF010025303858B8
:100C60000D0A000081B0F0B5C4B00E4607464993A6
:100C7000812000012F49085C002845D00292012004
:100C8000050204A82946EFF78EFAFCB20021C843FA
:100C90000C2C3AD8721E032A37D82748005DB04280
:100CA000084632D3F80535D50021B8050DD404A87F
:100CB00001904018691AA20022A39B582E4AFCF703
:100CC0003FFD0198EFF784FA014678050ED404AF92
:100CD0007818691AB20029A3D218121F1368264A7D
:100CE000FCF72EFD3846EFF773FA0146029A04AE80
:100CF00070180C46691A49AB0393FFF72DFC0119D4
:100D00003046FFF73DFE00E0002044B0F0BC02BCDE
:100D100001B00847FEF7E8FE034604A8019007A2C9
:100D20002946FCF70DFD0198EFF752FA0146B80588
:100D3000BDD5CAE708E10102F15601002531307541
:100D4000207C2000CE3D0100243E01001E3E01001B
:100D5000FD3D0100C83D0100E93D0100173E0100D5
:100D6000103E01000B3E0100C13D0100D43D0100D9
:100D7000E43D0100B93D010065470100033E01006B
:100D8000EF3D0100F63D0100DA3D010000000000EA
:100D9000F0B581B00B460120EFF31084044002D17E
:100DA000EFF3108172B6990F07D0022001212DA216
:100DB000FFF758FF002C3DD141E02249224D00278A
:100DC0006F54224AAB5A224AAE5AF3189EB2F60A20
:100DD00001D0204E9B19AB52EFF31086064002D192
:100DE000EFF3108372B6AA5A1C4BEB5A934202D10E
:100DF00016482F521AE06854934201D8164B5B1CD8
:100E00009B1A99B2890A00D0830210482B52286895
:100E100001280BD8411E8841A918091D9AB2104B10
:100E200000F0E2FC002801D006482F54002E03D029
:100E3000002C04D001B0F0BD62B6002CFAD162B62D
:100E400001B0F0BD0F08000008E101020C0800002D
:100E50000A08000000F8FFFFFF0700000808000074
:100E6000910D010055415254204572726F72202538
:100E7000780D0A0010B50446FEF768F8A08A00282D
:100E800000D010BDFDF7B8FD034988628861486D48
:100E9000401C486510BDC0463099010210B504469B
:100EA000FEF754F8A08A002800D010BD0A4CA06CB0
:100EB000401CA064FDF7A0FD6062606C002805D0B6
:100EC000FDF79AFD60650020606410BDA069206593
:100ED0000120606410BDC046C896010210B50A200A
:100EE00000242146FBF7B0FA09202146FBF7ACFAB3
:100EF0000124204600F038F80E200421FBF7A4FA64
:100F00000549204600F05AFAA2021549154B204621
:100F100000F028FB10BDC046E0940102B0B50E20E1
:100F200000242146FBF790FA0D202146FBF78CFAAE
:100F30000124204600F018F80A2004252946FBF772
:100F400083FA09202946FBF77FFA2046F8F7FCFDD3
:100F5000A2020349034B204600F004FBB0BDC0468B
:100F6000E8CD01029D17010070B5012801D90120CB
:100F700070BD48224243734B9C58A5691F218D4385
:100F8000A5610625A5600F2525629C18A27C002A74
:100F900005D1627C002A02D1227C002A14D0636829
:100FA000002B11D4251D0B40012216469E400C4BF0
:100FB0001E60BFF34F8FBFF36F8F2B68002B03D4DE
:100FC0000B409A4007490A60002803D0012804D149
:100FD000092000E00820F9F787F80020A06170BD23
:100FE00080E100E080E200E0F0B585B00D460278D7
:100FF000E348C368934219D0446D944216D0836885
:10100000934203D0016D914200D07FE09B1A591E9C
:101010008B41049348215943032D46D14418E1697B
:1010200000294ED01C34002020606DE09B1A5A1E0F
:1010300093410493032D1AD1039548225A438418EF
:10104000A26B0121EFF310850D4002D1EFF3108761
:1010500072B6A7691026B743A761A669002E01D111
:1010600018342160002D00D162B6039D0CE04821A8
:101070005943421891691832302902D01168102959
:101080004CD1802111600022482159434018002191
:10109000816301628162243000210160002A33D023
:1010A00004A82946904705B0F0BD4218916918324E
:1010B000302902D01168202939D180211160002205
:1010C00016E00395E26B0126EFF31085354002D15F
:1010D000EFF3108172B6A1692027B943A161A1691C
:1010E000002901D118342660002D00D162B6039D7D
:1010F0004821594340180021C163C1624163303027
:1011000000210160002ACBD105B0F0BD00920E4A4B
:101110002E329C480D490E4BFEF748FD1068009397
:10112000019098480949084A0A4BFEF73FFD1068AC
:1011300000930190044A243292480449054BFEF77B
:1011400035FDC04604950102B1020000A63E010033
:101150007B3E01005F3E0100F0B585B00490482160
:101160000A464243864B9C58E6690F2535409A183B
:10117000167C002E31D04F2040026169014200D11F
:1011800085E0A06904218843A0610220206201203B
:1011900081076918D161D36BEFF31084044002D149
:1011A000EFF3108572B695692026B5439561956970
:1011B000002D00D173E010463C30002C00D162B607
:1011C00000240460D4625463303200201060002B8D
:1011D00063D004A8984705B0F0BD0C2D5DD8C0467B
:1011E0007D442D796D00AF4467586B580658A16354
:1011F0005858585806009569202D04D015461835C2
:101200002D68302D49D1156B566B3432AE4217D252
:101210006669360714D5646815686E1C1660484305
:101220001818C06A445504980C4644431A19156BA3
:10123000566B3432AE4203D21C5966693607EAD483
:101240001268AA4229D14143585882690524A24311
:1012500082615A18D36B0121EFF31080084002D14C
:10126000EFF3108472B694692025AC4394619469BD
:10127000002C02D114461834216014463C34002856
:1012800000D162B600212160D16251639CE70C2D30
:1012900000D176E7012D00D173E705B0F0BD15460A
:1012A0001835286010463C30002C00D187E787E7CE
:1012B0000420206205B0F0BD0120206205B0F0BD21
:1012C00008252562164618369569102D02D0356816
:1012D000302D4BD10396566A15462835976AB7428A
:1012E00028D1A06902218843A061936B0121EFF30B
:1012F0001080084002D1EFF3108472B6039E346868
:101300001027BC4334603468002C00D1316014468F
:101310003834002800D162B60021216029601162B2
:10132000243200201060002BB7D052E70220206248
:1013300005B0F0BD2A68B242AFD262699207ACD55F
:101340002A68561C2E6048431818006A805C20608A
:1013500004980A4642439D18AC6A6E6AB4429CD215
:1013600028359C5862699207EAD496E73168009064
:101370000191044804A1094A09A3FEF717FCC046DD
:1013800004950102453E0100756172745F697271D6
:101390005F68616E646C6572000000003D030000D0
:1013A0005561727420256420737461746520676FC1
:1013B00065732077726F6E6720256400F0B585B085
:1013C0000E460546022804D3002E02D1012005B0A6
:1013D000F0BD002D03D0012D08D1092400E0082420
:1013E0002046F8F789FE2046FEF72EF8482169438B
:1013F000E74A505883691F240294A343836106235C
:1014000083600F230193036257180023BB62BB6301
:10141000FB633B627B62FB623B63317F3974727FAB
:101420007A74B27FBA7404937B637368B268F468A9
:10143000920022435B1E032B0ED8C0467B441B79CF
:101440005B009F4401050307082304E0282302E012
:10145000182300E038231A43C260C907090F7269D4
:101460009201D2B28918B2699207920E8918491C6A
:10147000816079613169012901D122210161012D48
:101480005CD831680E2959D23846123003900324B3
:10149000002D01D0204600E004204C432D490E19B8
:1014A000B178F8F7B9FE3968CA6880251046284334
:1014B000C8602848005D73781B021818C862AA43E8
:1014C000CA60F8F7F1FE03980078002809D1384681
:1014D00011300078002804D13846103000780028F8
:1014E00027D07868002815D4032102468A431B4977
:1014F00053588407E40EFF26A640B343A5401D437E
:1015000055500299014001208840A24908601449C1
:1015100008600EE08107C90EFF228A40019C04404A
:10152000083C032084430C48235893438D401D43BB
:1015300025500120B861049805B0F0BD0248034968
:10154000DA22034BFEF732FB453E0100B83E0100B4
:10155000953E0100C42D01001CED00E000E400E018
:1015600000E100E0F0B58FB00E900125002900D118
:101570004BE0039304910592002A00D145E001213C
:10158000EFF3108201910A4002D1EFF3108172B69D
:101590004827029747437E49CE19B5690023302D6D
:1015A00023D831461831C0467D442D796D00AF44B3
:1015B00020242626262626262626262626262626D3
:1015C0005E26262626262626262626262626262683
:1015D00018262626262626262626262626262626B9
:1015E00018000223002A0CD00CE0402D01D0802DE1
:1015F00005D10123002A04D004E020240C60002A35
:1016000000D162B61D46002B02D028460FB0F0BDB7
:10161000002575630399F1630499F16205993163BB
:101620005B4CE35959691322D202114205D00621BD
:1016300099600F21196271699960317C00290CD081
:10164000F56109950895079506950D950B9502216D
:101650000A91012810D017200FE0717C9A690029A7
:101660002CD0952002439A6128460FB0F0BD30245B
:101670000C60002AC5D0C5E71920049F0C90706843
:10168000002805D41F21084001998140414801608C
:1016900014209861B06806A9F8F776FE0E980299B2
:1016A00041436018806861583B4A0092091D3A46E0
:1016B000059BF8F7D9FE28460FB0F0BD3436110669
:1016C00002D580218A439A6131680025059A9142AA
:1016D0002DD205955D694F214A0215421BD1E905BE
:1016E00002D4029CF24F0AE0596833685C1C3460F3
:1016F000029C6043EE4F3818C06AC1540E982146D0
:1017000041437E18736B346BA34238D234367B5816
:101710005D691542E3D002211962019EB107294398
:101720003546E34CEFF31082324006D008E02946FC
:10173000019EEFF31082324002D1EFF3108372B6B4
:10174000029B4343E01883692024A3438361836998
:10175000002B05D0002A08D0C26B002A0AD154E71A
:10176000034618331E60002AF6D162B6C26B002A07
:1017700000D14AE70EA8904728460FB0F0BD294691
:10178000059D019E3C46EFF310823240D5D0D7E74D
:101790000495010280E200E0E90F010080B501201C
:1017A00082020249024BFFF7DDFE80BDE8CD010257
:1017B0009D170100B0B582B079208400E54D285D09
:1017C00001A90870652080002818F2F793F92F20EE
:1017D000C000285829190122024BFFF7C3FE02B0AE
:1017E000B0BDC046B5170100F0B591B0109001260C
:1017F000002900D19BE003930591002A00D196E0D7
:1018000007900121EFF310800291084002D1EFF31D
:10181000108172B604924823069307994B43D64928
:10182000C9188D690026302D6ED80C461834AD00CD
:10183000374602A675593E46AF46C046111901000B
:10184000191901001D1901001D1901001D190100C0
:101850001D1901001D1901001D1901001D190100AC
:101860001D1901001D1901001D1901001D1901009C
:101870001D1901001D1901001D19010001190100A8
:101880001D1901001D1901001D1901001D1901007C
:101890001D1901001D1901001D1901001D1901006C
:1018A0001D1901001D1901001D1901001D1901005C
:1018B0001D1901001D1901001D190100AF190100BA
:1018C0001D1901001D1901001D1901001D1901003C
:1018D0001D1901001D1901001D1901001D1901002C
:1018E0001D1901001D1901001D1901001D1901001C
:1018F0001D1901001D1901001D1901000119010028
:10190000022600280CD00CE0402D01D0802D05D1FE
:101910000126002804D004E010252560002800D10D
:1019200062B6002E069D944F049C079802D0304664
:1019300011B0F0BD00268E62039A8A63059A0A628E
:101940004C620A7C002A0BD00C960B960A960996DC
:1019500008960E9602220D9201282DD018202CE018
:101960008A7C2831002A3BD00A68A24216D22B4634
:101970004343FA585469A40710D50868441C0C6006
:10198000F918096A085C10601098294641437A18D2
:1019900011462831936A526A9342E8D345437859F5
:1019A000816982220A438261304611B0F0BD302540
:1019B00025600028B4D0B4E71A200F90C86808A9A1
:1019C000F8F7E2FC109845437A597819C06839490C
:1019D000009105992346F8F747FD304611B0F0BD58
:1019E000FB589A69140602D58024A2439A610A68BA
:1019F0000026049882422ED25D694F22520215427F
:101A000007980AD002211962029EB10729431FE0FC
:101A100028315D6915423E46F4D137465C69A4071A
:101A200002D40699544E0AE00C68661C0E600699B2
:101A30004843514E3018006A005D186010984143C9
:101A4000735871188C6A4E6AB442E1D329463E46F7
:101A5000069D494F01E0314607985A6A002AFCD199
:101A6000EFF31082029B1A4002D1EFF3108372B69B
:101A70004543781983691024A34383618369002B4C
:101A800005D0002A09D0826B002A0BD14FE703460C
:101A90001833029C1C60002AF5D162B6826B002AC2
:101AA00000D144E710A89047304611B0F0BDC046C1
:101AB00004950102E90F0100B0B5264900684A68A3
:101AC000824202D10D1D002016E080228A588242F7
:101AD00003D10D46803501200EE0FC228A58824257
:101AE00003D10D46FC35022006E02F22D2008B5890
:101AF00083422ED18D1803207C2242438C18A0688B
:101B0000012814D0002824D140342046F2F7E1FB0C
:101B100001462046F2F7B3FB2046F2F7DAFB002835
:101B200017D006C828680C4BFFF75EFEB0BD4034E6
:101B30002046F2F7CEFB01462046F2F7A0FB2046F6
:101B4000F2F7C7FB002804D006C82868024BFFF74D
:101B50004BFEB0BD60BE0102B91A010048214143ED
:101B6000054842189269D20601D4002070474058B7
:101B700041690120084070470495010280B5114871
:101B80000078C00110490978890101430F480078A5
:101B9000400108430E490978090101430D480078C6
:101BA000C00008430C490978890001430B480078BC
:101BB000400008430A4909780143C8B2F2F752FECF
:101BC00080BDC046EC9E0102C69601021D90010236
:101BD000ACEA0102A1AD0102ED9E0102DFD20102D9
:101BE000AC980102F0B587B001460127022505280F
:101BF0003A4600D02A4600200929014600D0114665
